:100000002FC200005EC200005CC200005AC20000A5
:1000100058C2000056C2000054C2000052C2000084
:1000200050C200004EC200004CC200004AC2000094
:1000300048C200000C94CE6044C2000042C20000DE
:1000400040C200003EC200003CC200003AC20000B4
:1000500038C2000036C2000034C200000C94246D87
:1000600030C200000C94D3700C9409712AC20000B5
:1000700028C2000026C2000024C2000022C20000E4
:1000800020C200001EC200001CC200001AC20000F4
:1000900018C2000016C2000014C200000C942351C4
:1000A00010C200000EC200000CC200000AC2000014
:1000B00008C2000006C2000004C2000002C2000024
:1000C00000C20000FEC10000FCC100000C947E7163
:1000D0000C94B471F6C100000C9429720C945F72F8
:1000E000F0C100001037F0361E371E371E371E379E
:1000F0001E371E371E371E371E371E371E371E3758
:1001000026362D3634363B3640364936503667363D
:100110006A361E376E3671367336763690369236BC
:100120009936A036B336BA36C136716E746E636EC8
:10013000676E6D6EAB6E786E7C6E826E866E8A6E4A
:10014000906E946E986EAB6E9E6EA26EA66E084A0E
:10015000D73B3BCE016E84BCBFFDC12F3D6C7431DB
:100160009ABD56833DDA3D00C77F11BED9E4BB4C32
:100170003E916BAAAABE000000803F07634236B7DB
:100180009BD8A71A39685618AEBAAB558C1D3CB728
:10019000CC5763BD6DEDFD753EF6177231BF0000A3
:1001A00000803F08000000BE922449123EABAAAA7C
:1001B0002ABECDCCCC4C3E00000080BEABAAAAAA81
:1001C0003E00000000BF000000803F000000000073
:1001D000084178D3BB4387D1133D190E3CC3BD42C0
:1001E00082AD2B3E68EC8276BED98FE1A93E4C8071
:1001F000EFFFBE01C4FF7F3F0000000000000000D1
:100200000A0B02090C0D0E08070304010000000090
:1002100000000000000000000000000000000000DE
:10022000000000000000000000001211100000009B
:1002300000000000000000000000000000000000BE
:1002400000000000010210202008081020401020AB
:10025000408002010201080402010102040810208A
:100260004080804020100804020180040201804088
:1002700020100804020108040201010204081020F1
:10028000408001020408102040800505050507058F
:1002900008080808020202020A0A08080404040402
:1002A000010101010101010103030303030303032E
:1002B000040707070C0C0C0C0C0C0C0C02020202BD
:1002C00006060606060606060B0B0B0B0B0B0B0BA6
:1002D000000020002300260029002C002F003200FF
:1002E00000010000030106010901000022002500B1
:1002F00028002B002E00310034000201000005010F
:1003000008010B0100002100240027002A002D0015
:100310003000330001010000040107010A014E41D1
:100320004E494E495459494E46CDCCCC3D0AD7236F
:100330003C17B7D13877CC2B329595E6241FB14FB7
:100340000A000020410000C84200401C4620BCBEFC
:100350004CCA1B0E5AAEC59D7400407A10F35A0069
:10036000A0724E18090010A5D4E80000E8764817DE
:100370000000E40B54020000CA9A3B000000E1F5C3
:1003800005000080969800000040420F000000A089
:100390008601000000102700000000E803000000B4
:1003A000006400000000000A0000000000010000DE
:1003B0000000002C76D888DC674F0823DFC1DFAE51
:1003C00059E1B1B796E5E3E453C63AE6519976961A
:1003D000E8E6C28426EB898C9B62ED407C6FFCEFE3
:1003E000BC9C9F40F2BAA56FA5F490055A2AF75C11
:1003F000936B6CF9676DC11BFCE0E40D47FEF520C3
:10040000E6B500D0ED902E0300943577050080848A
:100410001E080000204E0A000000C80C333333339E
:100420000F986E12831141EF8D2114893BE655160A
:10043000CFFEE6DB18D1844B381BF77C1D901DA442
:10044000BBE424203284725E228100C9F124ECA135
:10045000E53D27002E293A503B71E67191720C2A36
:1004600011241FBECFEFD1E2DEBFCDBF00E00CBF35
:1004700012E1A0E0B2E0E4E1FCE001E00BBF02C069
:1004800007900D92A43AB107D9F728E1A4EAB2E1A6
:1004900001C01D92A437B207E1F714E0CEE5D4E025
:1004A00000E006C022970109FE010BBF0E948C7E6E
:1004B000C435D10780E00807A9F70E94BA790C94E7
:1004C000F9859ECD20E232E1FC013183208308953D
:1004D000089520E232E1FC01318320830C94C87935
:1004E000EF92FF920F931F93CF93DF938C01EB0159
:1004F0007A0141E060E08BEB94E10E94195660EADA
:1005000074E08BEB94E10E9420736C2FD7FD02C046
:100510006F5F01C0609541E08BEB94E10E9419563A
:10052000B8018BEB94E10E941273B701882777FD25
:100530008095982FDF91CF911F910F91FF90EF90B1
:100540000C949D6D2F923F924F925F926F927F928B
:100550008F929F92AF92BF92CF92DF92EF92FF92D3
:100560000F931F93CF93DF93CDB7DEB72E970FB6C0
:10057000F894DEBF0FBECDBF8C017E876D87DC0196
:100580004D915C91119712962D913C9113974217C2
:1005900053072CF4942F852FA901292F382FD80128
:1005A000149660E070E0CB01E2E0F0E0ED84FE84C0
:1005B000EE15FF0544F5CD90DD90C216D3065CF430
:1005C0004901AA2497FCA094BA2C680D791D8A1DB4
:1005D0009B1D960116C04C155D055CF44A01AA24CA
:1005E00097FCA094BA2C680D791D8A1D9B1DA6014D
:1005F00008C0EE24D7FCE094FE2C6C0D7D1D8E1DF2
:100600009F1D3196D3CF0E94617B6B017C016D856C
:100610007E8562507109882777FD8095982F0E940A
:10062000617B9B01AC01C701B6010E94957A6B0109
:100630007C012D853E85243131050CF4BFC0480175
:10064000412C512C3201A12CB12CD4016D917D9102
:100650004D01882777FD8095982F0E94617BA70127
:1006600096010E94CA799B01AC010E94F57C9B0116
:10067000AC01C301B2010E94CB792B013C01BFEF59
:10068000AB1ABB0AED85FE85AE16BF06F1F6BF01BB
:1006900061507109882777FD8095982F0E94617BB2
:1006A0009B01AC01C301B2010E94957A0E94A87D12
:1006B0004B015C0120E030E040E85FE30E94367CC3
:1006C00018160CF07BC018870F83212C312C1B824D
:1006D0001C821D821E821A821982AF81B8858D917B
:1006E0009D91B887AF839C01442737FD4095542FD7
:1006F00029873A874B875C87CA01B9010E94617BD1
:10070000A70196010E94CA792B013C0120E030E04C
:10071000A9010E94367C181624F0C301B20190583A
:1007200002C0C301B201A50194010E94917A87FF22
:1007300013C08B819C81AD81BE8129853A854B8513
:100740005C85820F931FA41FB51F8B839C83AD8391
:10075000BE833FEF231A330A49815A814F5F5F4FAF
:100760005A8349838D859E854817590709F0B5CF6F
:1007700020E030E040EC5FE3C501B4010E94F57C6D
:100780004B015C0195E0291631040CF49CCF6B8180
:100790007C818D819E810E94617B6B017C01B10116
:1007A000882777FD8095982F0E94617B9B01AC0183
:1007B000C701B6010E94957A6B017C01C701B601A1
:1007C0002E960FB6F894DEBF0FBECDBFDF91CF914E
:1007D0001F910F91FF90EF90DF90CF90BF90AF905F
:1007E0009F908F907F906F905F904F903F902F9051
:1007F0000895CF93DF93EC01FB01248135810E94A2
:100800006179CE01DF91CF91089526E00C944F706D
:10081000DC01ED91FC910190F081E02D1994EF92B3
:10082000FF920F931F93CF93DF931F92CDB7DEB745
:100830007C01FC0100811181C80169830E94F8815B
:100840006981681719F0C8010E940082C7010F90E2
:10085000DF91CF911F910F91FF90EF900895EF924C
:10086000FF920F931F93CF93DF931F921F92CDB7E9
:10087000DEB707EE12E1875E92417C01C701800F6F
:10088000911FF80161918F019A838983CE010196AE
:10089000C6DFF3E105331F0789F787EE92E10F907A
:1008A0000F90DF91CF911F910F91FF90EF900895DE
:1008B0000F931F93CF93DF931F921F92CDB7DEB795
:1008C0000BEF14E1F80160818EED93E09A83898348
:1008D000CE010196A4DFF80161818FED93E09A8348
:1008E0008983CE0101969BDFC8010F900F90DF91A5
:1008F000CF911F910F910895CF92DF92EF92FF92C7
:100900000F931F93CF93DF93CDB7DEB72C970FB61E
:10091000F894DEBF0FBECDBF6C017B018A0177FF6B
:100920000EC0E09440E06E2D8BEB94E10E941956CE
:1009300060EA74E08BEB94E10E9420733EC040E0DB
:1009400060E08BEB94E10E94195660EA74E08BEB57
:1009500094E10E94207340E060E08BEB94E10E9400
:1009600019560E946E6D28EE33E040E050E00E9480
:100970005A7EBA01A9012AE0CE0107960E94987713
:10098000BE01695F7F4FCE0101960E94217760E032
:1009900070E1CE0101960E948478BC018BEB94E15A
:1009A0000E941273CE0101960E945676CE010796E0
:1009B0000E945676E114F10431F040E06E2D8BEB8D
:1009C00094E10E941956B6018BEB94E10E941273D8
:1009D0000E946E6D6093B7147093B8148093B9142D
:1009E0009093BA14B801882777FD8095982F0E94BC
:1009F0009D6D2C960FB6F894DEBF0FBECDBFDF9174
:100A0000CF911F910F91FF90EF90DF90CF900895BD
:100A10004F925F926F927F92AF92BF92CF92DF928E
:100A2000EF92FF920F931F93CF93DF93CDB7DEB773
:100A30002C970FB6F894DEBF0FBECDBF5C017B01D3
:100A40006A010E946E6D0091B7141091B814209144
:100A5000B9143091BA1440908A0450908B0460907D
:100A60008C0470908D04040D151D261D371D06176E
:100A700017072807390708F06AC0F7FE0EC0E09490
:100A800040E06E2D8BEB94E10E94195660EA74E011
:100A90008BEB94E10E9420733EC040E060E08BEB62
:100AA00094E10E94195660EA74E08BEB94E10E9495
:100AB000207340E060E08BEB94E10E9419560E94A5
:100AC0006E6D28EE33E040E050E00E945A7EBA019D
:100AD000A9012AE0CE0101960E949877BE016F5FBE
:100AE0007F4FCE0107960E94217760E070E1CE0132
:100AF00007960E948478BC018BEB94E10E941273EC
:100B0000CE0107960E945676CE0101960E94567637
:100B1000E114F10431F040E06E2D8BEB94E10E9482
:100B20001956B5018BEB94E10E9412730E946E6D11
:100B30006093B7147093B8148093B9149093BA1457
:100B4000B601882777FD8095982F0E949D6D2C9681
:100B50000FB6F894DEBF0FBECDBFDF91CF911F91CE
:100B60000F91FF90EF90DF90CF90BF90AF907F906C
:100B70006F905F904F9008958F929F92AF92BF9227
:100B8000CF92DF92EF92FF920F931F93CF93DF9359
:100B90006C017B01EA0177FF0DC0DF91CF911F91BE
:100BA0000F91FF90EF90DF90CF90BF90AF909F900C
:100BB0008F9096CC0E946E6D00918A0410918B04E8
:100BC00020918C0430918D048090B3149090B414D3
:100BD000A090B514B090B614080D191D2A1D3B1D28
:100BE0000617170728073907A0F541E060E08BEBEF
:100BF00094E10E94195660EA74E08BEB94E10E9444
:100C0000207341E06E2D8BEB94E10E941956B601E2
:100C10008BEB94E10E9412730E946E6D6093B3148B
:100C20007093B4148093B5149093B614BE018827C2
:100C300077FD8095982FDF91CF911F910F91FF90B5
:100C4000EF90DF90CF90BF90AF909F908F900C94DB
:100C50009D6DDF91CF911F910F91FF90EF90DF90ED
:100C6000CF90BF90AF909F908F9008958BEB94E1C1
:100C70000C941356CF93DF93CDB7DEB72C970FB6F6
:100C8000F894DEBF0FBECDBF61EB74E0CE010796D6
:100C90000E94C1766DEA74E1CE0107960E947378D6
:100CA000BC01CE0101960E94217748EC50E06FEF25
:100CB0007FEFCE01019620DECE0101960E9456768E
:100CC000CE0107960E94567665EB74E0CE0107963A
:100CD0000E94C17667EA74E1CE0107960E9473789C
:100CE000BC01CE0101960E94217740ED57E06FEFE5
:100CF0007FEFCE010196F4DBCE0101960E9456767D
:100D0000CE0107960E9456768091D4149091D51406
:100D1000019719F46AEB74E002C069EC74E0CE014B
:100D200001960E94C17648EC50E06FEF7FEFCE0154
:100D300001966EDECE0101960E94567667ED74E054
:100D4000CE0101960E94C17640ED57E06FEF7FEF34
:100D5000CE010196C5DBCE0101960E94567667EE64
:100D600074E0CE0101960E94C17648EC50E06FEF2E
:100D70007FEFCE0101964CDECE0101960E945676A1
:100D800067EF74E0CE0101960E94C17640ED57E016
:100D90006FEF7FEFCE010196A3DBCE0101960E949B
:100DA000567664E075E0CE0101960E94C17648EC6B
:100DB00050E06FEF7FEFCE0101962ADECE01019663
:100DC0000E94567661E175E0CE0101960E94C176DF
:100DD00040ED57E06FEF7FEFCE01019681DBCE0152
:100DE00001960E9456766CE175E0CE0101960E9454
:100DF000C17648EC50E06FEF7FEFCE01019608DE40
:100E0000CE0101960E94567668E275E0CE01019609
:100E10000E94C17640ED57E06FEF7FEFCE01019663
:100E20005FDBCE0101960E9456768091D41490919A
:100E3000D514039719F469E375E002C064E475E022
:100E4000CE0101960E94C17648EC50E06FEF7FEF33
:100E5000CE010196DDDDCE0101960E9456766EE44C
:100E600075E0CE0101960E94C17640ED57E06FEF2C
:100E70007FEFCE01019634DBCE0101960E945676BB
:100E800069E575E0CE0101960E94C17648EC50E01C
:100E90006FEF7FEFCE010196BBDDCE0101960E9480
:100EA000567666E675E0CE0101960E94C17640ED69
:100EB00057E06FEF7FEFCE01019612DBCE01019676
:100EC0000E94567665E775E0CE0101960E94C176D4
:100ED00048EC50E06FEF7FEFCE01019699DDCE0137
:100EE00001960E94567660E875E0CE0101960E9458
:100EF000C17640ED57E06FEF7FEFCE010196F0DA5B
:100F0000CE0101960E9456768091D4149091D5140A
:100F1000029719F46DE875E002C06EE975E0CE0144
:100F200001960E94C17648EC50E06FEF7FEFCE0152
:100F300001966EDDCE0101960E9456766EEA75E04E
:100F4000CE0101960E94C17640ED57E06FEF7FEF32
:100F5000CE010196C5DACE0101960E9456766BEB62
:100F600075E0CE0101960E94C17648EC50E06FEF2B
:100F70007FEFCE0101964CDDCE0101960E945676A0
:100F800067EC75E0CE0101960E94C17640ED57E016
:100F90006FEF7FEFCE010196A3DACE0101960E949A
:100FA000567667ED75E0CE0101960E94C17648EC59
:100FB00050E06FEF7FEFCE0101962ADDCE01019662
:100FC0000E94567667EE75E0CE0101960E94C176CA
:100FD00040ED57E06FEF7FEFCE01019681DACE0151
:100FE00001960E94567664EF75E0CE0101960E944C
:100FF000C17648EC50E06FEF7FEFCE01019608DD3F
:10100000CE0101960E94567660E076E0CE01019610
:101010000E94C17640ED57E06FEF7FEFCE01019661
:101020005FDACE0101960E9456762C960FB6F894A0
:10103000DEBF0FBECDBFDF91CF9108954F925F927B
:101040006F927F928F929F92AF92BF92CF92DF92D8
:10105000EF92FF92CF93DF93CDB7DEB72C970FB609
:10106000F894DEBF0FBECDBF01DE6EE170E080E020
:1010700090E00E949D6D85ED93E10E94CB532B0182
:101080003C0162E370E080E090E00E949D6D85EDA0
:1010900093E10E945C534B015C0162E370E080E0ED
:1010A00090E00E949D6D60913802709139028091AC
:1010B0003A0290913B020E94617BAB01BC0185ED3D
:1010C00093E10E9468556B017C0162E370E080E06F
:1010D00090E00E949D6DC301B2010E94617B20E0FF
:1010E00030E048EC52E40E94957AAB01BC0122E06A
:1010F000CE0101960E94C477BE016F5F7F4F8DEADB
:1011000093E10E942977CE0101960E94567664E50C
:1011100070E18DEA93E10E9451786DEA73E183EB0F
:1011200093E10E940C7760E570E1CE0101960E9488
:10113000C1766DEA73E1CE0101960E947378BC011D
:101140008DEA93E10E940C77CE0101960E945676BB
:1011500062E370E080E090E00E949D6D6BE870E1DA
:1011600089EB93E10E943F7721E0B501A401CE0114
:1011700001960E94C477BE016F5F7F4F89EB93E1B8
:101180000E944B78CE0101960E9456766BE076E085
:1011900089EB93E10E94517821E0B701A601CE01CD
:1011A00007960E94C477BE01695F7F4FCE0101960A
:1011B0000E9421776BE17DE0CE0101960E94847848
:1011C000BC0189EB93E10E944B78CE0101960E940D
:1011D0005676CE0107960E9456766DEA73E1CE01EF
:1011E00001960E9421776FEA74E0CE0101960E9479
:1011F000847869EB73E10E947378BC0189EB93E119
:101200000E940C77CE0101960E94567663EB73E143
:10121000CE0101960E9421774AE050E060E070E044
:10122000CE01019669DBCE0101960E94567621E03F
:10123000B501A401CE0101960E94C477BE016F5F83
:101240007F4F8FEB93E10E942977CE0101960E9498
:1012500056766FEB73E1CE0101960E9421774AE04A
:1012600050E06FEF7FEFCE0101963AD9CE010196A3
:101270000E9456766FED8BEB94E10E94217361E141
:1012800076E08BEB94E10E94207321E0B701A60188
:10129000CE0107960E94C477BE01695F7F4FCE01E1
:1012A00001960E9421776BE17DE0CE0101960E94BC
:1012B0008478BC018FEB93E10E940C77CE010196FC
:1012C0000E945676CE0107960E9456766FEB73E128
:1012D0008BEB94E10E94127364E170E080E090E097
:1012E0000E949D6D8091AA13882331F068E572E019
:1012F00080E090E00E949D6D2C960FB6F894DEBFC2
:101300000FBECDBFDF91CF91FF90EF90DF90CF90D8
:10131000BF90AF909F908F907F906F905F904F9015
:101320000895CF93DF93EC018C819D81892B61F02F
:10133000BE0187E996E10E942B73BE0181ED97E122
:10134000DF91CF910C942B73DF91CF9108951F9370
:10135000CF93DF93CDB7DEB7A8970FB6F894DEBF73
:101360000FBECDBF182F8CEE93E10E940B4E811162
:101370000EC064E176E0CE0101960E94C176CE01F6
:101380000196CFDFCE0101960E945676A9C0BE011C
:101390006F5F7F4F8CEE93E10E94ED4C112309F4B7
:1013A00099C061E476E087E996E10E943B736BE6C1
:1013B00076E087E996E10E942073BE016F5F7F4F60
:1013C00087E996E10E943B736AE776E087E996E158
:1013D0000E9420734D855E856F8578892AE030E014
:1013E00087E996E10E94177469E876E087E996E15B
:1013F0000E94207349895A896B897C892AE030E0F0
:1014000087E996E10E94177468E976E087E996E13A
:101410000E94207320E030E040E251E4698D7A8D33
:101420008B8D9C8D0E94F57CAB01BC0122E030E0ED
:1014300087E996E10E94317567EA76E087E996E1EF
:101440000E943B736BEA76E087E996E10E94207385
:1014500020E030E040E251E46D8D7E8D8F8D98A1CB
:101460000E94F57CAB01BC0122E030E087E996E107
:101470000E94317567EA76E087E996E10E943B7346
:101480006AEB76E087E996E10E94207320E030E085
:1014900040E251E469A17AA18BA19CA10E94F57C54
:1014A000AB01BC0122E030E087E996E10E94317592
:1014B00067EA76E087E996E10E943B7369EC76E0A3
:1014C00087E996E10E943B7366E972E187E996E15C
:1014D0000E943B7364EF71E080E090E00E949D6D9C
:1014E000A8960FB6F894DEBF0FBECDBFDF91CF91A7
:1014F0001F9108954F925F926F927F928F929F9269
:10150000AF92BF92CF92DF92EF92FF920F931F9311
:10151000CF93DF93CDB7DEB7CA54D1090FB6F89495
:10152000DEBF0FBECDBF8C0166E972E1CE01CD9664
:101530000E94C17666E972E1CE01C7960E94C1762B
:10154000BE016F5F7F4F8CEE93E10E949E4E4D88EF
:101550005E886F88788CC98CDA8CEB8CFC8C8D8DD6
:101560009E8DAF8DB8A12B968CAF9DAFAEAFBFAFA8
:101570002B97C8010197039708F0E1C1A7019601D5
:10158000C301B20190580E943E7A2BED3FE049EC36
:101590005FE30E94CB792091340230913502409173
:1015A0003602509137020E94CB794B015C0120E05A
:1015B00030E0A9010E94917A87FD09C080929913B9
:1015C00090929A13A0929B13B0929C1310C02BED93
:1015D0003FE049EC50E4C501B4010E94CB7960932F
:1015E000991370939A1380939B1390939C138090FC
:1015F000991390909A13A0909B13B0909C132BED8D
:101600003FE049EC50E4C501B4010E94367C181655
:1016100084F42BED3FE049EC50E4C501B4010E9495
:10162000CA796093991370939A1380939B13909344
:101630009C1320E030E044E353E4609199137091EF
:101640009A1380919B1390919C130E94F57C2BED33
:101650003FE049E450E40E94957A609395137093BB
:10166000961380939713909398130E942E7B4AE0D1
:10167000CE018B960E946D776EEE76E0CE01859658
:101680000E94C176BE01655D7F4FCE0185960E94A6
:10169000737868EF76E00E948478BC018FEB93E169
:1016A0000E940C77CE0185960E945676CE018B96CD
:1016B0000E9456768090951390909613A090971361
:1016C000B090981320E030E044EB52E4C501B4013F
:1016D0000E94917A181694F020E030E040E05FE339
:1016E000C501B4010E94CB790E942E7B4AE0CE0155
:1016F0008B960E946D776FEF76E023C020E030E09C
:1017000044E353E4C501B4010E94917A1816A4F190
:10171000A501940160E070E884E393E40E94CA7933
:1017200060939513709396138093971390939813E7
:101730000E942E7B4AE0CE018B960E946D7762E07C
:1017400077E0CE0185960E94C176BE01655D7F4F30
:10175000CE0185960E947378BC01CE01CD960E9481
:101760000C77CE0185960E945676CE018B960E940C
:10177000567668E970E163C020E030E047E853E462
:10178000C501B4010E94917A181604F120E030E0FE
:1017900044E353E4C501B4010E94CA7920E030E07B
:1017A00040E05FE30E94CB796093951370939613AA
:1017B00080939713909398130E942E7B4AE0CE015A
:1017C0008B960E946D7762E077E01FC0A5019401BF
:1017D00060E070E084EB93E40E94CA7920E030E09E
:1017E00040E05FE30E94CB7960939513709396136A
:1017F00080939713909398130E942E7B4AE0CE011A
:101800008B960E946D776FEF76E0CE0185960E94F1
:10181000C176BE01655D7F4FCE0185960E947378CB
:10182000BC01CE01CD960E940C77CE0185960E9418
:101830005676CE018B960E94567665E077E0CE0113
:10184000C7960E943F77BE01635C7F4FCE018596AD
:101850000E9421774AE050E060E070E0CE0185967A
:10186000D7D8CE0185960E9456760E946E6D209143
:101870008A0430918B0440918C0450918D048090A7
:10188000B7149090B814A090B914B090BA14280D61
:10189000391D4A1D5B1D261737074807590708F4ED
:1018A00041C20E946E6D0E945F7B4B015C016091A2
:1018B0008A0470918B0480918C0490918D040E9415
:1018C000617B20E030E040E85EE30E94F57C2796F3
:1018D0006CAF7DAF8EAF9FAF27976091B7147091BB
:1018E000B8148091B9149091BA140E94617B9B0145
:1018F000AC0127966CAD7DAD8EAD9FAD27970E9454
:10190000CB799B01AC01C501B4010E94917A87FD9E
:1019100009C26FEA74E0CE0185960E94C176BE01CD
:10192000695C7F4FCE0185960E947378BC01CE0121
:10193000CD960E944B78CE0185960E945676C801BE
:101940000297029708F0C8C120E030E040E251E47D
:10195000C301B2010E94F57C4B015C0120E030E044
:1019600040E251E4C701B6010E94F57C6B017C01A5
:1019700020E030E040E251E42B966CAD7DAD8EADC1
:101980009FAD2B970E94F57C2B013C010E946E6D50
:1019900020913513309136134091371350913813FD
:1019A000621B730B840B950B0E945F7B20E030E081
:1019B0004AE754E40E94957AAB01BC0123E0CE01D2
:1019C0008B960E94C4776BE177E0CE0185960E94EA
:1019D000C176BE01655D7F4FCE0185960E9473780A
:1019E00060E070E10E948478BC018DEA93E10E947E
:1019F0000C77CE0185960E945676CE018B960E947A
:101A000056766DEA73E1CE0185960E9421776FEBE1
:101A100073E1CE0185960E947378BE01635C7F4FAF
:101A20000E947378BC01CE01CD960E940C77CE0146
:101A300085960E94567667E077E089EB93E10E94F5
:101A40003F7721E0B501A401CE0185960E94C477BD
:101A5000BE016B5D7F4F89EB93E10E944B78CE0115
:101A600085960E94567621E0B301A201CE018596AB
:101A70000E94C47721E0B701A601CE01C1960E9461
:101A8000C4776FEA74E0CE018B960E94C176BE01E6
:101A90006F5C7F4FCE018B960E9473786FEA74E083
:101AA0000E948478BE016B5D7F4F0E94737862E173
:101AB00077E00E948478BC0189EB93E10E944B7827
:101AC000CE018B960E945676CE01C1960E94567624
:101AD000CE0185960E945676A5019401C501B401F8
:101AE0000E94F57C4B015C01A7019601C701B6017C
:101AF0000E94F57C9B01AC01C501B4010E94CB7929
:101B00006B017C01A3019201C301B2010E94F57C2B
:101B10009B01AC01C701B6010E94CB790E94A87D50
:101B200060939113709392138093931390939413F3
:101B300066E177E089EB93E10E945178409191133F
:101B400050919213609193137091941321E0CE0100
:101B50008B960E94C477BE01655D7F4FCE0185964E
:101B60000E94217768EA76E0CE0185960E9484780B
:101B7000BC018FEB93E10E940C77CE0185960E9409
:101B80005676CE018B960E9456766FEB73E189EB09
:101B900093E10E944B78C0909113D0909213E09003
:101BA0009313F090941320E030E04AE754E4C70127
:101BB000B6010E94367C87FD29C020E030E04AE76C
:101BC00054E4C701B6010E94957AAB01BC0123E041
:101BD000CE018B960E94F277BE01655D7F4FCE01EC
:101BE00085960E94217769EA76E0CE0185960E946B
:101BF0008478BC018FEB93E10E940C77CE0185962F
:101C00000E945676CE018B960E94567620E030E6F2
:101C10004AE656E460919113709192138091931368
:101C2000909194130E94917ABE01635C7F4F87FF6D
:101C30004FC0CE0185960E9421776AE177E0CE0100
:101C400085960E94847869EB73E10E947378BC01E9
:101C500089EB93E10E940C77CE0185960E9456761F
:101C60000330110599F469EB73E1CE0185960E946A
:101C70002177CE01859655DBCE0185960E9456765A
:101C800066E972E189EB93E10E943F776DE177E0CD
:101C9000CE018B960E94C1766FEB73E1CE018B96DD
:101CA0000E947378BC01CE0185960E9421774AE09C
:101CB00050E06FEF7FEFCE0185960E947002CE015B
:101CC00085960E945676CE018B960E94567604C069
:101CD00089EB93E10E940C776AE070E080E090E08D
:101CE0000E949D6DCE01C7960E945676CE01CD967C
:101CF0000E945676C65BDF4F0FB6F894DEBF0FBE6C
:101D0000CDBFDF91CF911F910F91FF90EF90DF90AA
:101D1000CF90BF90AF909F908F907F906F905F908B
:101D20004F9008956FED8BEB94E10E942173BE01FB
:101D3000695C7F4F8BEB94E10E941273EACD8F9226
:101D40009F92AF92BF92CF92DF92EF92FF920F934A
:101D50001F93CF93DF9300D000D0CDB7DEB78C01B7
:101D6000C0900A02D0900B02E0900C02F0900D029D
:101D700020E030E040E450E4C701B6010E94367C28
:101D800018166CF420E030E04AE754E4C701B601CD
:101D90000E94F57C0E942E7B6B017C0106C080E3D3
:101DA000C82E85E7D82EE12CF12C0E94360640E0A3
:101DB00060E08BEB94E10E94195666E277E08BEBD2
:101DC00094E10E94207341E060E08BEB94E10E947B
:101DD000195667E377E08BEB94E10E94207364E689
:101DE00070E080E090E00E949D6D0E946E6D6093B7
:101DF00035137093361380933713909338130E94E2
:101E00006E6D8090351390903613A0903713B0907C
:101E10003813DC01CB0188199909AA09BB098C1573
:101E20009D05AE05BF055CF4C80164DB0E946E6DC4
:101E300064E170E080E090E00E949D6DE0CF0130B1
:101E4000110509F041C069EB73E183EB93E10E9456
:101E50000C770E94360663EB73E1CE0101960E9477
:101E600021774AE050E060E070E0CE0101960E94E8
:101E70007C04CE0101960E9456766FE377E0CE0196
:101E800001960E94C1764AE050E06FEF7FEFCE01ED
:101E900001960E947002CE0101960E94567660E57E
:101EA00077E0CE0101960E94C17669EB73E1CE0125
:101EB00001960E947378BC0189EB93E10E940C7734
:101EC000CE0101960E94567626960FB6F894DEBF94
:101ED0000FBECDBFDF91CF911F910F91FF90EF907B
:101EE000DF90CF90BF90AF909F908F900895CF924A
:101EF000DF92EF92FF92CF93DF9300D000D0CDB767
:101F0000DEB70E9436066EE170E080E090E00E944D
:101F10009D6D85ED93E10E945C536B017C0164E64D
:101F200070E080E090E00E949D6D6BE870E189EBCD
:101F300093E10E943F7721E0B701A601CE0101960F
:101F40000E94C477BE016F5F7F4F89EB93E10E94CF
:101F50004B78CE0101960E94567669EB73E1CE0173
:101F600001960E9421774AE050E060E070E0CE01E7
:101F700001960E947C04CE0101960E9456766FED78
:101F80008BEB94E10E94217369E877E08BEB94E19D
:101F90000E94207368E877E089EB93E10E94517812
:101FA000C092A113D092A213E092A313F092A413B3
:101FB00020E030E040EF51E4C701B6010E94367CDA
:101FC00087FD03C06BE877E054C020E030E040EDCF
:101FD00051E4C701B6010E94367C87FD1FC06BE942
:101FE00077E0CE0101960E94C1764AE050E06FEFA3
:101FF0007FEFCE0101960E947002CE0101960E94F1
:10200000567680919604882331F06CED75E080E07F
:1020100090E00E949D6D6BEA77E02BC020E030E0FD
:1020200040EB51E4C701B6010E94367C87FD03C036
:102030006BEB77E01EC069EC77E0CE0101960E9461
:10204000C1764AE050E06FEF7FEFCE0101960E942B
:102050007002CE0101960E945676809196048823E4
:1020600031F06CED75E080E090E00E949D6D68EDD0
:1020700077E0CE0101960E94C1764AE050E06FEF12
:102080007FEFCE0101960E947002CE0101960E9460
:1020900056766CE271E080E090E00E949D6D809148
:1020A0009604882331F068EE73E080E090E00E94AF
:1020B0009D6D26960FB6F894DEBF0FBECDBFDF91A3
:1020C000CF91FF90EF90DF90CF900895CF92DF9265
:1020D000EF92FF92CF93DF93CDB7DEB72C970FB679
:1020E000F894DEBF0FBECDBF69ED74E0CE0101965E
:1020F0000E94C1764AE050E06FEF7FEFCE0101967B
:102100000E947002CE0101960E94567660916E0484
:1021100070916F048DE194E10E945B6BE12CF12CD6
:1021200064E670E080E090E00E949D6D60916E0436
:1021300070916F048DE194E10E945B6B2FEFE21AC6
:10214000F20A23E0E216F1045CF32AE0E216F1045D
:102150001CF4892B29F703C0892B09F0D4C06091A6
:102160001F1470912014882777FD8095982F0E9466
:10217000617B6B017C016093A1137093A213809328
:10218000A3139093A41360911D1470911E148827BB
:1021900077FD8095982F0E94617B60939D137093CB
:1021A0009E1380939F139093A01321E0B701A60183
:1021B000CE0107960E94C4776BE870E1CE010196CC
:1021C0000E94C176BE01695F7F4FCE0101960E94D9
:1021D0007378BC0189EB93E10E940C77CE010196E4
:1021E0000E945676CE0107960E94567640919D1326
:1021F00050919E1360919F137091A01321E0CE0126
:1022000007960E94C47766EE77E0CE0101960E94A1
:10221000C176BE01695F7F4FCE0101960E9473783F
:10222000BC0189EB93E10E944B78CE0101960E949C
:102230005676CE0107960E9456766EE57DE089EBD4
:1022400093E10E94517866E972E1CE0101960E9405
:10225000C17644E150E060E070E0CE0101960E945A
:102260007C04CE0101960E9456766091A113709174
:10227000A2138091A3139091A4130E942E7B4AE095
:10228000CE0101960E946D77BE016F5F7F4F83EB99
:1022900093E10E942977CE0101960E94567640E094
:1022A00066E08BEB94E10E94195663EB73E18BEBD4
:1022B00094E10E9412736FED8BEB94E10E94217305
:1022C00061E176E08BEB94E10E94207360919D13B5
:1022D00070919E1380919F139091A0130E942E7B6A
:1022E0004AE050E08BEB94E10E94FA736EE57DE0EA
:1022F0008BEB94E10E94207364E670E080E090E054
:102300000E949D6D18C06CEE77E0CE0101960E9490
:10231000C1764AE050E060E070E0CE0101960E9494
:102320007C04CE0101960E94567667EF77E089EB38
:1023300093E10E943F772C960FB6F894DEBF0FBE54
:10234000CDBFDF91CF91FF90EF90DF90CF900895B8
:10235000CF92DF92EF92FF92CF93DF93CDB7DEB7AC
:102360002C970FB6F894DEBF0FBECDBF69ED74E0B9
:10237000CE0101960E94C1764CE251E06FEF7FEFF3
:10238000CE0101960E947002CE0101960E945676FF
:1023900060916E0470916F048DE194E10E945B6B1B
:1023A000E12CF12C64E670E080E090E00E949D6DED
:1023B00060916E0470916F048DE194E10E945B6BFB
:1023C0002FEFE21AF20A23E0E216F1045CF32AE0AE
:1023D000E216F1041CF4892B29F703C0892B09F0BC
:1023E00057C160911F1470912014882777FD809544
:1023F000982F0E94617B6B017C016093A113709305
:10240000A2138093A3139093A41360911D14709151
:102410001E14882777FD8095982F0E94617B60931A
:102420009D1370939E1380939F139093A01321E0AC
:10243000B701A601CE0107960E94C4776BE870E150
:10244000CE0101960E94C176BE01695F7F4FCE0129
:1024500001960E947378BC0189EB93E10E940C778E
:10246000CE0101960E945676CE0107960E945676BE
:1024700040919D1350919E1360919F137091A013F2
:1024800021E0CE0107960E94C47766EE77E0CE0188
:1024900001960E94C176BE01695F7F4FCE01019611
:1024A0000E947378BC0189EB93E10E944B78CE01C6
:1024B00001960E945676CE0107960E9456766EE5EA
:1024C0007DE089EB93E10E94517866E972E1CE01EB
:1024D00001960E94C17644E150E060E070E0CE01D8
:1024E00001960E947C04CE0101960E94567660916E
:1024F000A1137091A2138091A3139091A4130E9431
:102500002E7B4AE0CE0101960E946D77BE016F5F7F
:102510007F4F83EB93E10E942977CE0101960E94C1
:10252000567640E066E08BEB94E10E94195663EB2F
:1025300073E18BEB94E10E9412736FED8BEB94E1EE
:102540000E94217361E176E08BEB94E10E9420739D
:1025500060919D1370919E1380919F139091A01391
:102560000E942E7B4AE050E08BEB94E10E94FA73CC
:102570006EE57DE08BEB94E10E94207364E670E0F1
:1025800080E090E00E949D6D85EC93E10E94A4792B
:10259000C090A113D090A213E090A313F090A413C5
:1025A00020E030E040EF51E4C701B6010E94367CE4
:1025B00087FD03C067E178E054C020E030E040EDE3
:1025C00051E4C701B6010E94367C87FD1FC06BE94C
:1025D00077E0CE0101960E94C1764AE050E06FEFAD
:1025E0007FEFCE0101960E947002CE0101960E94FB
:1025F000567680919604882331F06CED75E080E08A
:1026000090E00E949D6D6BEA77E02BC020E030E007
:1026100040EB51E4C701B6010E94367C87FD03C040
:102620006BEB77E01EC069EC77E0CE0101960E946B
:10263000C1764AE050E06FEF7FEFCE0101960E9435
:102640007002CE0101960E945676809196048823EE
:1026500031F06CED75E080E090E00E949D6D68EDDA
:1026600077E0CE0101960E94C1764AE050E06FEF1C
:102670007FEFCE0101960E947002CE0101960E946A
:10268000567662E370E080E090E00E949D6D01C0AC
:102690002EDC2C960FB6F894DEBF0FBECDBFDF91B7
:1026A000CF91FF90EF90DF90CF900895CF92DF927F
:1026B000EF92FF921F93CF93DF93CDB7DEB7AA9728
:1026C0000FB6F894DEBF0FBECDBF182F882331F0B0
:1026D00066E972E187E996E10E943B7381E294E149
:1026E0000E94E25BBE016F5F7F4F81E294E10E9436
:1026F0007E5BCE010D967C01112321F166E278E02C
:1027000087E996E10E943B73FE0131966F01F60165
:1027100041915191619171916F0126E030E087E91B
:1027200096E10E9431756FEA74E087E996E10E94B4
:102730002073CE14DF0459F766E972E187E996E168
:102740000E943B7323E938E144E85FE369817A81C1
:102750008B819C810E94F57C6D877E878F87988B0B
:1027600022E430E645E85FE36D817E818F819885C4
:102770000E94F57C698B7A8B8B8B9C8B25E83BEEDA
:1027800041E95FE369857A858B859C850E94F57CAC
:102790006D8B7E8B8F8B988FB70181E294E10E94C5
:1027A0005E5B112309F48FC0B70181E294E10E94BE
:1027B0007E5B64E378E087E996E10E943B736E01FB
:1027C000F9E1CF0ED11CF7014191519161917191C5
:1027D0007F0122E030E087E996E10E9431756FEADF
:1027E00074E087E996E10E942073EC14FD0459F728
:1027F00066E972E187E996E10E943B736E01F5E2BA
:10280000CF0ED11C9601AE01495D5F4FBE01675DE1
:102810007F4F81E294E10E94CE5C61E478E087E939
:1028200096E10E94207369A57AA54AE050E087E905
:1028300096E10E94FA736FEA74E087E996E10E94DC
:1028400020736FA178A54AE050E087E996E10E94E5
:10285000FA736FEA74E087E996E10E9420736DA134
:102860007EA14AE050E087E996E10E94FA7366E9AA
:1028700072E187E996E10E943B73B70181E294E13E
:102880000E940C5D6EE478E087E996E10E94207377
:10289000F70141915191619171917F012AE030E0FE
:1028A00087E996E10E9431756FEA74E087E996E165
:1028B0000E942073EC14FD0459F766E972E187E980
:1028C00096E10E943B7361E070E081E294E10E9436
:1028D000F75B112389F067E578E087E996E10E94CC
:1028E000207381E294E10E94565D4AE050E0BC0111
:1028F00087E996E10E94017424E030E043E050E073
:1029000062E070E081E294E10E94045C1123E9F14D
:102910006BE678E087E996E10E9420739E012B5DCB
:102920003F4FAE01495D5F4FBE01675D7F4F81E262
:1029300094E10E94685D69A57AA54AE050E087E9C4
:1029400096E10E94FA736FEA74E087E996E10E94CB
:1029500020736FA178A54AE050E087E996E10E94D4
:10296000FA736FEA74E087E996E10E9420736DA123
:102970007EA14AE050E087E996E10E94FA7366E999
:1029800072E187E996E10E943B7365E070E081E2C5
:1029900094E10E94215C112389F067E878E087E9DF
:1029A00096E10E94207381E294E10E94AB5D4AE0CF
:1029B00050E0BC0187E996E10E94017466E070E096
:1029C00081E294E10E942E5C112389F06AE978E0AB
:1029D00087E996E10E94207381E294E10E94BD5D47
:1029E0004AE050E0BC0187E996E10E94017467E08B
:1029F00070E081E294E10E94315C112389F062EB86
:102A000078E087E996E10E94207381E294E10E94D8
:102A1000CF5D4AE050E0BC0187E996E10E94017475
:102A200068E070E081E294E10E943E5C112389F04D
:102A300068EC78E087E996E10E94207381E294E1F6
:102A40000E94E15D4AE050E0BC0187E996E10E9406
:102A5000017469E070E081E294E10E944B5C112313
:102A600089F060EE78E087E996E10E94207381E2C8
:102A700094E10E94F35D4AE050E0BC0187E996E1F1
:102A80000E9401746AE070E081E294E10E94585C67
:102A9000112389F06AEF78E087E996E10E942073BC
:102AA00081E294E10E94055E4AE050E0BC0187E9C2
:102AB00096E10E9401746BE070E081E294E10E9473
:102AC000655C112389F060E179E087E996E10E9475
:102AD000207381E294E10E94175E4AE050E0BC015D
:102AE00087E996E10E9401746CE070E081E294E174
:102AF0000E94725C112309F48FC069E279E087E9D2
:102B000096E10E94207381E294E10E94295E4AE0EE
:102B100050E0BC0187E996E10E94017461E479E02C
:102B200087E996E10E94207381E294E10E944E5F62
:102B3000682F70E04AE050E087E996E10E94017456
:102B400068E579E087E996E10E94207381E294E1EB
:102B50000E94525F682F70E04AE050E087E996E1FA
:102B60000E9401746FE679E087E996E10E94207384
:102B700081E294E10E94565F682F70E04AE050E0E5
:102B800087E996E10E94017466E879E087E996E1B9
:102B90000E94207381E294E10E945A5F682F70E0E6
:102BA0004AE050E087E996E10E9401746FE979E01C
:102BB00087E996E10E94207381E294E10E945E5FC2
:102BC000682F70E04AE050E087E996E10E940174C6
:102BD00068EB79E087E996E10E94207381E294E155
:102BE0000E94625F682F70E04AE050E087E996E15A
:102BF0000E94017461ED79E087E996E10E942073FB
:102C000081E294E10E94665F682F70E04AE050E044
:102C100087E996E10E94017461E081E294E10E94FB
:102C2000035F61E081E294E10E94085F61E081E27C
:102C300094E10E940D5F112391F062EE79E087E943
:102C400096E10E94207381E294E10E946A5F682FFE
:102C500070E04AE050E087E996E10E94017460E08C
:102C600081E294E10E940D5F112391F06BEF79E016
:102C700087E996E10E94207381E294E10E946A5FF5
:102C8000682F70E04AE050E087E996E10E94017405
:102C900061E081E294E10E94125F112391F065E10D
:102CA0007AE087E996E10E94207381E294E10E9434
:102CB0006E5F682F70E04AE050E087E996E10E947D
:102CC000017460E081E294E10E94125F112391F0AF
:102CD00061E37AE087E996E10E94207381E294E162
:102CE0000E946E5F682F70E04AE050E087E996E14D
:102CF0000E94017461E081E294E10E94175F112358
:102D000091F06EE47AE087E996E10E94207381E217
:102D100094E10E94725F682F70E04AE050E087E91A
:102D200096E10E94017460E081E294E10E94175FE5
:102D3000112391F06AE67AE087E996E10E94207318
:102D400081E294E10E94725F682F70E04AE050E0F7
:102D500087E996E10E94017461E081E294E10E94BA
:102D60001C5F112391F067E87AE087E996E10E9401
:102D7000207381E294E10E94765F682F70E04AE060
:102D800050E087E996E10E94017460E081E294E1FD
:102D90000E941C5F112391F063EA7AE087E996E1D3
:102DA0000E94207381E294E10E94765F682F70E0B8
:102DB0004AE050E087E996E10E94017461E081E217
:102DC00094E10E94E55E61E081E294E10E94EA5EA6
:102DD00061E081E294E10E94EF5E60E081E294E1D3
:102DE0000E94F45E60E081E294E10E94F95E60E09E
:102DF00081E294E10E94FE5E112309F490C060EC30
:102E00007AE087E996E10E94207381E294E10E94D2
:102E10007A5F682F70E04AE050E087E996E10E940F
:102E2000017468ED7AE087E996E10E94207381E2FF
:102E300094E10E947E5F682F70E04AE050E087E9ED
:102E400096E10E94017466EF7AE087E996E10E94BC
:102E5000207381E294E10E94825F682F70E04AE073
:102E600050E087E996E10E94017464E17BE087E924
:102E700096E10E94207381E294E10E94865F682FB0
:102E800070E04AE050E087E996E10E9401746DE24B
:102E90007BE087E996E10E94207381E294E10E9441
:102EA0008A5F682F70E04AE050E087E996E10E946F
:102EB000017466E47BE087E996E10E94207381E279
:102EC00094E10E948E5F682F70E04AE050E087E94D
:102ED00096E10E9401746FE57BE087E996E10E942C
:102EE000207381E294E10E94925F682F70E04AE0D3
:102EF00050E087E996E10E94017462E77BE087E990
:102F000096E10E94207381E294E10E94965F682F0F
:102F100070E04AE050E087E996E10E94017460E0C9
:102F200081E294E10E94215F40ED5FE069E470E49A
:102F300081E294E10E94645E112309F449C067E8CC
:102F40007BE087E996E10E94207381E294E10E9490
:102F50003B5EAB01BC0122E030E087E996E10E94D4
:102F600032756BE97BE087E996E10E94207381E28C
:102F700094E10E949F5E4AE050E0682F87E996E165
:102F80000E94337462EB7BE087E996E10E94207334
:102F900061E081E294E10E949A5F682F70E04AE06C
:102FA00050E087E996E10E9401746AEC7BE087E9D2
:102FB00096E10E94207361E081E294E10E949E5FAD
:102FC000682F70E04AE050E087E996E10E940174C2
:102FD00041E061E081E294E10E94265F112399F0D3
:102FE00063EE7BE087E996E10E94207361E081E275
:102FF00094E10E94A25F682F70E04AE050E087E908
:1030000096E10E94017441E061E081E294E10E9456
:103010002B5F60E081E294E10E94E05E1123B1F059
:103020006BEF7BE087E996E10E94207381E294E1F7
:103030000E944A5F682F70E04AE050E087E996E11D
:103040000E94017481E294E10E94A65FAA960FB6E5
:10305000F894DEBF0FBECDBFDF91CF911F91FF90DF
:10306000EF90DF90CF9008952F923F924F925F9212
:103070006F927F928F929F92AF92BF92CF92DF9288
:10308000EF92FF920F931F93CF93DF93CDB7DEB7ED
:10309000EF970FB6F894DEBF0FBECDBF2B013C01FA
:1030A0002DA33EA34FA358A70E946E6D6CAF7DAFBA
:1030B0008EAF9FAF2DA13EA14FA158A5243631055B
:1030C000410551052CF034E620E090E080E004C09A
:1030D0003DA12EA19FA188A540E9441641E05406D8
:1030E0006104710434F040E9442E55245394612C5A
:1030F000712C4091AA13411104C03DA32EA39FA39C
:1031000088A7B301A2014A505109610971098AE0F7
:1031100090E0A0E0B0E084199509A609B709EBE0BA
:103120004E165104610471042CF049AF5AAF6BAFD5
:10313000272E04C089AF9AAFABAF2B2E3324339424
:103140001DA61EA61FA618AA8E01035F1F4F2DA540
:103150003EA54FA558A98DA19EA1AFA1B8A528173E
:1031600039074A075B070CF021C30E946E6D2CAD36
:103170003DAD4EAD5FAD621B730B840B950B0E9492
:103180005F7B20E030E04AE754E40E94957AAB018F
:10319000BC0123E0C8010E94C477B80183EB93E12E
:1031A0000E942977C8010E945676BE016F5F7F4F4B
:1031B00081E294E10E940C5D6EE07CE089EB93E19A
:1031C0000E943F77AE014F5F5F4F5AA749A7C12CBE
:1031D000D12C7601A9A5BAA58D909D90AD90BD90FA
:1031E000BAA7A9A7A5019401C501B4010E94F57C65
:1031F0009B01AC01C701B6010E94CB796B017C0138
:1032000023E0B501A401CE0143960E94F277BE01EE
:103210006D5E7F4FC8010E9421776FEA74E0C8019C
:103220000E948478BC0189EB93E10E944B78C8012D
:103230000E945676CE0143960E945676E9A5FAA5DD
:10324000E017F10739F6C701B6010E94A87D6B01AE
:103250007C01FDE24F16F1E05F066104710444F069
:103260000E94360640E060E08BEB94E10E94195624
:1032700023E0B701A601C8010E94C4776AE177E0A4
:10328000CE0143960E94C17663EB73E1CE01439673
:103290000E9473786BE17CE00E948478B8010E9400
:1032A000737860E27CE00E948478BC0189EB93E152
:1032B0000E944B78CE0143960E945676C8010E9428
:1032C00056762DEC3CEC4CE45FE3C701B6010E945E
:1032D000367C29813A814B815C8129A73AA74BA78B
:1032E0005CA718160CF0ADC12AE939E949E95FE39A
:1032F000C701B6010E94917A87FFA3C1332009F468
:10330000A0C189849A84AB84BC8420E030E0A90108
:10331000C501B4010E94917ACD80DE80EF80F884EF
:10332000882309F129A53AA54BA55CA5CA01B901D5
:103330000E94F57C69AB7AAB8BAB9CABA701960185
:10334000C701B6010E94F57C9B01AC0169A97AA96D
:103350008BA99CA90E94CB790E94A87DA50194010C
:103360000E943E7A04C06BED7FE089EC9FE320EE83
:103370003EE245E652E40E94F57C69AB7AAB8BAB4A
:103380009CAB20E030E0A901C701B6010E94917A10
:10339000882309F129A53AA54BA55CA5CA01B90165
:1033A0000E94F57C6DAB7EAB8FAB98AFA50194010D
:1033B000C501B4010E94F57C9B01AC016DA97EA9F9
:1033C0008FA998AD0E94CB790E94A87DA701960194
:1033D0000E943E7A04C06BED7FE089EC9FE320EE13
:1033E0003EE245E652E40E94F57C6DAB7EAB8FABCE
:1033F00098AF20E030E0A90169A57AA58BA59CA52E
:103400000E94917A8823F9F0A5019401C501B401C5
:103410000E94F57C4B015C01A7019601C701B60132
:103420000E94F57C9B01AC01C501B4010E94CB79DF
:103430000E94A87D29A53AA54BA55CA50E943E7ACD
:103440006B017C0108C09BEDC92E9FE0D92E99EC41
:10345000E92E9FE3F92E6BE177E0C8010E94C17667
:1034600063EB73E1C8010E94737863E27CE00E9421
:103470008478BC0189EB93E10E940C77C8010E941B
:1034800056766BE177E0C8010E94C17663EB73E189
:10349000C8010E9473786DE37CE00E948478BC01CF
:1034A00083EB93E10E940C77C8010E94567621E0DD
:1034B00049A95AA96BA97CA9C8010E94C47721E037
:1034C0004DA95EA96FA978ADCE0143960E94C4773D
:1034D00020EE3EE245E652E4C701B6010E94F57CCB
:1034E000AB01BC0121E0CE014F960E94C477BE0122
:1034F000615E7F4FCE0149960E9421776FEA74E0AA
:10350000CE0149960E948478BE016D5E7F4F0E9475
:1035100073786FEA74E00E948478B8010E9473782F
:10352000BC018DEA93E10E940C77CE0149960E947E
:103530005676CE014F960E945676CE0143960E9453
:103540005676C8010E9456763DE2431631E0530696
:103550006104710474F46DA57EA58FA598A925E07A
:1035600030E040E050E00E945A7E672B682B692BC8
:1035700091F563EB73E1C8010E94217745E050E0CB
:103580006FEF7FEFC8010E940805C8010E945676C0
:1035900066E47CE0C8010E94C17645E050E061EF3E
:1035A0007FEFC8010E947C04C8010E9456766FED2F
:1035B0008BEB94E10E9421736DEA73E1C8010E94D4
:1035C000217745E050E060E070E0C8010E94BC0552
:1035D000C8010E9456766DEA73E189EB93E10E947F
:1035E0004B784FE1441651046104710434F48DA505
:1035F0009EA5AFA5B8A9B7FD11C069EB73E1C801DD
:103600000E942177C8010E949109C8010E94567644
:1036100066E972E189EB93E10E943F7769AD7AAD8B
:103620008BAD922D0E949D6D2DA53EA54FA558A94D
:103630002F5F3F4F4F4F5F4F2DA73EA74FA758AB70
:10364000A9C023E049A55AA56BA57CA5C8010E9485
:10365000C4776BE177E0CE0143960E94C17663EBBD
:1036600073E1CE0143960E94737868E47CE00E9487
:103670008478B8010E94737861E27CE00E948478CB
:10368000BC0183EB93E10E940C77CE0143960E942C
:103690005676C8010E94567649855A856B857C8589
:1036A00023E0C8010E94F2774D815E816F817885A9
:1036B00023E0CE0149960E94F277BE01675E7F4FFC
:1036C000CE0143960E9421776DE47CE0CE014396C3
:1036D0000E948478B8010E94737861E27CE00E94C5
:1036E0008478BC018DEA93E10E940C77CE01439669
:1036F0000E945676CE0149960E945676C8010E94D5
:1037000056763DE2431631E053066104710474F4C9
:103710006DA57EA58FA598A925E030E040E050E09A
:103720000E945A7E672B682B692BF1F463EB73E1DF
:10373000C8010E9421774AE050E06FEF7FEFC80197
:103740000E940805C8010E9456766DEA73E1C8011F
:103750000E9421774AE050E060E070E0C8010E94DA
:10376000BC05C8010E94567669EB73E1C8010E944E
:103770002177C8010E949109C8010E94567666E926
:1037800072E189EB93E10E943F77C301B2010E948D
:103790009D6D312C8DA59EA5AFA5B8A90196A11D43
:1037A000B11D8DA79EA7AFA7B8ABD1CC63EB73E1DA
:1037B000CE010D960E9421774AE050E06FEF7FEF37
:1037C000CE010D960E947C04CE010D960E94567685
:1037D0003320B9F066E47CE0CE010D960E94C176FC
:1037E00045E050E061EF7FEFCE010D960E947C0432
:1037F000CE010D960E9456766FED8BEB94E10E9400
:1038000021736DEA73E1CE010D960E9421774AE0A3
:1038100050E06FEF7FEFCE010D960E947002CE0157
:103820000D960E945676EF960FB6F894DEBF0FBE47
:10383000CDBFDF91CF911F910F91FF90EF90DF905F
:10384000CF90BF90AF909F908F907F906F905F9040
:103850004F903F902F900895CF92DF92EF92FF927A
:103860000F931F93CF93DF93CDB7DEB72C970FB68F
:10387000F894DEBF0FBECDBF8091AA13811102C0A4
:103880000E94360684E397E10E94B17064E670E01E
:1038900080E090E00E949D6D60E57CE083EB93E129
:1038A0000E943F7763EB73E1CE0101960E9421777E
:1038B00044E150E060E070E0CE0101960E947C049B
:1038C000CE0101960E9456766CE57CE083EB93E195
:1038D0000E943F7763EB73E1CE0101960E9421774E
:1038E00044E150E06FEF7FEFCE0101960E9470023D
:1038F000CE0101960E94567660E070E084EA94E181
:103900000E94226D6B017C0104E010E0A70196018A
:10391000C701B6010E94E97D882309F43DC001502A
:10392000110909F023C16AE97EE083EB93E10E946B
:103930003F7763EB73E1CE0101960E9421774AE065
:1039400050E060E070E0CE0101960E947C04CE0160
:1039500001960E9456766BE67CE0CE0101960E94AD
:10396000C17663EB73E1CE0101960E947378BC01CE
:1039700089EB93E10E940C77CE0101960E94567666
:103980008091D4149091D514039709F0DEC0109261
:10399000D5141092D414D9C021E0B701A601CE01EC
:1039A00007960E94C4776DE77CE0CE0101960E94E5
:1039B000C176BE01695F7F4FCE0101960E94737888
:1039C000BC0189EB93E10E940C77CE0101960E9425
:1039D0005676CE0107960E94567669EB73E1CE01CA
:1039E00001960E94217742E350E06FEF7FEFCE0116
:1039F00001960E947002CE0101960E9456766FEDEC
:103A00008BEB94E10E94217369E877E08BEB94E102
:103A10000E94207368E877E089EB93E10E94517877
:103A200060E070E084EA94E10E94206D6B017C010B
:103A300004E010E0A7019601C701B6010E94E97DEC
:103A4000882359F00150110909F09FC066E972E11D
:103A50008FEB93E10E943F7759C021E0B701A601A7
:103A6000CE0107960E94C4776BE870E1CE01019603
:103A70000E94C176BE01695F7F4FCE0101960E9410
:103A80007378BC018FEB93E10E940C77CE01019615
:103A90000E945676CE0107960E9456766FEA74E031
:103AA000CE0101960E94C1766FEB73E1CE010196C3
:103AB0000E947378BC0183EB93E10E940C77CE01E6
:103AC00001960E94567663EB73E1CE0101960E9447
:103AD00021774AE050E06FEF7FEFCE0101960E9420
:103AE0000805CE0101960E9456766FED8BEB94E1AE
:103AF0000E94217369E877E08BEB94E10E942073C8
:103B000068E877E08FEB93E10E9451786FEB73E107
:103B1000CE0101960E9421776FEA74E0CE010196F2
:103B20000E94847869EB73E10E947378BC0189EB91
:103B300093E10E940C77CE0101960E94567683E0B5
:103B400090E09093D5148093D41464E670E080E004
:103B500090E00E949D6D8091AA13882329F160E274
:103B600073E080E090E00E949D6D1EC064E670E00E
:103B700080E090E00E949D6D60E070E084EA94E156
:103B80000E94226D6B017C01C1CE68EC70E080E088
:103B900090E00E949D6D60E070E084EA94E10E94F4
:103BA000206D6B017C0146CF2C960FB6F894DEBFDA
:103BB0000FBECDBFDF91CF911F910F91FF90EF907E
:103BC000DF90CF9008951F93CF93DF93182FC1E418
:103BD000D3E1812F0E94336E899399936CE370E057
:103BE00080E090E00E949D6D83E1C139D80789F79C
:103BF00068E270E081E493E10E94A20220E030E0FC
:103C000040EA50E40E94F57C20E030E040E85AE3CE
:103C10000E94F57CDF91CF911F9108954F925F92A2
:103C20006F927F928F929F92AF92BF92CF92DF92CC
:103C3000EF92FF920F931F93CF93DF93CDB7DEB731
:103C400064970FB6F894DEBF0FBECDBF7C018B0129
:103C500063E875E083EB93E10E943F770E943606AC
:103C600063EB73E1CE0101960E9421774AE050E0B8
:103C70006FEF7FEFCE0101960E947C04CE0101968A
:103C80000E945676C7019FDF698B7A8B8B8B9C8B4A
:103C900040901A0250901B0260901C0270901D020E
:103CA000A30192016091160270911702809118028F
:103CB000909119020E94CA794B015C0120E030E02A
:103CC000A9010E94917A882309F451C0C090220270
:103CD000D0902302E0902402F090250220E030E012
:103CE000A901C701B6010E94917A18160CF03FC0D5
:103CF00080911E0290911F02A0912002B09121029A
:103D00008D879E87AF87B88B9C01AD01C701B60137
:103D10000E94917A882359F1A70196016D857E85CD
:103D20008F8598890E94957A0E94827C6D877E8714
:103D30008F87988BA301920169897A898B899C89E5
:103D40000E94CA79A50194010E94957A2D853E852D
:103D50004F8558890E94F57C0E94027B9B01AC0133
:103D6000C701B6010E94F57C6B017C0103C0C12C28
:103D7000D12C760163EB73E1CE0101960E9421778D
:103D80004AE050E060E070E0CE0101960E947C04C1
:103D9000CE0101960E94567620E030E64AEE56E4C7
:103DA000C701B6010E94367C18163CF466E87CE038
:103DB00089EB93E10E943F7744C001151105B9F4E6
:103DC00021E0B701A601CE0107960E94C47765E9FC
:103DD0007CE0CE0101960E94C176BE01695F7F4FF3
:103DE000CE0101960E94737869E97CE01BC0023025
:103DF000110539F522E049895A896B897C89CE0100
:103E000007960E94C47765E97CE0CE0101960E9486
:103E1000C176BE01695F7F4FCE0101960E94737823
:103E20006DE97CE00E948478BC0189EB93E10E94FB
:103E30000C77CE0101960E945676CE0107960E941D
:103E4000567669EB73E1CE0101960E9421774AE034
:103E500050E06FEF7FEFCE0101960E947002CE011D
:103E600001960E94567664E670E080E090E00E9441
:103E70009D6D8091AA13882331F060E273E080E0A9
:103E800090E00E949D6D64960FB6F894DEBF0FBE61
:103E9000CDBFDF91CF911F910F91FF90EF90DF90F9
:103EA000CF90BF90AF909F908F907F906F905F90DA
:103EB0004F9008954F925F926F927F928F929F9250
:103EC000AF92BF92CF92DF92EF92FF92CF93C82F23
:103ED0008091BC1281110DC00E946E6D6093B01272
:103EE0007093B1128093B2129093B31281E08093D9
:103EF000BC128091B41281110DC00E946E6D60934E
:103F0000AC127093AD128093AE129093AF1281E019
:103F10008093B4121092401310923F13E0903F131D
:103F2000F090401388E2E816F1040CF08AC08C2F60
:103F30000E94336EF701EE0FFF1FEF5BFC4E918383
:103F4000808368E270E081E493E10E94A20220E0B5
:103F500030E040EA50E40E94F57C20E030E040E8A8
:103F60005AE30E94F57C6B017C016093A812709368
:103F7000A9128093AA129093AB1240902A025090FB
:103F80002B0260902C0270902D02A301920160918F
:103F900026027091270280912802909129020E94A6
:103FA000CA799B01AC0160E070E080EC90E40E9473
:103FB000CA794B015C0120E030E0A9010E94917AAE
:103FC00020E030E040E650E4811105C0C701B601B1
:103FD0000E94F57C1EC0C701B6010E94F57CA301BA
:103FE00092010E94CB7920E030E040E850E40E944A
:103FF000CA79A50194010E94957A20E030E040EC56
:1040000050E40E94F57C20E030E040E850E40E945B
:10401000CB796093A4127093A5128093A61290930B
:10402000A71264E170E080E090E00E949D6D8091B5
:104030003F139091401301969093401380933F1348
:104040006DCF6091A4127091A5128091A6129091EB
:10405000A712CF91FF90EF90DF90CF90BF90AF90DD
:104060009F908F907F906F905F904F900895CF9228
:10407000DF92EF92FF92CF93DF93CDB7DEB72C970D
:104080000FB6F894DEBF0FBECDBF60E575E083EBE1
:1040900093E10E943F7763EB73E1CE0101960E94AA
:1040A00021774AE050E060E070E0CE0101960E9486
:1040B0007C04CE0101960E945676809181029091F7
:1040C0008202F8DE6B017C0120E030E0A9010E9451
:1040D000367C87FD22C022E0B701A601CE010796FB
:1040E0000E94C47769EC7CE0CE0101960E94C17603
:1040F000BE01695F7F4FCE0101960E947378BC01BB
:1041000089EB93E10E940C77CE0101960E945676CE
:10411000CE0107960E94567606C06DEC7CE089EBD6
:1041200093E10E943F7769EB73E1CE0101960E9413
:1041300021774AE050E06FEF7FEFCE0101960E94B9
:104140007002CE0101960E9456762C960FB6F89416
:10415000DEBF0FBECDBFDF91CF91FF90EF90DF901C
:10416000CF9008952F923F924F925F926F927F92DD
:104170008F929F92AF92BF92CF92DF92EF92FF9277
:104180000F931F93CF93DF9300D01F92CDB7DEB76D
:104190006B017C015A8349835901FA0120813181E5
:1041A000428153810E94917A181614F0F50183C060
:1041B00010E00150104C000F111F000F111FE9817A
:1041C000FA81E00FF11F2081318142815381C701C3
:1041D000B6010E94367C87FF6BC011E0612E712C06
:1041E0004301880C991C880C991CE981FA81E80D1F
:1041F000F91D2080318042805380A2019101C701C6
:10420000B6010E94367C181614F41F5FE7CFA20196
:104210009101C701B6010E94917A8501080D191D0F
:10422000811102C0F80147C0C3018150904C880F32
:10423000991F880F991FA981BA81A80FB91F2D91C5
:104240003D914D915C9129833A834B835C83F501C9
:10425000E80FF91F80809180A280B380C701B6016A
:104260000E94CA796B017C01A5019401F80160816B
:104270007181828193810E94CA799B01AC01C7013F
:10428000B6010E94F57C6B017C0129813A814B814A
:104290005C81C201B1010E94CA799B01AC01C701D6
:1042A000B6010E94957AA50194010E94CB7907C0BE
:1042B000F501E00FF11F60817181828193810F9080
:1042C0000F900F900F90DF91CF911F910F91FF9062
:1042D000EF90DF90CF90BF90AF909F908F907F90A6
:1042E0006F905F904F903F902F900895CF92DF9204
:1042F000EF92FF921F93CF93DF93182FCAE0D0E085
:10430000C12CD12C7601812F0E94336EBC018827ED
:1043100077FD8095982F0E94617B9B01AC01C701BE
:10432000B6010E94CB796B017C0162E370E080E012
:1043300090E00E949D6D219731F720E030E040E24F
:1043400051E4C701B6010E94957A20E030E040EACE
:1043500050E40E94F57C20E030E040E85AE30E94FF
:10436000F57CDF91CF911F91FF90EF90DF90CF9080
:1043700008952F923F924F925F926F927F928F9209
:104380009F92AF92BF92CF92DF92EF92FF920F93E4
:104390001F93CF93DF93CDB7DEB73A011801290100
:1043A000A50194010E94957A4B015C0120E030E068
:1043B00040EC5FE3C201B1010E94F57C9B01AC01BE
:1043C000C501B4010E94367C181694F120E030E05B
:1043D00040E05FE3C701B6010E94F57C9B01AC01A0
:1043E000C501B4010E94917A87FD22C0F3012481A6
:1043F000358146815781C501B4010E94CA79F30114
:1044000020853185428553850E94957AF30120816C
:104410003181428153810E94CB799B01AC0160E0E4
:1044200070E080E291E40E94587D0E942E7B03C0E0
:104430006FEF7FEFCB01DF91CF911F910F91FF9035
:10444000EF90DF90CF90BF90AF909F908F907F9034
:104450006F905F904F903F902F9008954F925F9292
:104460006F927F928F929F92AF92BF92CF92DF9284
:10447000EF92FF920F931F93CF93DF93CDB7DEB7E9
:10448000A0970FB6F894DEBF0FBECDBF2FDF698FA8
:104490007A8F8B8F9C8F409045025090460260909F
:1044A000470270904802C0904102D0904202E090D2
:1044B0004302F09044028090490290904A02A090FA
:1044C0004B02B0904C0289829A82AB82BC824D82B0
:1044D0005E826F827886A7019601C301B2010E94B5
:1044E000CA796D8F7E8F8F8F98A320913D02309176
:1044F0003E0240913F0250914002C501B4010E942A
:10450000CA799B01AC016D8D7E8D8F8D98A10E9423
:10451000957A69877A878B879C87812C912CF8E024
:10452000AF2EF1E4BF2E93018201AE014F5F5F4FCA
:10453000698D7A8D8B8D9C8D1CDF6B017C010E94B7
:1045400036066CED7CE083EB93E10E943F7763EBF2
:1045500073E1CE010D960E94217742E350E060E0C6
:1045600070E0CE010D960E947C04CE010D960E9453
:1045700056762AE0B701A601CE0143960E949877AD
:1045800065EE7CE0CE010D960E94C176BE016D5EA7
:104590007F4FCE010D960E9473786AEE7CE00E94F8
:1045A0008478BC0189EB93E10E940C77CE010D96D3
:1045B0000E945676CE0143960E94567669EB73E1CF
:1045C000CE010D960E94217742E350E06FEF7FEF1E
:1045D000CE010D960E947002CE010D960E94567675
:1045E0008091AA13882331F060E273E080E090E0CC
:1045F0000E949D6DA0960FB6F894DEBF0FBECDBF92
:10460000DF91CF911F910F91FF90EF90DF90CF90AE
:10461000BF90AF909F908F907F906F905F904F90E2
:104620000895FC0120E030E0772767FD7095AB012D
:1046300042505109DF01A81BB90BA417B50724F498
:10464000A1912A0F311DF6CFA9014E5B5F4F860F56
:10465000971FFC013297208130E0322F22273196BC
:104660008081280F311D81E04217530709F080E057
:1046700008952F923F924F925F926F927F928F9206
:104680009F92AF92BF92CF92DF92EF92FF920F93E1
:104690001F93CF93DF93CDB7DEB763970FB6F89430
:1046A000DEBF0FBECDBF8B8B60E00E94AC6E8091F1
:1046B000AA13811105C08FE090E0A0E0B0E004C033
:1046C00082E090E0A0E0B0E08F87988BA98BBA8B56
:1046D0006AEC75E089EB93E10E943F7769EB73E147
:1046E000CE0101960E9421774AE050E06FEF7FEF04
:1046F000CE0101960E947C04CE0101960E9456765E
:10470000C12CD12C7601312C1D861E86212C02E372
:1047100010E0412C512C32018B890E94336EAA2764
:1047200097FDA095BA2F480E591E6A1E7B1E65E0A4
:1047300070E080E090E00E949D6D0150110961F7EA
:104740008090120290901302A0901402B090150273
:10475000C301B2010E94617B20E030E040EA50E4F6
:104760000E94F57C20E030E040E85AE30E94F57CAE
:1047700020E030E048E452E40E94957AA5019401DB
:104780000E94CA7920E030E040E751E40E94F57CC5
:104790002B013C01A50194016AE979E989E390E4E0
:1047A0000E94CA799B01AC01C301B2010E94957AB3
:1047B00020E030E0A9010E94CB7920E030E040E227
:1047C00051E40E94F57C5B018C01232D3D854E85D3
:1047D000522D0E94367C181624F43A2CBD860E8782
:1047E000212E20E030E0A901B501C8010E94917A94
:1047F00087FF04C0A12CB12C00E010E022E0A5014D
:10480000B801CE0107960E94C477BE01695F7F4F51
:10481000CE0101960E94217768E17DE0CE010196EC
:104820000E948478BC0183EB93E10E940C77CE0157
:1048300001960E945676CE0107960E94567663EB4B
:1048400073E1CE0101960E9421774AE050E060E0DA
:1048500070E0CE0101960E94BC05CE0101960E9437
:1048600056760E946E6D80908A0490908B04A09082
:104870008C04B0908D040091B3141091B414209165
:10488000B5143091B614800E911EA21EB31E86166A
:104890009706A806B90608F4E7C00E946E6D0E944C
:1048A0005F7B4B015C0160918A0470918B04809165
:1048B0008C0490918D040E94617B20E030E040E800
:1048C0005EE30E94F57C2B013C016091B314709172
:1048D000B4148091B5149091B6140E94617B9B0131
:1048E000AC01C301B2010E94CB799B01AC01C501AF
:1048F000B4010E94917A87FDB7C06CE370E080E05C
:1049000090E00E949D6D9FEFC91AD90AE90AF90A41
:104910008F859889A989BA898C159D05AE05BF0533
:104920000CF0F5CE64E670E080E090E00E949D6DB2
:104930000E94360664E670E080E090E00E949D6D83
:104940006DE17DE083EB93E10E943F7763EB73E1E0
:10495000CE0101960E94217744E150E060E070E0D2
:10496000CE0101960E947C04CE0101960E945676EB
:1049700022E0432D5D856E85722DCE0107960E9443
:10498000C477BE01695F7F4FCE0101960E942177F7
:1049900068E17DE0CE0101960E948478BC0183EB42
:1049A00093E10E940C77CE0101960E945676CE01CB
:1049B00007960E94567663EB73E1CE0101960E9442
:1049C000217742E350E06FEF7FEFCE0101960E9426
:1049D0007002CE0101960E945676E091BB14F091D0
:1049E000BC140190F081E02D60E08BEB94E119950F
:1049F00062E370E080E090E00E949D6D65E27DE002
:104A0000CE0101960E94C17663EB73E1CE0101965F
:104A10000E94737869E27DE00E94847869EB73E11B
:104A20000E947378BC0189EB93E10E940C77CE0160
:104A300001960E94567663960FB6F894DEBF0FBEBD
:104A4000CDBFDF91CF911F910F91FF90EF90DF903D
:104A5000CF90BF90AF909F908F907F906F905F901E
:104A60004F903F902F900895E091BB14F091BC14AB
:104A70000190F081E02D60E08BEB94E119953DCF42
:104A8000FF920F931F93CF93DF93F82E0AE010E06D
:104A9000C0E0D0E08F2D0E94336EC80FD91F65E0B3
:104AA00070E080E090E00E949D6D0150110991F747
:104AB000CE016AE070E00E94117ECB01DF91CF91C0
:104AC0001F910F91FF9008950F931F93CF93DF9342
:104AD000CDB7DEB72E970FB6F894DEBF0FBECDBFB1
:104AE0008D879E870E9436068D859E85C9DF8C0145
:104AF00062E370E080E090E00E949D6DB80188273D
:104B000077FD8095982F0E94617B20E030E040EA9D
:104B100050E40E94F57C20E030EC4FE754E40E9422
:104B2000957AAB01BC0123E0CE0107960E94C477C1
:104B300066E27DE0CE0101960E94C176BE01695F0A
:104B40007F4FCE0101960E9473786FE27DE00E9454
:104B50008478BC0189EB93E10E940C77CE01019629
:104B60000E945676CE0107960E94567668E775E059
:104B700083EB93E10E943F7763EB73E1CE010196F3
:104B80000E9421774AE050E068E070E0CE01019693
:104B90000E947C04CE0101960E94567669EB73E177
:104BA000CE0101960E9421774AE050E06FEF7FEF3F
:104BB000CE0101960E947002CE0101960E945676A7
:104BC00063EB73E189EB93E10E944B788091AA1328
:104BD000882331F060E273E080E090E00E949D6DF8
:104BE0002E960FB6F894DEBF0FBECDBFDF91CF91EA
:104BF0001F910F910895CF93DF93CDB7DEB72C9718
:104C00000FB6F894DEBF0FBECDBF3ADF9093A61368
:104C10008093A51362E370E080E090E00E949D6DB8
:104C20006091A5137091A6134AE0CE0101960E94EF
:104C30006D77BE016F5F7F4F89EB93E10E9429770B
:104C4000CE0101960E94567680911B1490911C14FF
:104C5000892B09F45FC067E174E1CE0107960E94D9
:104C60002177BE01695F7F4FCE0101960E942177B7
:104C700044E150E060E070E0CE0101960E947C04C7
:104C8000CE0101960E94567662E37DE0CE01019648
:104C90000E94C17669EB73E1CE0101960E947378A0
:104CA000BC0183EB93E10E940C77CE0101960E9438
:104CB000567663EB73E1CE0101960E94217744E1C1
:104CC00050E06FEF7FEFCE0101960E947002CE019F
:104CD00001960E945676BE01695F7F4FCE01019614
:104CE0000E9421776FEA74E0CE0101960E948478D9
:104CF00063EB73E10E947378BC0189EB93E10E943E
:104D00000C77CE0101960E945676CE0107960E943E
:104D1000567654C06DE37DE083EB93E10E943F77CC
:104D200063EB73E1CE0101960E94217744E150E0EC
:104D300060E070E0CE0101960E947C04CE010196F5
:104D40000E94567661E47DE0CE0101960E94C17614
:104D500069EB73E1CE0101960E947378BC0183EB8D
:104D600093E10E940C77CE0101960E94567663EB88
:104D700073E1CE0101960E94217744E150E06FEF8C
:104D80007FEFCE0101960E947002CE0101960E9433
:104D9000567662E37DE0CE0101960E94C17669EB12
:104DA00073E1CE0101960E947378BC0189EB93E117
:104DB0000E940C77CE0101960E9456768091AA132C
:104DC000882331F060E273E080E090E00E949D6D06
:104DD0002C960FB6F894DEBF0FBECDBFDF91CF91FA
:104DE00008950F931F93CF93DF93CDB7DEB72C9722
:104DF0000FB6F894DEBF0FBECDBF8C0181E00E94DC
:104E0000306E64E670E080E090E00E949D6D0E944C
:104E10003606C80135DE60E074E0681B790B4AE0B5
:104E2000CE0107960E946D7761E47DE0CE01019688
:104E30000E94C176BE01695F7F4FCE0101960E943C
:104E40007378BC0189EB93E10E940C77CE01019647
:104E50000E945676CE0107960E94567640E066E0A4
:104E60008BEB94E10E94195668E47DE0CE01019637
:104E70000E94C17642E350E068E070E0CE01019606
:104E80000E947C04CE0101960E94567669EB73E184
:104E9000CE0101960E94217742E350E06FEF7FEF51
:104EA000CE0101960E947002CE0101960E945676B4
:104EB00061E57DE0CE0101960E94C17669EB73E168
:104EC000CE0101960E947378BC0189EB93E10E94A8
:104ED0000C77CE0101960E9456768091AA13882302
:104EE00031F060E273E080E090E00E949D6D2C96CE
:104EF0000FB6F894DEBF0FBECDBFDF91CF911F91EB
:104F00000F9108950F9390E0BBDDBC01882777FDDA
:104F10008095982F0E94617B2DE038E643E55BE3A6
:104F20000E94F57C06E021E532E049E652E01AD91C
:104F300020E030E048EC52E40E94F57C20E030E0D4
:104F400048EA51E40E94F57C20914D0230914E02D6
:104F500040914F02509150020E94957A0F9108950E
:104F6000CF92DF92EF92FF92CF93DF93CDB7DEB770
:104F70002C970FB6F894DEBF0FBECDBFC3DF6B0119
:104F80007C016DED7CE083EB93E10E943F7763EB66
:104F900073E1CE0101960E94217742E350E060E088
:104FA00070E0CE0101960E947C04CE0101960E9421
:104FB000567622E0B701A601CE0107960E94C4777B
:104FC00066EE7CE0CE0101960E94C176BE01695F6B
:104FD0007F4FCE0101960E9473786BE57DE00E94C1
:104FE0008478BC0189EB93E10E940C77CE01019695
:104FF0000E945676CE0107960E94567669EB73E1C1
:10500000CE0101960E94217742E350E06FEF7FEFDF
:10501000CE0101960E947002CE0101960E94567642
:105020008091AA13882331F060E273E080E090E081
:105030000E949D6D2C960FB6F894DEBF0FBECDBFBB
:10504000DF91CF91FF90EF90DF90CF900895CF92B6
:10505000DF92EF92FF920F9390E012DDBC01882760
:1050600077FD8095982F0E94617B2DE038E643E51F
:105070005BE30E94F57C06E021E532E049E652E080
:1050800071D820E030E048EC52E40E94F57C6B01DE
:105090007C0120E030E0A9010E94917A181634F0DA
:1050A000C12CD12C48EAE42E41E4F42EC0924D02EA
:1050B000D0924E02E0924F02F09250020F91FF9078
:1050C000EF90DF90CF9008959F92AF92BF92CF92D2
:1050D000DF92EF92FF920F931F93CF93DF935C01C8
:1050E000C0E5D4E00EE314E051E2E52E53E1F52EE5
:1050F000CC24C394D12C75E1972E80913C049091DF
:105100003D048C159D050CF49DC081E0A816B104EA
:1051100029F4F70180819181F80108C0F2E0AF160F
:10512000B10431F4F80180819181F701918380838A
:10513000F80180819181009739F488819981909359
:1051400061048093600422C08130910539F4888124
:10515000998190936F0480936E0418C082309105FA
:1051600039F48881998190936D0480936C040EC00A
:10517000039761F48881998190936304809362041A
:1051800066E972E187E194E10E943F77F80121919D
:1051900031918F012430310539F4888199819093C0
:1051A00082028093810228C02530310539F488813C
:1051B000998190936B0480936A041EC02630310558
:1051C00039F48881998190936704809366041EC0A6
:1051D0002730310539F48881998190936504809353
:1051E000640428C02A30310539F48881998190936C
:1051F0006904809368041EC02531310539F4888123
:105200009981909371048093700414C02B30310500
:105210008CF0888199819093630480936204929EBC
:10522000B001939E700D11246D577D4F87E194E17D
:105230000E943F77FFEFCF1ADF0A229682E0E80E46
:10524000F11C5BCFDF91CF911F910F91FF90EF90F9
:10525000DF90CF90BF90AF909F9008958F929F92D4
:10526000AF92BF92CF92DF92EF92FF920F931F9275
:105270001F9283E08F93E7E08E2EF6E0AF2EA5E03D
:10528000CA2EB4E0EB2E00E021E042E06FE38BEBAE
:1052900094E10E949B5760E67DE08DEA94E10E94D4
:1052A000C17666E67DE087EA94E10E94C17620E15E
:1052B00041E168E184EA94E10E94386C04E022E76D
:1052C00034E046E754E06AE774E085E394E10E9445
:1052D000485881E294E10E94415B66E972E187E10E
:1052E00094E10E94C1768091660490916704909346
:1052F0001614809315148090450290904602A09059
:105300004702B09048022091410230914202409100
:10531000430250914402C501B4010E94CA796B0155
:105320007C01609311147093121480931314909362
:1053300014146091490270914A0280914B0290913D
:105340004C02609305147093061480930714909395
:1053500008148092091490920A14A0920B14B0922F
:105360000C1420913D0230913E0240913F02509139
:1053700040020E94CA799B01AC01C701B6010E949C
:10538000957A60930D1470930E1480930F1490937C
:1053900010144FEF5FEFBA018CEE93E10E943A4D8B
:1053A00085ED93E10E94515266E972E18BEC93E145
:1053B0000E94C17666E972E185EC93E10E94C176B4
:1053C00066E972E18FEB93E10E94C17666E972E1D2
:1053D00089EB93E10E94C17666E972E183EB93E188
:1053E0000E94C17666E972E18DEA93E10E94C1767E
:1053F0000F900F900F90609132027091330286EE01
:1054000092E10F91FF90EF90DF90CF90BF90AF901F
:105410009F908F900C947A618DEA93E10E9456766A
:1054200083EB93E10E94567689EB93E10E945676D6
:105430008FEB93E10E94567685EC93E10E945676BD
:105440008BEC93E10E94567680E292E19093ED130B
:105450008093EC1387E194E10E94567687EA94E109
:105460000E9456768DEA94E10C945676CF92DF92A4
:10547000EF92FF920F931F93CF93DF93CDB7DEB7D9
:1054800069970FB6F894DEBF0FBECDBF6B017C01EC
:1054900084E397E10E94B17064E670E080E090E000
:1054A0000E949D6D40E855E260E070E084E397E182
:1054B0000E94050464E670E080E090E00E949D6D2B
:1054C00060E57CE083EB93E10E943F7763EB73E15F
:1054D000CE0101960E94217742E350E06FEF7FEF0B
:1054E000CE0101960E947C04CE0101960E94567660
:1054F0006EE67DE083EB93E10E943F7763EB73E11F
:10550000CE0101960E94217742E350E06FEF7FEFDA
:10551000CE0101960E947002CE0101960E9456763D
:105520008091D4149091D5148D7F00E0019709F4F7
:1055300069C012E40E946E6D6C197D098E099F0985
:10554000683B7B408105910508F05CC084E397E1EE
:105550000E94426F892B09F44EC04CED55E060E08B
:1055600070E084E397E10E946E75198F41E050E08E
:10557000BE01675E7F4F84E397E10E9455768823E2
:10558000D1F14FE150E06CED74E184E397E10E94CA
:1055900074758091DC148D3471F56FE18CED94E1BC
:1055A00040D8882341F18091DF1490E0982F88271C
:1055B0002091E014820F911D9093DB148093DA14F4
:1055C0008091E11490E0982F88272091E214820FB7
:1055D000911D9093D9148093D8148091E31490E096
:1055E000982F88272091E414820F911D9093D7144F
:1055F0008093D61401E062E370E080E090E00E94C6
:105600009D6D98CF0E946E6D6C197D098E099F0962
:10561000683B7B408105910510F40111D3C00E94C5
:10562000360663EB73E1CE0101960E94217742E3D7
:1056300050E066E070E0CE0101960E947C04CE014D
:1056400001960E945676002309F4DBC082E090E0C8
:105650009093D5148093D4146091D6147091D7147C
:105660004AE0CE0101960E946D776091D814709146
:10567000D9144AE0CE0107960E946D776091DA1442
:105680007091DB144AE0CE0143960E946D77BE0113
:105690006D5E7F4FCE010D960E9421776EED70E119
:1056A000CE010D960E948478BE01695F7F4F0E94F3
:1056B00073786EED70E10E948478BE016F5F7F4F5A
:1056C0000E947378BC0189EB93E10E940C77CE01B4
:1056D0000D960E945676CE0143960E945676CE01D4
:1056E00007960E945676CE0101960E94567669EB87
:1056F00073E1CE0101960E9421774AE050E06FEFFE
:105700007FEFCE0101960E947002CE0101960E94A9
:10571000567669E77DE08BEB94E10E9420736091FF
:10572000D6147091D7144AE0CE0101960E946D778D
:105730006091D8147091D9144AE0CE0107960E9466
:105740006D776091DA147091DB144AE0CE014396D4
:105750000E946D776FE77DE0CE010D960E94C176C5
:10576000BE016D5E7F4FCE010D960E9473786FEA89
:1057700074E00E948478BE01695F7F4F0E94737855
:105780006FEA74E00E948478BE016F5F7F4F0E94D1
:10579000737869E77DE00E948478BC0189EB93E12E
:1057A0000E940C77CE010D960E945676CE0143964C
:1057B0000E945676CE0107960E945676CE0101963B
:1057C0000E94567662E370E080E090E00E949D6D5A
:1057D00084E397E10E94B17062E370E080E090E0C2
:1057E0000E949D6D69960FB6F894DEBF0FBECDBFC7
:1057F000DF91CF911F910F91FF90EF90DF90CF90AD
:1058000008956AE97EE089EB93E10E943F7769EBB6
:1058100073E1CE0101960E9421774AE050E060E0FA
:1058200070E0CE0101960E94BC05CE0101960E9457
:1058300056766FE87DE089EB93E10E943F77809197
:10584000D4149091D514029709F0BCCF1092D514BE
:105850001092D414B7CF7F928F929F92AF92BF9243
:10586000CF92DF92EF92FF920F931F93CF93DF932C
:1058700000D000D0CDB7DEB74C0184E397E10E94A1
:10588000B17040E052EC61E070E084E397E10E9487
:1058900005044CED55E060E070E084E397E10E9480
:1058A0006E7564E670E080E090E00E949D6DA12C32
:1058B000B12C712CA814B9040CF051C065E070E053
:1058C00080E090E00E949D6D00E010E0C12CD12CA2
:1058D000760171100FC084E397E10E94426F892B1B
:1058E00031F485E1C816D104E104F1041CF403305D
:1058F000110554F08FEFA81AB80A64E670E080E052
:1059000090E00E949D6DD6CF84E397E10E94426FA4
:10591000892B69F084E397E10E945B6FE1E0F0E09E
:10592000EC0FFD1FE00FF11F80830F5F1F4F65E03D
:1059300070E080E090E00E949D6D023011054CF017
:1059400089818B3B31F4772473948A818A3A09F0F8
:10595000712C8FEFC81AD80AE80AF80ABACF872D37
:1059600026960FB6F894DEBF0FBECDBFDF91CF9164
:105970001F910F91FF90EF90DF90CF90BF90AF906D
:105980009F908F907F9008958F929F92AF92BF9239
:10599000CF92DF92EF92FF920F931F93CF93DF93FB
:1059A000CDB7DEB72C970FB6F894DEBF0FBECDBFD4
:1059B00020E042E060E18BEB94E10E941F584EE84A
:1059C00054E060E08BEB94E10E94D5568BEB94E1C0
:1059D0000E9455568EED93E090933E1380933D13B5
:1059E0000E94F8818093FB148FED93E00E94F88170
:1059F0008093FC148091FB149091FC1418161906E6
:105A000054F410929604019731F41092FC14109201
:105A1000FB140E94580462EA7DE08BEB94E10E9443
:105A2000207340E855E260E070E087E996E10E946B
:105A3000050440E855E260E070E081ED97E10E94E6
:105A4000050464E670E080E090E00E949D6D809126
:105A50009604882331F068EE73E080E090E00E94C5
:105A60009D6D87E996E10E945B6F182F823709F4DC
:105A700001C110923E1310923D1367EEC62E62E1F3
:105A8000D62EE12CF12CC7010E94F881F6018193FA
:105A90006F01FFEFEF1AFF0A8EE4E816F10499F7A1
:105AA0004091E7125091E8126091E9127091EA1268
:105AB00045365105610571050CF4DCC04093380290
:105AC0005093390260933A0270933B028091EB123B
:105AD0009091EC12A091ED12B091EE1280933402ED
:105AE00090933502A0933602B09337028091EF1263
:105AF0009091F012A091F112B091F21280932E02C7
:105B000090932F02A0933002B093310263E073E1CF
:105B1000CE0101960E94C176BE016F5F7F4F8DEA74
:105B200094E10E942977CE0101960E9456768091D9
:105B3000F3129091F412A091F512B091F6128093A5
:105B4000220290932302A0932402B0932502809115
:105B5000F7129091F812A091F912B091FA12809375
:105B60001E0290931F02A0932002B0932102809105
:105B7000FB129091FC12A091FD12B091FE12809345
:105B80001A0290931B02A0931C02B0931D028091F5
:105B9000FF1290910013A0910113B0910213809312
:105BA000160290931702A0931802B09319028091E5
:105BB0000B1390910C13A0910D13B0910E138093C1
:105BC000450290934602A0934702B0934802809109
:105BD0000F1390911013A0911113B0911213809391
:105BE000410290934202A0934302B09344028091F9
:105BF000131390911413A0911513B0911613809361
:105C0000490290934A02A0934B02B0934C028091B8
:105C1000171390911813A0911913B0911A13809330
:105C20003D0290933E02A0933F02B09340028091C8
:105C30001B1390911C13A0911D13B0911E13809300
:105C40004D0290934E02A0934F02B0935002809168
:105C5000311390913213A0913313B0913413809388
:105C6000120290931302A0931402B093150281E0E4
:105C700090E02ADA0EE8010F023070F08091E7120E
:105C80009091E812A091E912B091EA12853691053F
:105C9000A105B1050CF020C1809138029091390224
:105CA000A0913A02B0913B028093E7129093E812E0
:105CB000A093E912B093EA128091340290913502D8
:105CC000A0913602B09137028093EB129093EC12C0
:105CD000A093ED12B093EE1280912E0290912F02BC
:105CE000A0913002B09131028093EF129093F012A4
:105CF000A093F112B093F212123751F420E030E089
:105D000048E050E063E073E18DEA94E10E94E078BE
:105D10008091220290912302A0912402B091250249
:105D20008093F3129093F412A093F512B093F612AD
:105D300080911E0290911F02A0912002B091210239
:105D40008093F7129093F812A093F912B093FA127D
:105D500080911A0290911B02A0911C02B0911D0229
:105D60008093FB129093FC12A093FD12B093FE124D
:105D70008091160290911702A0911802B091190219
:105D80008093FF1290930013A0930113B09302131A
:105D90008091450290914602A0914702B09148023D
:105DA00080930B1390930C13A0930D13B0930E13C9
:105DB0008091410290914202A0914302B09144022D
:105DC00080930F1390931013A0931113B093121399
:105DD0008091490290914A02A0914B02B0914C02ED
:105DE0008093131390931413A0931513B093161369
:105DF00080913D0290913E02A0913F02B0914002FD
:105E00008093171390931813A0931913B0931A1338
:105E100080914D0290914E02A0914F02B09150029C
:105E200080931B1390931C13A0931D13B0931E1308
:105E30008091120290911302A0911402B091150268
:105E40008093311390933213A0933313B093341390
:105E500063EB7DE087E996E10E943B734FE1A42E5E
:105E600043E1B42E5CE3C52E54E0D52EE12CF12C99
:105E700080913C0490913D048E159F051CF14601D4
:105E8000F601819191916F01F501819391935F01E9
:105E90004AE050E0B70187E996E10E94FA7369ECA5
:105EA0007DE087E996E10E942073F40160817181B1
:105EB0004AE050E087E996E10E940174FFEFEF1A93
:105EC000FF0AD6CF023040F410923E1310923D13D9
:105ED00080E090E00E942F0464E670E080E090E0B3
:105EE0000E949D6D86EE92E10E947F616EEC7DE0E6
:105EF000CE0101960E94C1764AE050E06FEF7FEF3D
:105F0000CE0101960E947C04CE0101960E94567635
:105F100061EB74E0CE0107960E94C1766DEA74E1F0
:105F2000CE0107960E947378BC01CE0101960E94B3
:105F300021774AE050E06FEF7FEFCE0101960E949B
:105F40007002CE0101960E945676CE0107960E94FD
:105F500056766CEC7DE0CE0107960E94C1766DEA24
:105F600074E1CE0107960E9473786EED7DE00E9489
:105F70008478BC01CE0101960E942177CE01019662
:105F80000E949109CE0101960E945676CE01079695
:105F90000E94567664E670E080E090E00E949D6D7D
:105FA0008DEF94E10E94B14F64E670E080E090E0F4
:105FB0000E949D6D63E270E08DEF94E10E94C44FFA
:105FC00061E070E08DEF94E10E9408048DEF94E1B0
:105FD0000E94385083E090E09093D5148093D414BD
:105FE00060E070E084EA94E10E94226D6B017C0124
:105FF00062E370E080E090E00E949D6DA701960151
:10600000C701B6010E94E97D882309F465C060E0FC
:1060100070E084EA94E10E94206D6B017C0162E3F0
:1060200070E080E090E00E949D6DA7019601C7019D
:10603000B6010E94E97D882309F44EC081E090E01A
:106040009093D5148093D41440E052EC61E070E05A
:1060500084E397E10E94050464E670E080E090E04C
:106060000E949D6D82E090E0F6DB882339F060E0CD
:106070007EE087E996E10E943B732EC01092D51412
:106080001092D41484E397E10E94B17064E670E04A
:1060900080E090E00E949D6D40E855E260E070E095
:1060A00084E397E10E94050484E397E10E94426F34
:1060B000892B91F069E17EE087E996E10E943B73CC
:1060C00082E090E09093D5148093D41464E670E05D
:1060D00080E090E00E949D6D8091D4149091D51441
:1060E000039731F463E37EE087E996E10E943B7316
:1060F00063E085ED93E10E94FE52811111C068E4D6
:106100007EE0CE0101960E94C176CE0101960E94EA
:106110009109CE0101960E94567610923C028FC0E2
:1061200040E050E0BA0185ED93E10E941E550E94C7
:10613000617B20E030E048EC52E40E94957AAB01AC
:10614000BC0122E0CE0107960E94C4776EE67EE095
:10615000CE0101960E94C176BE01695F7F4FCE01DC
:1061600001960E94737864E570E10E948478BC0116
:1061700089EB93E10E940C77CE0101960E9456763E
:10618000CE0107960E94567669EB73E187E996E1A6
:106190000E942B73609138027091390280913A020B
:1061A00090913B020E94617B20E030E048EC52E499
:1061B0000E94957AAB01BC0122E0CE0107960E94B5
:1061C000C47762E87EE0CE0101960E94C176BE01EE
:1061D000695F7F4FCE0101960E94737864E570E19C
:1061E0000E948478BC0189EB93E10E940C77CE0178
:1061F00001960E945676CE0107960E94567669EB6C
:1062000073E187E996E10E942B73113629F481E04E
:106210000E94561381E011C087E996E10E945B6FEE
:10622000182F64E670E080E090E00E949D6D1136CA
:1062300071F380E00E94561380E00E94A70964E693
:1062400070E080E090E00E949D6D8091960488232C
:1062500031F068EE73E080E090E00E949D6D67EFA2
:106260007EE085EC93E10E943F7782E090E090939E
:10627000A8138093A7138091960481110E94A811FE
:106280002C960FB6F894DEBF0FBECDBFDF91CF9135
:106290001F910F91FF90EF90DF90CF90BF90AF9044
:1062A0009F908F9008952F923F924F925F926F929E
:1062B0007F928F929F92AF92BF92CF92DF92EF9296
:1062C000FF920F931F93CF93DF93CDB7DEB72B973A
:1062D0000FB6F894DEBF0FBECDBF1C018BEB8F83D2
:1062E0008AEA888781E0898784E6829D9001839D80
:1062F000300D11243B872A87E12CF12CC12CD12CA5
:10630000812C912C5401C214D30494F1C501B40121
:106310000E94617B20E030E040E251E40E94957AE7
:106320006B017C01B101882777FD8095982F0E9431
:10633000617B9B01AC01C701B6010E94957A2B9647
:106340000FB6F894DEBF0FBECDBFDF91CF911F9186
:106350000F91FF90EF90DF90CF90BF90AF909F9004
:106360008F907F906F905F904F903F902F90089507
:106370002A853B85E216F3064CF6C7016AE070E019
:106380000E94257E892B79F4E0913417F09135171E
:106390000280F381E02D43E050E0BE01695F7F4F52
:1063A00084E397E1199565E070E080E090E00E9459
:1063B0009D6D3FEFE31AF30A00E010E0412C512CF1
:1063C000320184E397E10E94426F892B39F424E083
:1063D00042165104610471040CF095CF063011058A
:1063E0000CF091CF84E397E10E94426F892B69F012
:1063F00084E397E10E945B6FE1E0F0E0EC0FFD1FAA
:10640000E00FF11F80830F5F1F4F65E070E080E0B9
:1064100090E00E949D6D0630110501F599818F81F4
:1064200098131CC09A818885981318C09B81898510
:10643000981314C02C818D8190E0A0E0B0E0BA2FB9
:10644000A92F982F8827820F911DA11DB11D880E9D
:10645000991EAA1EBB1E8FEFC81AD80A9FEF491AB1
:10646000590A690A790AADCFCF92DF92EF92FF9273
:10647000CF93DF93CDB7DEB72C970FB6F894DEBF7E
:106480000FBECDBF84E397E10E94B17040E052ECB3
:1064900061E070E084E397E10E9405044CED55E073
:1064A00060E070E084E397E10E946E7564E670E05E
:1064B00080E090E00E949D6D60E57CE089EB93E1D7
:1064C0000E943F7769EB73E187E996E10E942B73A5
:1064D00062E370E080E090E00E949D6D69EB73E103
:1064E000CE0101960E94217742E350E06FEF7FEFEB
:1064F000CE0101960E947C04CE0101960E94567640
:106500006BEC74E083EB93E10E943F7763EB73E104
:10651000CE0101960E94217744E150E06FEF7FEFBA
:10652000CE0101960E947002CE0101960E9456761D
:106530008091D4149091D514019731F484E090E0C7
:10654000B2DE6B017C0103C0C12CD12C760180919D
:10655000D4149091D514892B29F481E090E0A3DE26
:106560006B017C0120E030E040EA51E4C701B60154
:106570000E94367C181664F521E0B701A601CE0111
:1065800007960E94C47760E17DE0CE0101960E94EB
:10659000C176BE01695F7F4FCE0101960E9473787C
:1065A0006DE07DE00E948478BC0189EB93E10E945C
:1065B0000C77CE0101960E945676CE0107960E9476
:1065C000567681E090E09093D5148093D41410C057
:1065D00069E97EE089EB93E10E943F778091D414D2
:1065E0009091D514019721F41092D5141092D414DF
:1065F00069EB73E1CE0101960E9421774AE050E0F9
:1066000060E070E0CE0101960E947C04CE0101960C
:106610000E94567669EB73E1CE0101960E942177C4
:106620006FEA74E0CE0101960E94847863EB73E117
:106630000E947378BC0189EB93E10E940C77CE0134
:1066400001960E94567684E397E10E94B170809192
:10665000AA13882331F060E273E080E090E00E94AA
:106660009D6D2C960FB6F894DEBF0FBECDBFDF91A7
:10667000CF91FF90EF90DF90CF900895FF920F930E
:106680001F93CF93DF93CDB7DEB72C970FB6F89457
:10669000DEBF0FBECDBF1092AB1366E972E18BEC8B
:1066A00093E10E943F7711E087E996E10E94426FF3
:1066B0002091AB131816190684F521112EC087E915
:1066C00096E10E945B6F8093AC138A3041F08D306D
:1066D00031F0682F8BEC93E10E94607817C0109323
:1066E000AB1365EA7EE0CE0101960E94C1766BECA9
:1066F00073E1CE0101960E947378BC0187E996E1AF
:106700000E942B73CE0101960E9456766AE070E0DB
:1067100080E090E00E949D6DC7CF222361F0209120
:10672000AB138091CF139091D01321116CC00097BF
:1067300009F069C0B0C000E010E0FF24F39481EDDF
:1067400097E10E94426F18161906A4F581ED97E1B2
:106750000E945B6F8093AC138A3071F08D3061F0D2
:106760009091AB13911108C0682F8BEC93E10E94BC
:1067700060780F5F1F4F17C08091CF139091D01397
:10678000892B89F0F092AB1381ED97E10E94426F63
:106790001816190644F466E972E18BEC93E10E9445
:1067A0003F771092AB136FE070E080E090E00E94C2
:1067B0009D6DC5CF62E370E080E090E00E949D6D2A
:1067C000012B09F4ACCF6EEA7EE0CE0101960E9467
:1067D000C1766BEC73E1CE0101960E947378BC0127
:1067E00087E996E10E942B73CE0101960E945676AE
:1067F00081ED97E10E94CA6F64E670E080E090E06E
:106800000E949D6D8CCF019709F069C06FE37DE018
:10681000CE0107960E94C176BE01695F7F4F8BEC67
:1068200093E10E94C078811115C063EB7EE0CE0138
:1068300001960E94C176BE016F5F7F4F8BEC93E1A2
:106840000E94C07811E0811110E0CE0101960E94F3
:10685000567601C010E0CE0107960E9456761123AD
:1068600099F040E050E06BEC73E1CE0101960E949C
:10687000F903BE016F5F7F4F85EC93E10E9429779A
:10688000CE0101960E94567664E170E080E090E0CF
:106890000E949D6D24C064E670E080E090E00E945C
:1068A0009D6D0E946E6DCB0168EE73E00E94257EA7
:1068B000CB0164E670E00E94257E823691057CF073
:1068C0008091AA1381110BC085EC93E10E94A479F9
:1068D000613071058105910511F40E94A8112C9673
:1068E0000FB6F894DEBF0FBECDBFDF91CF911F91E1
:1068F0000F91FF9008954F925F926F927F928F92C7
:106900009F92AF92BF92CF92DF92EF92FF92CF937E
:10691000DF93CDB7DEB760970FB6F894DEBF0FBE3A
:10692000CDBF8091AA13811105C08EE190E0A0E057
:10693000B0E004C082E090E0A0E0B0E08D879E87E8
:10694000AF87B88B65EB7EE089EB93E10E943F77E0
:1069500069EB73E1CE0101960E9421774AE050E095
:106960006FEF7FEFCE0101960E947002CE0101967B
:106970000E945676812C912C5401C12CD12C760189
:1069800063E270E08DEF94E10E94C44F67E070E035
:106990008DEF94E10E9408048DEF94E10E9438503D
:1069A00066E970E080E090E00E949D6D63E270E037
:1069B0008DEF94E10E94C44F60E270E08DEF94E1AE
:1069C0000E9408048DEF94E10E94385066E970E05F
:1069D00080E090E00E949D6D42E050E063E270E054
:1069E0008DEF94E10E943650412C512C32018DEFF5
:1069F00094E10E941C4F181619066CF48DEF94E177
:106A00000E94244F762C652C542C4424480E511C93
:106A1000611C711CECCFC301B2010E94617B2AE9A9
:106A200039E949E95FE30E94957A0E942E7BAB0128
:106A3000BC01C416D506E606F70614F46A017B010C
:106A40002AE0CE0107960E949877BE01695F7F4FCA
:106A5000CE0101960E94217765EC7EE0CE01019681
:106A60000E948478BC0183EB93E10E940C77CE01F5
:106A700001960E945676CE0107960E94567663EBE9
:106A800073E1CE0101960E9421774EE150E060E073
:106A900070E0CE0101960E940805CE0101960E9489
:106AA00056769FEF891A990AA90AB90A8D859E859B
:106AB000AF85B88988159905AA05BB050CF060CF8C
:106AC0002AE0B701A601CE0107960E949877BE0181
:106AD000695F7F4FCE0101960E94217765EC7EE0D1
:106AE000CE0101960E948478BC0183EB93E10E9461
:106AF0000C77CE0101960E945676CE0107960E9431
:106B0000567663EB73E1CE0101960E9421774AE04D
:106B100050E060E070E0CE0101960E947C04CE015E
:106B200001960E9456762AE0B701A601CE0107968B
:106B30000E94987769EC7EE0CE0101960E94C176B2
:106B4000BE01695F7F4FCE0101960E9473786CECA5
:106B50007EE00E94847869EB73E10E947378BC0147
:106B600089EB93E10E940C77CE0101960E94567644
:106B7000CE0107960E94567662E370E080E090E0D6
:106B80000E949D6D60960FB6F894DEBF0FBECDBF1C
:106B9000DF91CF91FF90EF90DF90CF90BF90AF90BB
:106BA0009F908F907F906F905F904F900895EF929D
:106BB000FF920F931F93CF93DF9300D000D0CDB7F8
:106BC000DEB78C01E090A713F090A81361ED7EE092
:106BD00087E996E10E9420734AE050E0B80187E916
:106BE00096E10E940174C8010596059700F1809115
:106BF000A7139091A8138017910709F46DC10E9403
:106C000036061093A8130093A7134AE0B801CE01EB
:106C100001960E946D77BE016F5F7F4F85EC93E117
:106C20000E942977CE0101960E94567655C10E3FEB
:106C30008FEF180709F476C1F8017996E332F10570
:106C400008F0FCC0EE58FF4F0C94767E80917004E3
:106C5000909171040E9439231FC180916404909126
:106C600065040E94B02718C1809166049091670462
:106C70000E942E2211C10E946E6D0E94362A0CC104
:106C800060E070E080916A0490916B040E940E1E97
:106C900003C180916004909161040E946425FCC04E
:106CA0008091A91391E089278093A9138091AA1359
:106CB000882331F069EB73E181ED97E10E942B733A
:106CC00068EC70E080E090E00E949D6DE5C010925D
:106CD000AA13E2C081E08093AA13DEC00E943A06A4
:106CE000DBC0C2DBD9C00E946610D6C080913C02D6
:106CF000882309F4D1C066E972E1CE0101960E94B1
:106D0000C1764AE050E061E070E0CE0101960E9459
:106D10007C04CE0101960E9456760E941E08BCC0DB
:106D2000EADDBAC080916C0490916D040E94F12656
:106D3000B3C080916204909163040E94FB25ACC0B3
:106D400080913C02882309F4A7C08091AA1388236C
:106D500029F082E090E00E947A0A9EC083E090E0F1
:106D60000E949F0E99C00E942C1C81ED97E10E9409
:106D7000CA6F92C080918102909182020E94372056
:106D80008BC080913C02882309F486C08091AA13AD
:106D900081111BC020E030E04AE754E460910A0210
:106DA00070910B0280910C0290910D020E94F57C73
:106DB00020E030E046E153E40E94957A0E942E7B69
:106DC00026E930E040E050E008C021E030E040E05B
:106DD00050E064EF71E080E090E00E9434185CC005
:106DE0008091FB149091FC14892BA1F481E090E038
:106DF0009093FC148093FB148EED93E090933E13DC
:106E000080933D130E94580468EC70E080E090E0AD
:106E10000E949D6DE091C412F091C51219953CC07D
:106E200020E042E060E18BEB94E10E941F588BEB85
:106E300094E10E9455560E9436062EC0F092A81387
:106E4000E092A7136AED7EE089EB93E10E943F7721
:106E500066E972E1CE0101960E94C1764AE050E0F7
:106E600060E070E0CE0101960E947C04CE010196A4
:106E70000E94567669EB73E1CE0101960E9421775C
:106E80004AE050E06FEF7FEFCE0101960E94700262
:106E9000CE0101960E9456768091BD139091BE134B
:106EA000009799F0419718F40230110544F569EB09
:106EB00073E1CE0101960E942177CE0101960E94D6
:106EC0009109CE0101960E94567664E670E080E05A
:106ED00090E00E949D6D26C06FEA74E0CE0101969D
:106EE0000E94C1764AE050E06FEF7FEFCE0101963D
:106EF0000E940805CE0101960E9456769DCE69EB50
:106F000073E1CE0101960E9421774AE050E06FEFD5
:106F10007FEFCE0101960E947002CE0101960E9481
:106F20005676C5CF26960FB6F894DEBF0FBECDBFFE
:106F3000DF91CF911F910F91FF90EF900895FF92F5
:106F40000F931F93CF93DF9300D000D0CDB7DEB760
:106F5000823409F472C0D4F4803309F48EC07CF416
:106F6000833209F481C08A3209F0A5C069EF7EE05E
:106F70008BEC93E10E943F778FEF9FEFF8C0813356
:106F800009F48AC0813409F44DC095C0813609F4F2
:106F900049C034F4833409F45BC0843449F08BC0B5
:106FA000833609F455C00CF448C0843609F083C018
:106FB0008091C9139091CA13892B09F4DAC085EC2A
:106FC00093E10E94A47997FDD4C067EE7EE087E943
:106FD00096E10E94207365EC73E187E996E10E94D7
:106FE0002B7385EC93E10E94A479DC01CB014AEF7D
:106FF0005FEF6FEF7FEF481B590B6A0B7B0B2AE0AB
:10700000CE0101960E949877BE016F5F7F4F85EC9D
:1070100093E10E942977CE0101960E94567685EC75
:1070200093E1A2C06DEE7EE08BEC93E10E943F778E
:107030008091A7139091A8139AC060EF7EE08BEC2B
:1070400093E10E943F771092AA138CEF9FEF8FC0BD
:1070500063EF7EE08BEC93E10E943F7781E08093C9
:10706000AA138DEF9FEF83C066EF7EE08BEC93E178
:107070000E943F778EEF9FEF7AC067E07FE085EC5C
:1070800093E10E943F7767E07FE08BEC93E10E9401
:107090003F7780E090E06BC06AEF7EE085EC93E1A3
:1070A0000E943F776AEF7EE08BEC93E10E943F778E
:1070B00081E090E05CC0682FCE0101960E94557778
:1070C000BE016F5F7F4F85EC93E10E942977CE016F
:1070D00001960E94567685EC93E10E94A479CB013B
:1070E00066DD64E670E080E090E00E949D6D49C03E
:1070F0000F5F1F4F093E83E0180769F06EE170E0F3
:1071000080E090E00E949D6D85E394E10E94215B08
:10711000F82EFF2069F36AE270E06F197109F7FC3D
:1071200073954AE0CE0101960E946D77BE016F5FB4
:107130007F4F8BEC93E10E942977CE0101960E944C
:1071400056766BEC73E185EC93E10E940C7767EE69
:107150007EE087E996E10E9420736F2D87E996E132
:107160000E944B738BEC93E10E94A479CB011FDD4D
:1071700008C085E394E10E94215BF82E00E010E056
:10718000C8CF26960FB6F894DEBF0FBECDBFDF91F5
:10719000CF911F910F91FF9008950F931F93CF935D
:1071A000DF9300D000D0CDB7DEB74091DA12509116
:1071B000DB126091DC127091DD1220E130E087E992
:1071C00096E10E9448748091DA129091DB12A091AE
:1071D000DC12B091DD12883025E09207A105B105DF
:1071E00009F4F7C108F08DC0893421E09207A105A8
:1071F000B10509F4F1C1E0F5843421E09207A1055D
:10720000B10509F4DAC1E8F4813421E09207A1055F
:10721000B10509F4C3C138F480349140A105B1052A
:1072200009F4ADC1DCC1823421E09207A105B105AA
:1072300009F4BDC183349140A105B10509F4BAC177
:10724000CEC1863421E09207A105B10509F4BBC186
:1072500008F4B6C1873421E09207A105B10509F40D
:10726000B5C188349140A105B10509F4B2C1B7C1D7
:10727000823025E09207A105B10509F498C1E8F430
:10728000843721E09207A105B10509F443C138F420
:1072900082379140A105B10509F447C1A0C181150C
:1072A00025E09207A105B10509F469C18130954037
:1072B000A105B10509F472C192C1853025E092079C
:1072C000A105B10509F47CC170F4833025E0920773
:1072D000A105B10509F46EC184309540A105B10541
:1072E00009F46BC17CC1863025E09207A105B10588
:1072F00009F469C187309540A105B10509F466C15B
:107300006EC18D3B22E492072FEFA207B10509F46D
:1073100027C108F04BC08F3E20E192072FEFA20754
:10732000B10509F453C118F5823325E09207A10590
:10733000B10509F4FAC038F489309540A105B105CA
:1073400009F44AC14CC1843325E09207A105B10577
:1073500009F4E0C08D3F9240AF4FB10509F03FC145
:107360006DEE7EE08BEC93E10E943F77DBC08D3DBC
:1073700022E292072FEFA207B10509F4CBC038F43F
:10738000873E9841AF4FB10509F41AC128C18F3C1F
:1073900020E392072FEFA207B10509F40EC1873C45
:1073A0009843AF4FB10509F414C119C1873928E6D4
:1073B00092072FEFA207B10509F4F0C048F58D3A06
:1073C00022E592072FEFA207B10509F4BAC038F4FD
:1073D000853B9A44AF4FB10509F4D1C000C1853A4D
:1073E0002AE592072FEFA207B10509F4F5C08D3900
:1073F0009246AF4FB10509F0F2C060EF7EE08BEC32
:1074000093E10E943F771092AA138CEF9FEF80C008
:10741000873528EA92072FEFA207B105F9F078F433
:1074200085382AE792072FEFA207B10509F4CBC0F0
:1074300087369849AF4FB10509F4B9C0D0C08F3431
:1074400020EB92072FEFA207B10509F4B3C08D33EB
:10745000924CAF4FB10509F468C0C1C086EE92E10D
:107460000E94966100E010E066EC72E186EE92E127
:107470000E944B62892B39F40F5F1F4F093E83E056
:10748000180709F031C16DE07FE087E996E10E94BD
:1074900020734091CA125091CB126091CC1270911E
:1074A000CD122AE030E087E996E10E94487480918D
:1074B000CA129091CB12A091CC12B091CD12833010
:1074C00025E09207A105B10509F4C8C008F0AFC0D6
:1074D000843421E09207A105B10509F4CFC008F07A
:1074E000D6C0823421E09207A105B10509F4D7C0C6
:1074F00008F0B4C081349140A105B10509F082C003
:107500006CEF7EE085EC93E10E943F7789EF9FEF7F
:107510004EDB7EC06DEE7EE08BEC93E10E943F7708
:107520001092AA138BEF9FEFF3CF63EF7EE08BEC0B
:1075300093E10E943F7781E08093AA138DEF9FEF44
:10754000E7CF66EF7EE085EC93E10E943F7766EF40
:107550007EE08BEC93E10E943F778EEF9FEFD8CFD8
:1075600069EF7EE085EC93E10E943F7769EF7EE072
:107570008BEC93E10E943F778FEF9FEFC9CF67E0DD
:107580007FE085EC93E10E943F7767E07FE08BEC42
:1075900093E10E943F7780E090E0BACF6AEF7EE00F
:1075A00085EC93E10E943F7781E090E0B1CF82E0EB
:1075B00090E0AECF83E090E0ABCF84E090E0A8CF46
:1075C00085E090E0A5CF86E090E0A2CF87E090E054
:1075D0009FCF88E090E09CCF89E090E099CF40E099
:1075E00050E06BEC73E1CE0101960E94F903BE01FD
:1075F0006F5F7F4F85EC93E10E942977CE01019662
:107600000E94567664E670E080E090E00E949D6DF6
:1076100086EE92E10E94966126960FB6F894DEBF40
:107620000FBECDBFDF91CF911F910F9108958F3C79
:1076300020E392072FEFA207B10501F1C0F08736D2
:1076400028E992072FEFA207B10549F18F3420EB0B
:1076500092072FEFA207B10509F03FC062E07FE07B
:1076600085EC93E10E943F7787EF9FEF51CF853004
:1076700025E09207A105B10509F148F565E07FE035
:1076800085EC93E10E943F7786EF9FEF41CF8130F9
:1076900025E09207A105B10509F432CF48F06FEF5C
:1076A0007EE085EC93E10E943F7788EF9FEF30CF3B
:1076B00085349140A105B10509F0A4CF69E07FE0D0
:1076C00085EC93E10E943F7785EF9FEF21CF873EC6
:1076D0009841AF4FB10591F395CF87399846AF4F99
:1076E000B10509F08FCF0CCF6EE170E080E090E043
:1076F0000E949D6DB9CE8F929F92AF92BF92CF9212
:10770000DF92EF92FF920F931F93CF93DF93CDB74A
:10771000DEB7A6970FB6F894DEBF0FBECDBF66EDFD
:1077200072E186EE92E10E944B62892BD9F08BEBDD
:1077300094E10E9455560E9436066FEA74E0CE012D
:1077400001960E94C1764AE050E060E070E0CE0110
:1077500001960E947C04CE0101960E9456761DDDA2
:107760000C94574C66E972E18BEC93E10E943F77F1
:107770000E943E336AE070E080E090E00E949D6DE0
:107780008091CF139091D013009711F40C94384C42
:10779000019709F046C06DE27DE0CE010F960E9490
:1077A000C176BE01615F7F4F8BEC93E10E94C07890
:1077B00081112AC06EE07DE0CE0109960E94C1765B
:1077C000BE01675F7F4F8BEC93E10E94C07881110F
:1077D00015C069E877E0CE0101960E94C176BE012E
:1077E0006F5F7F4F8BEC93E10E94C07811E08111B5
:1077F00010E0CE0101960E94567601C010E0CE0145
:1078000009960E94567601C010E0CE010F960E94A4
:107810005676112331F06BEC73E185EC93E10E9415
:107820000C778091CF139091D0130497F0F562EF0D
:1078300075E0CE0101960E94C176BE016F5F7F4F59
:107840008BEC93E10E94C078182FCE0101960E9424
:107850005676112351F141E050E06BEC73E1CE011B
:1078600009960E94F903CE0109960E94A479DC01D1
:10787000CB014AEF5FEF6FEF7FEF481B590B6A0BAD
:107880007B0B2AE0CE0101960E949877BE016F5FC4
:107890007F4F85EC93E10E942977CE0101960E94EB
:1078A0005676CE0109960E9456766FE17FE0CE01B2
:1078B00009960E94C176BE01675F7F4F8BEC93E112
:1078C0000E94C078811116C063E27FE0CE0101966C
:1078D0000E94C176BE016F5F7F4F8BEC93E10E94E7
:1078E000C07811E0811101C010E0CE0101960E9424
:1078F000567601C011E0CE0109960E9456761123FA
:1079000009F4EFC267E27FE0CE0101960E94C176E2
:10791000CE0101960E949109CE0101960E945676F1
:10792000609138027091390280913A0290913B0245
:107930000E94617B20E030E048EC52E40E94957A9E
:10794000AB01BC0122E0CE010F960E94C47763E335
:107950007FE0CE0109960E94C176BE01615F7F4F34
:10796000CE0109960E94737864E570E10E948478E4
:10797000BC01CE0101960E942177CE0101960E94A2
:107980009109CE0101960E945676CE0109960E9479
:107990005676CE010F960E94567640913402509151
:1079A0003502609136027091370224E0CE010F96C5
:1079B0000E94C47768E47FE0CE0109960E94C176F8
:1079C000BE01615F7F4FCE0109960E947378BC01B2
:1079D000CE0101960E942177CE0101960E94910965
:1079E000CE0101960E945676CE0109960E945676E7
:1079F000CE010F960E94567640911E0250911F02B2
:107A0000609120027091210222E0CE0109960E942D
:107A1000C47740911602509117026091180270913C
:107A2000190223E0CE010F960E94C47740912202F2
:107A300050912302609124027091250222E0CE0130
:107A400045960E94C47740911A0250911B026091A2
:107A50001C0270911D0223E0CE0181960E94C47722
:107A600065E67FE0CE014B960E94C176BE016F5D58
:107A70007F4FCE014B960E9473786AE77FE00E94A9
:107A80008478BE016B5E7F4F0E9473786DE77FE064
:107A90000E948478BE01615F7F4F0E9473786AE71D
:107AA0007FE00E948478BE01675F7F4F0E947378F9
:107AB00063E87FE00E948478BC01CE0101960E94B9
:107AC0002177CE0101960E949109CE0101960E9474
:107AD0005676CE014B960E945676CE0181960E9434
:107AE0005676CE0145960E945676CE010F960E949C
:107AF0005676CE0109960E94567668E87FE0CE0160
:107B000009960E94C1766DEA74E1CE0109960E9441
:107B10007378BC01CE0101960E942177CE010196B7
:107B20000E949109CE0101960E945676CE010996D7
:107B30000E9456764091450250914602609147025C
:107B40007091480223E0CE0109960E94C4772091EB
:107B5000490230914A0240914B0250914C0260E040
:107B600070E080E291E40E94587DAB01BC0121E00D
:107B7000CE0145960E94F27769E97FE0CE010F962B
:107B80000E94C176BE016B5E7F4FCE010F960E94B0
:107B900073786CEA7FE00E948478BE01675F7F4F54
:107BA0000E9473786FE27DE00E948478BC01CE0170
:107BB00001960E942177CE0101960E949109CE0183
:107BC00001960E945676CE010F960E945676CE01FF
:107BD00045960E945676CE0109960E9456764091AF
:107BE000410250914202609143027091440223E0AD
:107BF000CE0109960E94C47720913D0230913E0249
:107C000040913F025091400260E070E080E291E4D8
:107C10000E94587DAB01BC0121E0CE0145960E9437
:107C2000F27762EB7FE0CE010F960E94C176BE0133
:107C30006B5E7F4FCE010F960E9473786CEA7FE0F7
:107C40000E948478BE01675F7F4F0E9473786FE265
:107C50007DE00E948478BC01CE0101960E942177CC
:107C6000CE0101960E949109CE0101960E9456769E
:107C7000CE010F960E945676CE0145960E9456760A
:107C8000CE0109960E94567640914D0250914E02C7
:107C900060914F027091500222E0CE010F960E9437
:107CA000C47765EC7FE0CE0109960E94C176BE01E3
:107CB000615F7F4FCE0109960E9473786BED7FE084
:107CC0000E948478BC01CE0101960E942177CE01EA
:107CD00001960E949109CE0101960E945676CE012E
:107CE00009960E945676CE010F960E9456764091D4
:107CF000120250911302609114027091150222E059
:107D0000CE010F960E94C47762EE7FE0CE01099605
:107D10000E94C176BE01615F7F4FCE0109960E942D
:107D200073786FE27DE00E948478BC01CE010196F9
:107D30000E942177CE0101960E949109CE01019601
:107D40000E945676CE0109960E945676CE010F9675
:107D50000E9456760EE3C02E04E0D02E01E010E023
:107D600085E1E82E80913C0490913D0480179107B5
:107D70000CF44FC0F601A190B1906F014AE0B5013B
:107D8000CE0109960E946D774AE0B801CE01459672
:107D90000E946D7765EF7FE0CE010F960E94C1765D
:107DA000BE016B5E7F4FCE010F960E9473786FE02D
:107DB00077E00E948478BE01675F7F4F0E947378EE
:107DC0006DEF7FE00E948478EA9CB001EB9C700D1F
:107DD00011246D577D4F0E948478BC01CE0101961D
:107DE0000E942177CE0101960E949109CE01019651
:107DF0000E945676CE010F960E945676CE01459689
:107E00000E945676CE0109960E9456760F5F1F4F4C
:107E1000A9CF40910E0250910F0260911002709113
:107E2000110222E0CE010F960E94C47763E070E158
:107E3000CE0109960E94C176BE01615F7F4FCE01DF
:107E400009960E9473786FE37DE00E948478BC01FC
:107E5000CE0101960E942177CE0101960E949109E0
:107E6000CE0101960E945676CE0109960E94567662
:107E7000CE010F960E94567640910A0250910B0255
:107E800060910C0270910D0222E0CE010F960E94CB
:107E9000C47763E170E1CE0109960E94C176BE010C
:107EA000615F7F4FCE0109960E9473786FE37DE09A
:107EB0000E948478BC01CE0101960E942177CE01F8
:107EC00001960E949109CE0101960E945676CE013C
:107ED00009960E945676CE010F960E94567610E0C3
:107EE00001C011E08BEB94E10E9455560E943606CA
:107EF0006FEA74E0CE0101960E94C1764AE050E03C
:107F000060E070E0CE0101960E940805CE01019666
:107F10000E9456768091CF139091D01383309105B3
:107F200008F06FC0019739F460E070E08BEC93E1EA
:107F30000E94DF78F82E8091CF139091D013029792
:107F400009F050C062EF75E0CE0101960E94C17643
:107F5000BE016F5F7F4F8BEC93E10E94C078182FBA
:107F6000CE0101960E9456761123E1F161E070E0A6
:107F70008BEC93E10E94DF78682FCE0101960E947E
:107F80005577BE016F5F7F4F85EC93E10E94347798
:107F9000CE0101960E94567660E070E08BEC93E192
:107FA0000E94DF78F82E6EE070E1CE0101960E940B
:107FB000C1766BEC73E1CE0101960E9473786FEA93
:107FC00074E00E948478BC0187E996E10E941273F4
:107FD000CE0101960E94567665EC73E187E996E141
:107FE0000E942B738F2D0E949F370E946E6D6093AD
:107FF000D1137093D2138093D3139093D4130C9412
:10800000574C21E030E040E050E06BEC73E1CE01F2
:1080100001960E946179BE016F5F7F4F83EB93E110
:108020000E942977CE0101960E94567660E570E1A4
:10803000CE0109960E94C176BE01675F7F4F8BEC2F
:1080400093E10E94C078811116C063E87CE0CE0104
:1080500001960E94C176BE016F5F7F4F8BEC93E16A
:108060000E94C07801E0811101C000E0CE010196BC
:108070000E94567601C001E0CE0109960E94567614
:10808000002309F4CDC042E050E06BEC73E1CE0177
:1080900001960E94F903BE016F5F7F4F83EB93E16E
:1080A0000E942977CE0101960E94567663EB73E118
:1080B00087E996E10E942B7383EB93E10E94AE79EE
:1080C00020E030E048EC52E40E94F57C0E942E7BD8
:1080D000AB01BC01409338025093390260933A02DD
:1080E00070933B022AE030E087E996E10E94177422
:1080F000609138027091390280913A0290913B026E
:108100008B019C0100591F452140310901341C4954
:1081100021053105D0F063E270E1CE0101960E94A5
:10812000C17663EB73E1CE0101960E94737866E33A
:1081300070E10E948478BC0189EB93E10E940C7786
:10814000CE0101960E9456764DC019821A821B827A
:108150001C821D821E821F8218860E94617B20E085
:1081600030E048EC52E40E94957A8E010F5F1F4F79
:1081700022E047E00E94D67EBC0189EB93E10E9499
:108180003F7766E470E1CE0109960E94C17669EB03
:1081900073E1CE0109960E94737863E570E10E9455
:1081A0008478BC0189EB93E10E940C77CE0109969B
:1081B0000E94567610923E1310923D138091380221
:1081C00090913902A0913A02B0913B028093E7125C
:1081D0009093E812A093E912B093EA1280E090E045
:1081E0000E942F046CEC7DE0CE0109960E94C176BE
:1081F00069EB73E1CE0109960E947378BC01CE0150
:1082000001960E942177CE0101960E949109CE012C
:1082100001960E945676CE0109960E94567610E08D
:1082200068E570E1CE0109960E94C176BE01675FE4
:108230007F4F8BEC93E10E94C078811116C06EE5F0
:1082400070E1CE0101960E94C176BE016F5F7F4F43
:108250008BEC93E10E94C07801E0811101C000E045
:10826000CE0101960E94567601C001E0CE0109962A
:108270000E945676002309F475C026E030E045E000
:1082800050E06BEC73E1CE0101960E946179BE0172
:108290006F5F7F4F83EB93E10E942977CE010196B8
:1082A0000E94567683EB93E10E94A4796B017C01D6
:1082B00069ED7FE0CE0109960E94C176BE01675F3D
:1082C0007F4F8BEC93E10E945879AC014F5F5F4F79
:1082D0006BEC73E1CE0101960E94F903BE016F5F62
:1082E0007F4F83EB93E10E942977CE0101960E9494
:1082F0005676CE0109960E94567683EB93E10E9452
:10830000A479DB01EEE3F4E021E030E040913C04AD
:1083100050913D04421753075CF0408151814A1748
:108320005B0711F4118210822F5F3F4F3296EECF20
:10833000F601EE0FFF1FE45CFB4F7183608382E068
:1083400090E00E9464286BEC73E187E996E10E945B
:108350002B7310923E1310923D1380E090E00E9428
:108360002F0410E064E670E1CE0109960E94C17608
:10837000BE01675F7F4F8BEC93E10E94C078811153
:1083800016C06AE670E1CE0101960E94C176BE0178
:108390006F5F7F4F8BEC93E10E94C07801E0811109
:1083A00001C000E0CE0101960E94567601C001E0B6
:1083B000CE0109960E945676002331F1EEE3F4E0F7
:1083C00081E090E020913C0430913D04281739076A
:1083D00074F0863091051CF49183808305C09C0164
:1083E0002E5F3F4F3183208301963296EBCF82E0A0
:1083F00090E00E94642810923E1310923D1380E09A
:1084000090E00E942F0410E060E770E1CE01099631
:108410000E94C176BE01675F7F4F8BEC93E10E94A3
:10842000C078811116C068E770E1CE0101960E9404
:10843000C176BE016F5F7F4F8BEC93E10E94C078E5
:1084400001E0811101C000E0CE0101960E94567644
:1084500001C001E0CE0109960E945676002399F1F1
:1084600060E870E1CE0101960E94C17667EA74E18E
:10847000CE0101960E947378BC0189EB93E10E94C2
:108480000C77CE0101960E9456766CEC7DE0CE0111
:1084900009960E94C17669EB73E1CE0109960E94AC
:1084A0007378BC01CE0101960E942177CE0101961E
:1084B0000E949109CE0101960E945676CE0109963E
:1084C0000E94567610E06AE870E1CE0109960E949B
:1084D000C176BE01675F7F4F8BEC93E10E94C0784D
:1084E000811116C06EE870E1CE0101960E94C1763E
:1084F000BE016F5F7F4F8BEC93E10E94C07801E07B
:10850000811101C000E0CE0101960E94567601C0A3
:1085100001E0CE0109960E945676002309F460C05E
:1085200043E050E06BEC73E1CE0101960E94F90349
:10853000BE016F5F7F4F83EB93E10E942977CE01ED
:1085400001960E94567663EB73E187E996E10E94FB
:108550002B7310923E1310923D1363EB73E18DEA7F
:1085600094E10E940C7720E030E048E050E063E0C6
:1085700073E18DEA94E10E94E07880913D1390913F
:108580003E130E942F0462E970E1CE0101960E9421
:10859000C1766DEA74E1CE0101960E947378BC0148
:1085A000CE0109960E942177CE0101960E9456764F
:1085B000BE01675F7F4F81ED97E10E94127368EB08
:1085C0007BE080E090E00E949D6D63E073E187E9CD
:1085D00096E10E943B73CE0109960E94567610E008
:1085E0006AE970E1CE0109960E94C176BE01675F1B
:1085F0007F4F8BEC93E10E94C078811116C06DEF24
:108600007CE0CE0101960E94C176BE016F5F7F4F74
:108610008BEC93E10E94C07801E0811101C000E081
:10862000CE0101960E94567601C001E0CE01099666
:108630000E945676002309F441C044E050E06BEC00
:1086400073E1CE0101960E94F903BE016F5F7F4F77
:1086500083EB93E10E942977CE0101960E94567622
:108660006FE970E1CE0101960E94C17663EB73E180
:10867000CE0101960E947378BC01CE0109960E943A
:108680002177CE0101960E945676BE01675F7F4F2B
:1086900081ED97E10E94127368EB7BE080E090E04F
:1086A0000E949D6DBE01675F7F4F87E996E10E9442
:1086B0002B73CE0109960E94567610E066EA70E1AF
:1086C000CE010F960E94C176BE01615F7F4F8BEC99
:1086D00093E10E94C07881112BC069EA70E1CE015C
:1086E00009960E94C176BE01675F7F4F8BEC93E1D4
:1086F0000E94C078811116C06CEA70E1CE0101962B
:108700000E94C176BE016F5F7F4F8BEC93E10E94A8
:10871000C07801E0811101C000E0CE0101960E9405
:10872000567601C001E0CE0109960E94567601C03E
:1087300001E0CE010F960E945676002309F42CC169
:10874000AAE0AA2EB12CC12CD12C760188248A94BF
:10875000B3E09B2E6EE170E080E090E00E949D6DA2
:10876000809181020E94336EB4010E94257E882789
:1087700077FD8095982F0E94617B20E030E040EAF1
:1087800050E40E94F57C9B01AC01C701B6010E9438
:10879000CB796B017C0121E0A21AB108D9F620E067
:1087A00030E040E251E40E94957A6B017C016FEA6F
:1087B00070E1CE0109960E94C176BE01675F7F4FCE
:1087C0008BEC93E10E94C078811116C063EB70E1DD
:1087D000CE0101960E94C176BE016F5F7F4F8BEC88
:1087E00093E10E94C07801E0811101C000E0CE0158
:1087F00001960E94567601C001E0CE0109960E94C2
:108800005676002309F43FC020E030E040E650E413
:10881000C701B6010E94F57C9B01AC0160E070E0ED
:1088200080E890E40E94CA79AB01BC0140932A021F
:1088300050932B0260932C0270932D0222E0CE0104
:1088400001960E94C477BE016F5F7F4F89EB93E171
:108850000E942977CE0101960E94567667EB70E15F
:10886000CE0101960E94C17669EB73E1CE010196BB
:108870000E947378BC0189EB93E10E940C77CE01D2
:1088800001960E94567666EC70E1CE0109960E9430
:10889000C176BE01675F7F4F8BEC93E10E94C07889
:1088A000811116C06BEC70E1CE0101960E94C17679
:1088B000BE016F5F7F4F8BEC93E10E94C07801E0B7
:1088C000811101C000E0CE0101960E94567601C0E0
:1088D00001E0CE0109960E945676002309F43FC0BC
:1088E00020E030E040E650E4C701B6010E94F57C8C
:1088F0009B01AC0160E070E080E291E40E94CA79E3
:10890000AB01BC01409326025093270260932802DA
:108910007093290222E0CE0101960E94C477BE0125
:108920006F5F7F4F89EB93E10E942977CE0101961B
:108930000E94567660ED70E1CE0101960E94C176EC
:1089400069EB73E1CE0101960E947378BC0189EB5B
:1089500093E10E940C77CE0101960E9456766CEC52
:108960007DE0CE0109960E94C17669EB73E1CE01EC
:1089700009960E947378BC01CE0101960E9421776E
:10898000CE0101960E949109CE0101960E94567671
:10899000CE0109960E94567660EE70E1CE010196F6
:1089A0000E94C176BE016F5F7F4F8BEC93E10E9406
:1089B000C078082FCE0101960E945676002309F454
:1089C0006DC08091CF139091D013079708F466C0C3
:1089D00046E050E06BEC73E1CE0101960E94F90392
:1089E000BE016F5F7F4F83EB93E10E942977CE0139
:1089F00001960E94567683EB93E10E94AE79AB011B
:108A0000BC0140930E0250930F02609310027093CA
:108A1000110221E0CE0109960E94C47763E070E163
:108A2000CE0101960E94C176BE01675F7F4FCE01E5
:108A300001960E9473786FE37DE00E948478BC0108
:108A400089EB93E10E940C77CE0101960E94567645
:108A5000CE0109960E94567669EB73E1CE0101962C
:108A60000E942177CE0101960E949109CE010196C4
:108A70000E9456760E946E6D28EE33E040E050E092
:108A80000E94387ECA01B9010E945F7B609339134E
:108A900070933A1380933B1390933C1367EE70E10D
:108AA000CE0101960E94C176BE016F5F7F4F8BECB5
:108AB00093E10E94C078082FCE0101960E9456765D
:108AC000002309F45AC08091CF139091D0130797D7
:108AD00008F453C046E050E06BEC73E1CE01019620
:108AE0000E94F903BE016F5F7F4F83EB93E10E9409
:108AF0002977CE0101960E94567683EB93E10E947E
:108B0000AE79AB01BC0140930A0250930B02609313
:108B10000C0270930D0221E0CE0109960E94C477E9
:108B200063E170E1CE0101960E94C176BE01675FEC
:108B30007F4FCE0101960E9473786FE37DE00E9423
:108B40008478BC0189EB93E10E940C77CE010196F9
:108B50000E945676CE0109960E94567669EB73E123
:108B6000CE0101960E942177CE0101960E949109C3
:108B7000CE0101960E94567610E06EEE70E1CE01B5
:108B800009960E94C176BE01675F7F4F8BEC93E12F
:108B90000E94C078811116C062EF70E1CE0101968B
:108BA0000E94C176BE016F5F7F4F8BEC93E10E9404
:108BB000C07801E0811101C000E0CE0101960E9461
:108BC000567601C001E0CE0109960E945676002338
:108BD00009F47CC080916A0490916B040E94E31DAB
:108BE00060931A0270931B0280931C0290931D02E3
:108BF0006093FB127093FC128093FD129093FE120F
:108C000080E090E0A0E8BFE38093220290932302EB
:108C1000A0932402B09325028093F3129093F41250
:108C2000A093F512B093F61266EF70E187E996E132
:108C30000E94207340911A0250911B0260911C0205
:108C400070911D0222E030E087E996E10E943275C2
:108C500010923E1310923D1380E090E00E942F048A
:108C600040911A0250911B0260911C0270911D02EA
:108C700022E0CE0109960E94C47761E171E1CE0144
:108C800001960E94C176BE01675F7F4FCE010196BB
:108C90000E947378BC0189EB93E10E940C77CE01AE
:108CA00001960E945676CE0109960E94567669EB8F
:108CB00073E1CE0101960E942177CE0101960E94B8
:108CC0009109CE0101960E94567610E06AE171E1A9
:108CD000CE0109960E94C176BE01675F7F4F8BEC83
:108CE00093E10E94C078811116C060E271E1CE016B
:108CF00001960E94C176BE016F5F7F4F8BEC93E1BE
:108D00000E94C07801E0811101C000E0CE0101960F
:108D10000E94567601C001E0CE0109960E94567667
:108D2000002309F48BC08091CF139091D013079743
:108D3000F8F046E050E06BEC73E1CE0101960E9442
:108D4000F903BE016F5F7F4F83EB93E10E942977A8
:108D5000CE0101960E94567683EB93E10E94AE7994
:108D600060934D0270934E0280934F029093500295
:108D7000809164040E94272880914D0290914E02B8
:108D8000A0914F02B091500280931B1390931C133B
:108D9000A0931D13B0931E1366E271E187E996E17B
:108DA0000E94207340914D0250914E0260914F02FB
:108DB0007091500222E030E087E996E10E9432751E
:108DC00010923E1310923D1380E090E00E942F0419
:108DD00040914D0250914E0260914F0270915002AD
:108DE00022E0CE0109960E94C47767E371E1CE01CB
:108DF00001960E94C176BE01675F7F4FCE0101964A
:108E00000E947378BC0189EB93E10E940C77CE013C
:108E100001960E945676CE0109960E94567669EB1D
:108E200073E1CE0101960E942177CE0101960E9446
:108E30009109CE0101960E94567610E061E471E13D
:108E4000CE0109960E94C176BE01675F7F4F8BEC11
:108E500093E10E94C078811116C066E471E1CE01F1
:108E600001960E94C176BE016F5F7F4F8BEC93E14C
:108E70000E94C07801E0811101C000E0CE0101969E
:108E80000E94567601C001E0CE0109960E945676F6
:108E9000002309F4C5C08091CF139091D013069799
:108EA00008F145E050E06BEC73E1CE0101960E94C1
:108EB000F903BE016F5F7F4F83EB93E10E94297737
:108EC000CE0101960E94567683EB93E10E94AE7923
:108ED0000E94777C6093490270934A0280934B0210
:108EE00090934C0280916604909167040E947621D1
:108EF00020E030E048E051E40E94957A609345021A
:108F000070934602809347029093480260930B133C
:108F100070930C1380930D1390930E13809149025C
:108F200090914A02A0914B02B0914C02809313138E
:108F300090931413A0931513B09316136BE471E17F
:108F400087E996E10E9420732091490230914A02FC
:108F500040914B0250914C0260E070E080E291E45D
:108F60000E94587DAB01BC0121E030E087E996E129
:108F70000E9431756BE571E187E996E10E942073EB
:108F8000409145025091460260914702709148021B
:108F900022E030E087E996E10E94327510923E139C
:108FA00010923D1380E090E00E942F044091450212
:108FB00050914602609147027091480223E0CE0131
:108FC00009960E94C47762E671E1CE0101960E9483
:108FD000C176BE01675F7F4FCE0101960E94737814
:108FE0006DE97CE00E948478BC0189EB93E10E94EA
:108FF0000C77CE0101960E945676CE0109960E940A
:10900000567669EB73E1CE0101960E942177CE017D
:1090100001960E949109CE0101960E94567610E0B9
:109020006BE671E1CE0109960E94C176BE01675FD1
:109030007F4F8BEC93E10E94C078811116C060E7EE
:1090400071E1CE0101960E94C176BE016F5F7F4F34
:109050008BEC93E10E94C07801E0811101C000E037
:10906000CE0101960E94567601C001E0CE0109961C
:109070000E945676002309F4C5C08091CF139091C9
:10908000D013069708F145E050E06BEC73E1CE0198
:1090900001960E94F903BE016F5F7F4F83EB93E15E
:1090A0000E942977CE0101960E94567683EB93E1C8
:1090B0000E94AE790E94777C60933D0270933E02DD
:1090C00080933F02909340028091660490916704E0
:1090D0000E94762120E030E048E051E40E94957A39
:1090E0006093410270934202809343029093440242
:1090F00060930F13709310138093111390931213B6
:1091000080913D0290913E02A0913F02B0914002B9
:109110008093171390931813A0931913B0931A13F5
:1091200065E771E187E996E10E94207320913D0295
:1091300030913E0240913F025091400260E070E069
:1091400080E291E40E94587DAB01BC0121E030E057
:1091500087E996E10E9431756BE571E187E996E157
:109160000E9420734091410250914202609143025B
:109170007091440222E030E087E996E10E94327566
:1091800010923E1310923D1380E090E00E942F0455
:109190004091410250914202609143027091440219
:1091A00023E0CE0109960E94C47764E871E1CE0104
:1091B00001960E94C176BE01675F7F4FCE01019686
:1091C0000E9473786DE97CE00E948478BC0189EB91
:1091D00093E10E940C77CE0101960E945676CE0153
:1091E00009960E94567669EB73E1CE0101960E94C2
:1091F0002177CE0101960E949109CE0101960E942D
:10920000567610E06DE871E1CE0109960E94C176B4
:10921000BE01675F7F4F8BEC93E10E94C0788111A4
:1092200016C061E971E1CE0101960E94C176BE01CE
:109230006F5F7F4F8BEC93E10E94C07801E081115A
:1092400001C000E0CE0101960E94567601C001E007
:10925000CE0109960E945676002309F48CC060E086
:10926000809170040E94AC6E09E110E0C12CD12CF9
:109270007601809170040E94336EBC01882777FDCF
:109280008095982F0E94617B9B01AC01C701B601BC
:109290000E94CB796B017C016AE070E080E090E095
:1092A0000E949D6D0150110921F720E030E040EA55
:1092B00050E4C701B6010E94F57C20E030E040E8B0
:1092C0005AE30E94F57C20E030E048EC51E40E9433
:1092D000957A609312027093130280931402909314
:1092E000150260933113709332138093331390936C
:1092F000341310923E1310923D1380E090E00E94D0
:109300002F04409112025091130260911402709147
:10931000150222E0CE0109960E94C47762EE7FE03A
:10932000CE0101960E94C176BE01675F7F4FCE01DC
:1093300001960E9473786FE27DE00E948478BC0100
:1093400089EB93E10E940C77CE0101960E9456763C
:10935000CE0109960E94567669EB73E1CE01019623
:109360000E942177CE0101960E949109CE010196BB
:109370000E94567610E065E971E1CE0109960E94DF
:10938000C176BE01675F7F4F8BEC93E10E94C0788E
:10939000811116C069E971E1CE0101960E94C17682
:1093A000BE016F5F7F4F8BEC93E10E94C07801E0BC
:1093B000811101C000E0CE0101960E94567601C0E5
:1093C00001E0CE0109960E945676002309F47CC084
:1093D00080916A0490916B040E94E31D60931602D1
:1093E0007093170280931802909319026093FF12F2
:1093F00070930013809301139093021380E090E523
:10940000A3ECB7E480931E0290931F02A093200266
:10941000B09321028093F7129093F812A093F9125F
:10942000B093FA126DE971E187E996E10E94207329
:109430004091160250911702609118027091190222
:1094400022E030E087E996E10E94327510923E13E7
:1094500010923D1380E090E00E942F04409116028C
:1094600050911702609118027091190222E0CE010A
:1094700009960E94C4776AEB71E1CE0101960E94C1
:10948000C176BE01675F7F4FCE0101960E9473785F
:10949000BC0189EB93E10E940C77CE0101960E94FA
:1094A0005676CE0109960E94567669EB73E1CE019D
:1094B00001960E942177CE0101960E949109CE016A
:1094C00001960E94567610E065EC71E1CE01099696
:1094D0000E94C176BE01675F7F4F8BEC93E10E94D3
:1094E000C078811116C069EC71E1CE0101960E942D
:1094F000C176BE016F5F7F4F8BEC93E10E94C07815
:1095000001E0811101C000E0CE0101960E94567673
:1095100001C001E0CE0109960E945676002309F4AD
:10952000B1C08091CF139091D0130497F8F044E02C
:1095300050E06BEC73E1CE0101960E94F903BE018D
:109540006F5F7F4F83EB93E10E942977CE010196F5
:109550000E94567683EB93E10E94AE7960932202DB
:10956000709323028093240290932502809122021B
:1095700090912302A0912402B09125028093F312CE
:109580009093F412A093F512B093F6126DEC71E182
:1095900087E996E10E9420734091220250912302B4
:1095A000609124027091250222E030E087E996E183
:1095B0000E94317580916A0490916B040E94E31DB2
:1095C00060931A0270931B0280931C0290931D02F9
:1095D0006093FB127093FC128093FD129093FE1225
:1095E00065EE71E187E996E10E94207340911A02CD
:1095F00050911B0260911C0270911D0222E030E02C
:1096000087E996E10E94327510923E1310923D1345
:1096100080E090E00E942F0440911A0250911B02BA
:1096200060911C0270911D0222E0CE0109960E94F9
:10963000C4776FEE71E1CE0101960E94C176BE0142
:10964000675F7F4FCE0101960E947378BC0189EB62
:1096500093E10E940C77CE0101960E945676CE01CE
:1096600009960E94567669EB73E1CE0101960E943D
:109670002177CE0101960E949109CE0101960E94A8
:10968000567610E067EF71E1CE0109960E94C1762F
:10969000BE01675F7F4F8BEC93E10E94C078811120
:1096A00016C06BEF71E1CE0101960E94C176BE013A
:1096B0006F5F7F4F8BEC93E10E94C07801E08111D6
:1096C00001C000E0CE0101960E94567601C001E083
:1096D000CE0109960E945676002309F4B1C080910C
:1096E000CF139091D0130497F8F044E050E06BEC66
:1096F00073E1CE0101960E94F903BE016F5F7F4FB7
:1097000083EB93E10E942977CE0101960E94567661
:1097100083EB93E10E94AE7960931E0270931F0267
:10972000809320029093210280911E0290911F024B
:10973000A0912002B09121028093F7129093F81229
:10974000A093F912B093FA126FEF71E187E996E1F5
:109750000E94207340911E0250911F0260912002CE
:109760007091210222E030E087E996E10E94317594
:1097700080916A0490916B040E94E31D609316022D
:109780007093170280931802909319026093FF124E
:1097900070930013809301139093021365EE71E1AF
:1097A00087E996E10E9420734091160250911702BA
:1097B000609118027091190222E030E087E996E189
:1097C0000E94327510923E1310923D1380E090E09B
:1097D0000E942F04409116025091170260911802C6
:1097E0007091190222E0CE0109960E94C4776FEEB3
:1097F00071E1CE0101960E94C176BE01675F7F4F85
:10980000CE0101960E947378BC0189EB93E10E941E
:109810000C77CE0101960E945676CE0109960E94E1
:10982000567669EB73E1CE0101960E942177CE0155
:1098300001960E949109CE0101960E94567637C08A
:109840001123A9F16CEC7DE0CE0101960E94C17656
:109850006BEC73E1CE0101960E947378BC0187E93D
:1098600096E10E942B73CE0101960E9456761FC08E
:1098700085E394E10E94215B182F882319F18BEB7B
:1098800094E10E94555666E972E185EC93E10E94ED
:109890003F7767E172E187E996E10E942073612FCB
:1098A00087E996E10E944B73812F0E949F370E94A7
:1098B0006E6D6093D1137093D2138093D3139093F2
:1098C000D41341C08091AA13882331F10E946E6D98
:1098D000F8EECF2EF3E0DF2EE12CF12CA70196015C
:1098E0000E94387ECA01B9010E945F7B2091391322
:1098F00030913A1340913B1350913C130E94CA7926
:1099000020910E0230910F024091100250911102ED
:109910000E94367C181614F10E946E6DC090D1130F
:10992000D090D213E090D313F090D4136C197D092A
:109930008E099F0968347E4E8105910520F08BEBDE
:1099400094E10E944F568091AA13882331F164E676
:1099500070E080E090E00E949D6D1FC00E946E6DDF
:10996000A70196010E94387ECA01B9010E945F7B5F
:109970006093391370933A1380933B1390933C1385
:109980008091A7139091A8130E94D73564E170E0ED
:1099900080E090E00E949D6DD6CFA6960FB6F89419
:1099A000DEBF0FBECDBFDF91CF911F910F91FF9012
:1099B000EF90DF90CF90BF90AF909F908F900895E1
:1099C00020E232E1FC0131832083089520E232E17C
:1099D000FC01318320830C94C8790F931F93CF939C
:1099E000DF938C01EB0188E2FB0111928A95E9F784
:1099F0004BE050E06AE272E1CE010E9454811B8686
:109A000041E050E060E070E04C875D876E877F87C3
:109A1000F801458956896789708D488B598B6A8B07
:109A20007B8B42E050E060E070E04C8B5D8B6E8B96
:109A30007F8B1CA21DA21EA21FA240E050E068E482
:109A400074E4488F598F6A8F7B8F40E050E068E460
:109A500074EC4C8F5D8F6E8F7F8F4DEC5CEC6CE403
:109A60007EE348A359A36AA37BA3DF91CF911F9103
:109A70000F91089526E332E1FC0131832083458B69
:109A8000568B678B708F0895CF93DF931F921F9231
:109A9000CDB7DEB78DEF94E12A8349836BD249813C
:109AA000642F8DEF94E11FD22A81622F8DEF94E114
:109AB0001AD28DEF94E10F900F90DF91CF91D8C221
:109AC0000F931F93CF93DF938C01EB01262F41E07F
:109AD0006EE1DADFF801D483C383C038D10509F41D
:109AE0005BC0DCF4C034D105A9F1C036D10509F45E
:109AF00042C0A09709F08AC080E090E8A9E8B4E4E9
:109B000080939B0490939C04A0939D04B0939E0427
:109B100080E090E0A5E7B4E471C0C03CD10509F451
:109B20004CC0C03ED10509F459C0C03AD10509F076
:109B30006DC080E090E0A8ECB3E480939B04909328
:109B40009C04A0939D04B0939E0480E090E0AFE756
:109B5000B3E454C080E090ECA5E5B4E480939B04AA
:109B600090939C04A0939D04B0939E0480E090E0A9
:109B7000AEE3B4E443C080E090E8A7E2B4E48093AD
:109B80009B0490939C04A0939D04B0939E0480E05A
:109B900090E0A6E1B4E432C080E090E0A1EEB3E44E
:109BA00080939B0490939C04A0939D04B0939E0487
:109BB00080E090E0A8ECB3E421C080E090E0A5EA6A
:109BC000B3E480939B0490939C04A0939D04B09372
:109BD0009E0480E090E8A3E9B3E410C080E090E048
:109BE000A6E6B3E480939B0490939C04A0939D0409
:109BF000B0939E0480E090E0ADE4B3E480939704DA
:109C000090939804A0939904B0939A04DF91CF9114
:109C10001F910F910895CF93DF93EC018DEF94E1A5
:109C2000A0D120E042E06EE1CE012EDF60E270E0E4
:109C3000CE0146DF81E0DF91CF9108956F927F9250
:109C40008F929F92AF92BF92CF92DF92EF92FF924C
:109C50000F931F93CF93DF93EC016EE18DEF94E1AF
:109C600089D1E091FD14F091FE140190F081E02D76
:109C700063E08DEF94E119958DEF94E1F9D146E021
:109C80006EE18DEF94E1F0D18DEF94E1D5D00697A0
:109C9000DCF38DEF94E1D8D0682E8DEF94E1D4D031
:109CA000782E8DEF94E1D0D0C82E8DEF94E1CCD0FA
:109CB000D82E8DEF94E1C8D0882E8DEF94E1C4D0DA
:109CC000982EB62CA12CA728B501882777FD809562
:109CD000982F0E94617B6D837E838F839887F82CF9
:109CE000E12CE928B701882777FD8095982F0E94FD
:109CF000617B69877A878B879C871C2D00E00D2903
:109D0000B801882777FD8095982F0E94617B6D8729
:109D10007E878F87988B198A1A8A1B8A1C8ADF9103
:109D2000CF911F910F91FF90EF90DF90CF90BF9058
:109D3000AF909F908F907F906F900895CF92DF9219
:109D4000EF92FF920F931F93CF93DF938C01EB0160
:109D500084E2FB0111928A95E9F7C8016FDF84E282
:109D600090E0A0E0B0E088839983AA83BB83F801E8
:109D700085899689A789B08D8C839D83AE83BF83A7
:109D800082E090E0A0E0B0E088879987AA87BB874F
:109D9000188A198A1A8A1B8AC0909B04D0909C0446
:109DA000E0909D04F0909E04A70196016581768164
:109DB000878190850E94957A20E030E048EC52E45B
:109DC0000E94F57C6C8B7D8B8E8B9F8BA7019601FF
:109DD000F80161857285838594850E94957A20E0DB
:109DE00030E048EC52E40E94F57C688F798F8A8FCE
:109DF0009B8F209197043091980440919904509141
:109E00009A04F80165857685878590890E94957A00
:109E100020E030E048EC52E40E94F57C6C8F7D8FAE
:109E20008E8F9F8F81E0DF91CF911F910F91FF90D7
:109E3000EF90DF90CF90089580912D1590E02091C4
:109E40002E15821B9109089520912E1580912D15B4
:109E5000281750F4E22FF0E0E15DFA4E808190E0A7
:109E60002F5F20932E1508958FEF9FEF0895E091B7
:109E70002E1580912D15E81730F4F0E0E15DFA4ED3
:109E8000808190E008958FEF9FEF08950895CF921D
:109E9000DF92EF92FF920F931F93CF93DF937C019A
:109EA000CB018A0120910915222389F0EB016B0176
:109EB000C40ED51ECC15DD0561F06991D701ED9179
:109EC000FC910190F081E02DC7011995F3CF642F2B
:109ED00091D1C801DF91CF911F910F91FF90EF9029
:109EE000DF90CF900895CF93DF931F92CDB7DEB769
:109EF0006983209109152223D1F020910A1520327F
:109F000040F021E030E0FC013383228380E090E0E8
:109F100014C080910B15E82FF0E0E45FFA4E9981B0
:109F200090838F5F80930B1580930A1504C061E0C6
:109F3000CE0101965FD181E090E00F90DF91CF914B
:109F40000895FC011382128248EE53E060E070E055
:109F5000448355836683778384E492E1918380838D
:109F6000089510922E1510922D1510920B15109227
:109F70000A1583C081E08093091560932C15109217
:109F80000B1510920A150895F5CF0F93062F21E0B7
:109F900040910A156CE075E180912C15D4D0109297
:109FA0000B1510920A15109209150F9108958F92B2
:109FB0009F92AF92BF92CF92DF92EF92FF920F9358
:109FC0001F93CF93DF93EC01F62ED42E4801590155
:109FD000EE2009F1CFDF1E2D143008F013E01150F0
:109FE000B8F0E881F98128E0129FB0011124A501A1
:109FF000940104C056954795379527956A95D2F7F1
:10A00000CA01B9010190F081E02DCE011995E7CF89
:10A0100060E0CE01BADF4D2D413208F040E22C2D38
:10A020006FE275E18F2D47D010922E1580932D157C
:10A03000DF91CF911F910F91FF90EF90DF90CF9024
:10A04000BF90AF909F908F900895CF92EF920F9313
:10A050001F93C22EE12C00E010E09801A8DF1F91B1
:10A060000F91EF90CF90089521E0EFCF21E0EDCF59
:10A0700061E08BCF8DEF94E164CF1092BC1581E04D
:10A080008093BA151092B91561E084E10E94E56EE3
:10A0900061E085E10E94E56EE9EBF0E080818E7F72
:10A0A000808380818D7F808388E48093B80085E4FD
:10A0B0008093BC000895413208F043C09091BC15D4
:10A0C0009111FCCF91E09093BC152093BA152FEF1E
:10A0D00020934F1510929415240F2093931590936D
:10A0E000BB159091BB15880F892B8093BB15809170
:10A0F000B915813061F41092B9158091BB15809328
:10A10000BB008091BC0083FDF8CF85EC01C085EEDB
:10A110008093BC008091BC158130E1F3809194154F
:10A12000841710F44091941525E935E1FB01D9011C
:10A130008A2F821B841718F48D918193F9CF842F75
:10A14000089580E008950F93413208F04AC090913D
:10A15000BC159111FCCF92E09093BC150093BA15F9
:10A160009FEF90934F151092941540939315FB0118
:10A1700065E975E1DB019A2F961B941718F491910C
:10A180009D93F9CF1092BB159091BB15880F892B29
:10A190008093BB158091B915813061F41092B91587
:10A1A0008091BB158093BB008091BC0083FDF8CFEC
:10A1B00085EC01C085EE8093BC00222321F08091C4
:10A1C000BC158230E1F380914F158F3F61F0809193
:10A1D0004F15803251F080914F15803341F483E068
:10A1E00007C081E005C080E003C082E001C084E0D8
:10A1F0000F910895613298F42091BC15243089F4B0
:10A2000060937115FC0183E795E1DC012A2F281B7F
:10A21000261718F421912D93F9CF80E0089581E05D
:10A22000089582E0089585ED8093BC008091BC0084
:10A2300084FDFCCF1092BC15089585EC8093BC0082
:10A240001092BC1508951F920F920FB60F92112411
:10A250000BB60F922F933F934F935F936F937F9320
:10A260008F939F93AF93BF93EF93FF938091B90028
:10A27000887F803609F49DC070F5883209F45CC08F
:10A2800090F4803109F455C038F4882309F4F3C000
:10A29000883009F44EC0F2C0883109F44DC08032D4
:10A2A00009F45EC0EBC0803409F469C050F4803317
:10A2B00009F456C0883309F0E1C080934F15BDDF23
:10A2C000DDC0803509F44FC0883509F45DC088349D
:10A2D00009F0D4C0D2C0883909F4C3C0A8F48837C3
:10A2E00009F467C038F4883609F463C0803709F48C
:10A2F00060C0C4C0883809F4B4C0803909F45FC0B4
:10A30000803809F0BBC05BC0803B09F482C038F4E0
:10A31000803A09F466C0883A09F47BC0AFC0803C3B
:10A3200009F4A3C0883C09F4A0C0883B09F486C0A6
:10A33000A5C08091BB1510C0909194158091931584
:10A34000981770F5E091941581E08E0F8093941525
:10A35000F0E0EB56FA4E80818093BB0085EC82C022
:10A3600080934F158AC0E091941581E08E0F809301
:10A3700094158091BB00F0E0EB56FA4E80839091EB
:10A380009415809193156AC0E091941581E08E0F29
:10A39000809394158091BB00F0E0EB56FA4E8083D9
:10A3A0008091BA15811169C081E08093B91584EA62
:10A3B0005DC083E08093BC1510925015CFCF809183
:10A3C0005015803208F04DC0E091501581E08E0F9D
:10A3D000809350158091BB00F0E0EF5AFA4E8083D5
:10A3E000BDCF2BDF80915015803230F4E0915015B5
:10A3F000F0E0EF5AFA4E10826091501570E0E09153
:10A40000B515F091B61581E595E1199510925015A5
:10A4100035C084E08093BC151092721510927115AE
:10A42000E091B715F091B8151995809171158111CA
:10A4300005C081E08093711510927315E09172153B
:10A4400081E08E0F80937215F0E0ED58FA4E808116
:10A450008093BB009091721580917115981708F444
:10A460007DCF85E88093BC0009C085EC8093BC005B
:10A470001092BC1503C010924F15D5DEFF91EF91DD
:10A48000BF91AF919F918F917F916F915F914F910C
:10A490003F912F910F900BBE0F900FBE0F901F900A
:10A4A00018950895CF92DF92EF92FF92FC01858973
:10A4B0009689481B590B61097109A389B4899A01CE
:10A4C000AB010E947C7E6B017C018FE0F594E794E8
:10A4D000D794C7948A95D1F765857685882777FDC7
:10A4E0008095982F2BE0660F771F881F991F2A955C
:10A4F000D1F727853089442737FD4095542F2C0DFF
:10A500003D1D4E1D5F1D0E945A7E2C0D3D1D4E1D92
:10A510005F1DCA01B901FF90EF90DF90CF900895C1
:10A520001F93CF93DF931F92CDB7DEB7162F67E748
:10A5300070E08DEF94E1498327DD612F8DEF94E189
:10A54000D2DC4981642F8DEF94E1CDDC8DEF94E175
:10A550000F90DF91CF911F918BCDCF93C62F67E7DF
:10A5600070E08DEF94E110DD6C2F8DEF94E1BBDC9A
:10A570008DEF94E17DDD67E770E08DEF94E104DD20
:10A5800041E050E067E770E08DEF94E16FDD8DEF23
:10A5900094E15ADCC82F8DEF94E16ADD8C2FCF91C6
:10A5A0000895CF93DF93C62F67E770E08DEF94E1B6
:10A5B000EBDC6C2F8DEF94E196DC8DEF94E158DDB0
:10A5C00067E770E08DEF94E1DFDC42E050E067E7A1
:10A5D00070E08DEF94E14ADD8DEF94E135DCD82F0A
:10A5E00080E0C82F8DEF94E12FDCC82BD92B8DEFA5
:10A5F00094E13EDDCE01DF91CF910895CF93DF93BB
:10A60000EC01643008F063E068838DEF94E1A9DC2D
:10A6100060EDCE01A2DF853509F039C06AEACE01CE
:10A62000C0DF9A8389836CEACE01BBDF9C838B8376
:10A630006EEACE01B6DF9E838D8360EBCE01B1DF83
:10A640009A8B898B62EBCE01ACDF9C8B8B8B64EB9E
:10A65000CE01A7DF9E8B8D8B66EBCE01A2DF9887A4
:10A660008F8368EBCE019DDF9A8789876AEBCE01E5
:10A6700098DF9C878B876CEBCE0193DF9E878D875D
:10A680006EEBCE018EDF988B8F8781E001C080E07A
:10A69000DF91CF910895CF93DF93EC014EE264EF09
:10A6A0003FDF65E070E080E090E00E949D6D66EF26
:10A6B000CE01DF91CF9175CFCF93DF93EC01EBDF2C
:10A6C000AC0160E070E0CE01EDDE685F7F4F8F4F40
:10A6D0009F4F34E095958795779567953A95D1F793
:10A6E0000E94617B20E030E040E251E40E94957AD4
:10A6F000DF91CF910895CF92DF92EF92FF92CF93A7
:10A70000DF93EC0148814295440F440F407C4C5C40
:10A7100064EF06DF8881811105C065E070E080E0AC
:10A7200090E012C0813029F468E070E080E090E0B1
:10A730000BC0823029F46EE070E080E090E004C04D
:10A740006AE170E080E090E00E949D6D66EFCE01CE
:10A7500028DF6C01E12CF12CFE2CED2CDC2CCC2420
:10A7600068EFCE01FADEA7019601282BCA01B901D4
:10A77000488128E030E0241B310904C09695879574
:10A78000779567952A95D2F7DF91CF91FF90EF905B
:10A79000DF90CF9008952F923F924F925F926F92E9
:10A7A0007F928F929F92AF92BF92CF92DF92EF9261
:10A7B000FF920F931F93CF93DF93CDB7DEB72A9706
:10A7C0000FB6F894DEBF0FBECDBF9A87898763DFCF
:10A7D0008C0189859A858FDF6D837E838F8398872F
:10A7E000A80160E070E089859A855CDE4B015C0120
:10A7F00080EA881A8FE0980AA108B108A50194019F
:10A80000C501B4010E94027E2B013C010CE075944D
:10A810006794579447940A95D1F7A985BA851196FC
:10A820002D903C9012971C9115960D90BC91A02DE7
:10A830000E94867E6B017C018DE0F594E794D794AD
:10A84000C7948A95D1F7E985FA85A781B085A301D8
:10A8500092010E94867EBB2797FDB095AB2FC80E54
:10A86000D91EEA1EFB1EF2E0CF0ED11CE11CF11C2A
:10A8700032E0F594E794D794C7943A95D1F780E8FD
:10A88000D80EE11CF11CE985FA85A189B289A701DE
:10A8900096010E947C7EDC01CB014FE0B695A79526
:10A8A000979587954A95D1F789839A83AB83BC8323
:10A8B0006101EE24D7FCE094FE2C52E0CC0CDD1CB0
:10A8C000EE1CFF1C5A95D1F7A185B285A301920118
:10A8D0000E94867E2B013C016BE07594679457942F
:10A8E00047946A95D1F7A381B481A50194010E9490
:10A8F000867EEBE09595879577956795EA95D1F7F4
:10A90000460E571E681E791EC40CD51CE61CF71C8B
:10A91000012E04C0CC0CDD1CEE1CFF1C0A94D2F7E7
:10A9200092E0C90ED11CE11CF11CC701B60124E064
:10A9300030E040E050E00E945A7E8D819E81AF81E0
:10A94000B885821B930BA40BB50B9C01AD0160E590
:10A9500073EC80E090E004C09695879577956795B5
:10A960001A95D2F70E94027E97FD0DC0660F771FE1
:10A97000881F991F29813A814B815C810E94387E12
:10A9800049015A010CC029813A814B815C810E94A6
:10A99000387E49015A01880C991CAA1CBB1C9927B6
:10A9A000B7FC9A958B2D7A2D692D9B01AC010E94E5
:10A9B000027E9B01AC01AEEDBBE00E947C7E6C018F
:10A9C000FF24D7FCF094EF2CA3E4B3EEA50194018F
:10A9D0000E94887EBB2797FDB095AB2FC80ED91E6D
:10A9E000EA1EFB1E9FECC90E9EE0D91EE11CF11C65
:10A9F000A4E0F594E794D794C794AA95D1F7C80C2E
:10AA0000D91CEA1CFB1CC701B6012A960FB6F894A4
:10AA1000DEBF0FBECDBFDF91CF911F910F91FF9091
:10AA2000EF90DF90CF90BF90AF909F908F907F90EE
:10AA30006F905F904F903F902F9008958F929F92CC
:10AA4000AF92BF92CF92DF92EF92FF92CF93DF93BC
:10AA500000D01F92CDB7DEB74A015B019CDE6B01CF
:10AA60007C0120E03AE24DE257E4C501B4010E94C6
:10AA7000957A9B01AC0160E070E080E89FE30E9462
:10AA8000CA7926EF38E248EA50E40E94587D9B01DB
:10AA9000AC01C701B60129833A834B835C830E94D2
:10AAA000617B29813A814B815C810E94957A0E9469
:10AAB0002E7B0F900F900F900F90DF91CF91FF9012
:10AAC000EF90DF90CF90BF90AF909F908F900895C0
:10AAD000CF93DF9300D01F92CDB7DEB79A01AB01C1
:10AAE00029833A834B835C8356DE0E94617B2981F4
:10AAF0003A814B815C810E94957A21E03EED42E4EF
:10AB00005EE30E94587D9B01AC0160E070E080E84C
:10AB10009FE30E94CA7920E03AE24DE257E40E94A6
:10AB2000F57C0F900F900F900F90DF91CF910895CB
:10AB3000FC0112828FEF8183108213820895FC0141
:10AB40008381882331F0611103C08FEF81830895E1
:10AB5000118208958DEF94E10DDA8DEF94E188DA9A
:10AB600091E0811190E0892F0895CF93DF93EC015C
:10AB70006A838DEF94E1F5D96A81CE01EBDF8B8397
:10AB8000882321F08DEF94E15FD988838B8190E059
:10AB9000DF91CF910895CF93DF93EC018B818823D0
:10ABA00091F089818095862388836A818DEF94E175
:10ABB000E1D968818DEF94E196D98DEF94E158DA6F
:10ABC000282F30E002C020E030E081E090E0232B2D
:10ABD00011F080E090E0DF91CF91089508950895FD
:10ABE000DC01ED91FC910284F385E02D41E01995A3
:10ABF00081E090E00895FC011382128224E532E1A5
:10AC0000318320830895DC01ED91FC910084F1856E
:10AC1000E02D6FEF1994DC01ED91FC910284F38536
:10AC2000E02D40E0199461E0F6DF80ED97E00C94B0
:10AC3000C36DCF93DF93CDB7DEB728970FB6F894E7
:10AC4000DEBF0FBECDBF1D8220E42E8334E13F83E3
:10AC500034E5388719822A8320E12B8320E52C8371
:10AC6000FC012781421710F04FEF420FFC013085A5
:10AC700050E0FE01E40FF51F303121F4243011F4CF
:10AC8000218101C02581260F2068622F28960FB6EA
:10AC9000F894DEBF0FBECDBFDF91CF91BCCFFC01DA
:10ACA00065816B7F65836860B6CFFC016581262F67
:10ACB000246025836C60AFCFCF93DF93EC014230EB
:10ACC00018F08C8188608C834F836887222329F059
:10ACD000413019F48C8184608C8364E670E080E0FC
:10ACE00090E00E949D6D6C8164FD31C0E881F98126
:10ACF0000284F385E02D42E063E0CE01199584E9FA
:10AD000091E10E94C36DE881F9810284F385E02D11
:10AD100042E063E0CE01199586E990E00E94C36DA0
:10AD2000E881F9810284F385E02D42E063E0CE0101
:10AD3000199586E990E00E94C36DE881F98102844B
:10AD4000F385E02D42E062E0CE01199513C0606208
:10AD5000CE0161DF84E991E10E94C36D6C81606284
:10AD6000CE0159DF86E990E00E94C36D6C8160627C
:10AD7000CE0151DF86E990E00E94C36D6C81606274
:10AD8000CE0149DF8CE390E00E94C36D84E08D83A7
:10AD9000CE018BDFCE0147DF82E08E8366E0CE01FD
:10ADA0003ADFCE01DF91CF912ECFCF92DF92FF928B
:10ADB0000F931F93CF93DF931F921F92CDB7DEB7F0
:10ADC0008C01677088E0689FB00111246064C8013D
:10ADD00049835A8320DF8EE190E00E94C36D498150
:10ADE000C42E5A81D52EF12CD6016D916D01D8015A
:10ADF000ED91FC910190F081E02DC801199588E258
:10AE000090E00E94C36DF394B8E0FB12EDCF0F9079
:10AE10000F90DF91CF911F910F91FF90DF90CF9016
:10AE2000089521E001C0220F6A95EAF7DC011C9623
:10AE30002C931C971A965C934E931997ED91FC9165
:10AE40000084F185E02D60E01994FC012485222323
:10AE500091F081859285009719F4611105C006C0B3
:10AE6000019721F4611102C0258701C0158665850F
:10AE7000CF010E9690CE08950F931F93CF93DF933B
:10AE8000EC018C01025F1F4F6B85C8016EDE0197DC
:10AE900051F461E0C80153DE1C8260E0C8017BDE32
:10AEA00081E090E002C080E090E0DF91CF911F91BF
:10AEB0000F9108958F92AF92CF92EF920F93CF930D
:10AEC000DF93CDB7DEB7FC01638714861586128643
:10AED000118681E0982F01C0990F4A95EAF7928B6D
:10AEE000982F01C0990F2A95EAF7938B982F01C0EC
:10AEF000990F0A95EAF7948B982F01C0990FEA945D
:10AF0000EAF7958B982F01C0990FCA94EAF7968BB0
:10AF1000982F01C0990FAA94EAF7978B01C0880F68
:10AF20008A94EAF7808FDF91CF910F91EF90CF90C5
:10AF3000AF908F9008954F925F926F927F928F9211
:10AF4000AF92CF92EF920F931F93CF93DF9300D0E6
:10AF5000CDB7DEB73C011B894C885D882B834A83C3
:10AF6000698349DE84E692E1F30191838083C30122
:10AF70000E96DEDD2B814A816981C3019BDFA20130
:10AF8000612FC3010F900F900F90DF91CF911F9110
:10AF90000F91EF90CF90AF908F907F906F905F90D8
:10AFA0004F903FCFFF920F931F93CF93DF93EC010E
:10AFB000F62E8C01025F1F4F6A896F29C801EBDDF5
:10AFC0006A8960956F21C801DF91CF911F910F9120
:10AFD000FF90E1CD20E030E050E060FF05C0FC01D3
:10AFE000E20FF31F7589572B66952F5F3F4F243073
:10AFF000310599F7413011F4FC014489FC01658564
:10B00000652B642BCFCF0F931F93CF93DF93EC016E
:10B01000142F062F0F70423011F440E009C070E089
:10B0200084E0759567958A95E1F7CE01D3DF412FCE
:10B03000602FCE01DF91CF911F910F91CBCF0F9356
:10B040001F93CF93DF9300D0CDB7DEB78C012B8356
:10B050004A83698311DF2B814A816981C8010F907E
:10B060000F900F90DF91CF911F910F9125CEFC0192
:10B0700010821482138215820895862F642F0C94F7
:10B08000AC6E862F642F0C94E56E862F0C941A6F8D
:10B090004F925F926F927F928F929F92AF92BF92E8
:10B0A000CF92DF92EF920F93CF93DF93EC014B019E
:10B0B0003A0159010296DBDF84E792E199838883A4
:10B0C0006E018CE1C80ED11C26018CE3480E511C88
:10B0D000C601CDDF86E0C80ED11CC414D504C1F76B
:10B0E000FE01EE59FF4F718260823296B182A082DA
:10B0F000329600833196E08237979182808238962B
:10B100008AE090E091838083329684EF91E091838E
:10B11000808333961182108271971082118212827D
:10B120001382C459DF4F1882DF91CF910F91EF90B6
:10B13000DF90CF90BF90AF909F908F907F906F9057
:10B140005F904F9008952F923F924F925F926F922F
:10B150007F928F929F92AF92BF92CF92DF92EF92A7
:10B16000FF920F931F93CF93DF93CDB7DEB728974E
:10B170000FB6F894DEBF0FBECDBF98878F83F12C3A
:10B180004C0186E6880E911C0F8118850E591F4FC1
:10B19000D4018C91F816A0F4AF81B8858D919C9163
:10B1A000F801A081B181AF0DB11DFC012081318179
:10B1B00042E06C918F819885F9011995F394E8CF5D
:10B1C000512CEF81F885E959FF4FFA83E9830F810C
:10B1D00018850C591F4FC12CD12C7601C3948F8137
:10B1E00098858E599F4F9C838B83A981BA818C91BE
:10B1F000581608F088C0A52CB12CAF81B8858D9168
:10B200009C91F801A081B181AA0DBB1DFC01208198
:10B21000318141E06C918F819885F9011995AF8159
:10B22000B8858D919C91F801A081B181AA0DBB1DBB
:10B23000FC012281338140E06C918F819885F90176
:10B240001995D701C601052C04C0880F991FAA1FA4
:10B25000BB1F0A94D2F79C011C0120943094412C0E
:10B26000D4018C91EF81F88540815181481648F5D1
:10B27000642C712CEB81FC81A081B181A60DB71DDE
:10B28000FA01448155816C918F8198852D833E838D
:10B29000FA011995660C771C2D813E81EF81F885A6
:10B2A000E60DF71D892B29F480859185822B932B40
:10B2B00004C0808591858221932191878087439462
:10B2C000CFCFF801A081B181AA0DBB1DFA01228167
:10B2D000338141E06C918F819885F9011995AF8197
:10B2E000B8858D919C91F801A081B181AA0DBB1DFB
:10B2F000FC012081318140E06C918F819885F901BA
:10B300001995539472CF28960FB6F894DEBF0FBEEE
:10B31000CDBFDF91CF911F910F91FF90EF90DF9004
:10B32000CF90BF90AF909F908F907F906F905F90E5
:10B330004F903F902F900895FC0180E090E0258D84
:10B34000368D2617370739F0019636968A309105E3
:10B35000B1F78FEF9FEF0895DC0126E0629FA00D0B
:10B36000B11D112490965C934E935F9721E09196C6
:10B370002C939197FC01E459FF4F20813196019065
:10B38000F081E02D222331F0309749F0611107C0A0
:10B39000DC0102C0309719F05C968C9119940895E5
:10B3A000CF92DF92FF920F931F93CF93DF931F9261
:10B3B000CDB7DEB76C01F62EFC0186E0689FE00D8C
:10B3C000F11D112411A2878D90A181309105E9F022
:10B3D0001CF4892B51F044C08230910591F1039700
:10B3E00009F03EC040E050E030C04423C9F141E0E4
:10B3F00050E0C601B1DF0E946E6DF601E85AFF4FC2
:10B4000060837183828393832BC049830E946E6D16
:10B41000F601E85AFF4F0081118122813381601BC0
:10B42000710B820B930B72960081118120E030E04A
:10B430004981061717072807390718F442E050E03A
:10B4400004C041110DC043E050E06F2DC6010F90C4
:10B45000DF91CF911F910F91FF90DF90CF907CCF24
:10B460000F90DF91CF911F910F91FF90DF90CF90C0
:10B4700008952F923F924F925F926F927F928F9298
:10B480009F92AF92BF92CF92DF92EF92FF920F9373
:10B490001F93CF93DF931F92CDB7DEB71C01FC0142
:10B4A0004AE08FEF9FEF278D30A1232B21F4148EDC
:10B4B000968F858F11A2415036964111F4CF712C91
:10B4C000610126E6C20ED11C510187E6A80EB11C0F
:10B4D0004101A0E68A0E911C46E0442ED6018C91D3
:10B4E000781608F053C0612C8101070D111D070D5E
:10B4F000111D085F1F4FF501E0806E1408F044C075
:10B50000F80140815181062C02C0569547950A9456
:10B51000E2F741707E9C70011124E60CF11CD4010D
:10B52000ED91FC91EE0DFF1D5080B701C1014983E3
:10B5300003DF498197FD02C0682F1BC0019611F5FA
:10B54000442301F180E090E060E070E0F101E80F59
:10B55000F91F248D211110C0469EF001479EF00D69
:10B560001124E20DF31D548EF68EE58E10A2178E77
:10B5700041E0C10115DF06C06F5F7F4F06966A305C
:10B58000710521F76394B7CF7394A8CF20E030E022
:10B5900080E0F101E20FF31F91A1911181E02A5F98
:10B5A0003F4F2C333105A9F70F90DF91CF911F91B9
:10B5B0000F91FF90EF90DF90CF90BF90AF909F9052
:10B5C0008F907F906F905F904F903F902F90089555
:10B5D000CF92DF92EF92FF920F931F93CF93DF935F
:10B5E0008C010E946E6DE801C45ADF4FC880D9807B
:10B5F000EA80FB806C197D098E099F09F801E859E2
:10B60000FF4FC080D180E12CF12CC616D706E8068A
:10B61000F90660F4C80197DDC8012BDF182F0E94DE
:10B620006E6D688379838A839B8301C010E0812FCC
:10B63000DF91CF911F910F91FF90EF90DF90CF900E
:10B6400008950F931F93CF93DF93EC018C0104595E
:10B650001F4F81E0F8018083CE01BADF882349F0D3
:10B6600089A1882331F08F8D98A1019711F48C8DD9
:10B6700003C0F801108280E0DF91CF911F910F91FC
:10B680000895FC0181E08083118243EC5BEA66E768
:10B690007BE3428353836483758348ED5BE666E70F
:10B6A0007BE3468357836087718742EF54EE64E6FD
:10B6B0007BE342875387648775870895FC01DB012C
:10B6C0004D915D916D917C91139742835383648377
:10B6D000758314964D915D916D917C91179746837A
:10B6E00057836087718718964D915D916D917C911C
:10B6F0001B9742875387648775870895CF93DF939D
:10B70000FC01EB0142815381648175814883598337
:10B710006A837B8346815781608571854C835D8315
:10B720006E837F8382859385A485B5858887998775
:10B73000AA87BB87DF91CF9108950F931F93CF9373
:10B74000DF93082F6EE07DE087E996E10E94207389
:10B75000C7E0D0E010E0B8010C2E02C075956795E7
:10B760000A94E2F76170772742E050E087E996E1BA
:10B770000E94FA73219778F7DF91CF911F910F9173
:10B7800008951F93CF93DF931F92CDB7DEB7162F87
:10B7900063E570E08DEF94E149830E94C44F612F0F
:10B7A0008DEF94E10E94734F4981642F8DEF94E1F6
:10B7B0000E94734F8DEF94E10F90DF91CF911F9115
:10B7C0000C943850CF93DF93EC018DEF94E10E94FD
:10B7D000B14F40E06DE2CE01D4DF40E16DE2CE0139
:10B7E000D0DF48E06DE2CE01DF91CF91CACF6F3F4D
:10B7F000710534F4AB0177FF05C040E050E002C0B2
:10B800004FEF50E06DE1BDCFEF92FF921F93CF93CA
:10B81000DF931F92CDB7DEB77C01142F462F6EE168
:10B820002983AFDF412F6FE1C701ABDF2981422FB1
:10B8300060E2C7010F90DF91CF911F91FF90EF90D1
:10B84000A0CF6F3F710534F4AB0177FF05C040E036
:10B8500050E002C04FEF50E061E293CF462F62E22A
:10B8600090CF6F3F710534F4AB0177FF05C040E026
:10B8700050E002C04FEF50E063E283CF6F3F7105AD
:10B8800034F4AB0177FF05C040E050E002C04FEF59
:10B8900050E064E276CF6F3F710534F4AB0177FF7F
:10B8A00005C040E050E002C04FEF50E065E269CFD4
:10B8B0006F3F710534F4AB0177FF05C040E050E005
:10B8C00002C04FEF50E066E25CCF6F3F710534F489
:10B8D000AB0177FF05C040E050E002C04FEF50E001
:10B8E00068E24FCF6F3F710534F4AB0177FF05C0BD
:10B8F00040E050E002C04FEF50E069E242CFAF922B
:10B90000BF92CF92DF92EF92FF920F931F93CF934C
:10B91000DF938C01C62F7A01690163E570E08DEF3A
:10B9200094E10E94C44F6C2F8DEF94E10E94734FFD
:10B930008DEF94E10E94385063E570E08DEF94E163
:10B940000E94C44FA70163E570E08DEF94E10E946F
:10B950003650E6015E01AC18BD088DEF94E10E94FF
:10B960001C4F892B31F08DEF94E10E94244F899375
:10B97000F1CFAE14BF0421F0F801108281E0818381
:10B980008DEF94E1DF91CF911F910F91FF90EF9098
:10B99000DF90CF90BF90AF900C943850CF92DF9251
:10B9A000EF92FF920F931F93CF93DF93EC016B0104
:10B9B0007A0189019C01225F3F4F46E050E062E33B
:10B9C0009EDF8F8590E0982F88272E85822BF601A9
:10B9D00091838083898990E0982F88272889822BFA
:10B9E000F701918380838B8990E0982F88272A899B
:10B9F000822BF80191838083DF91CF911F910F916A
:10BA0000FF90EF90DF90CF9008959B012C5F3F4F08
:10BA1000AB014E5F5F4FC2CFAF92BF92CF92DF922A
:10BA2000EF92FF920F931F93CF93DF9300D000D03C
:10BA3000CDB7DEB77C015B01BE016F5F7F4FE5DFF5
:10BA4000CE0101966C01870175015E0197E0A90E98
:10BA5000B11CF601619171916F01882777FD809586
:10BA6000982F0E94617BF8012281338144815581A6
:10BA70000E94F57CF70161937193819391937F010B
:10BA80000C5F1F4FCA14DB0421F726960FB6F894FB
:10BA9000DEBF0FBECDBFDF91CF911F910F91FF9001
:10BAA000EF90DF90CF90BF90AF900895CF93DF934A
:10BAB0001F92CDB7DEB79E012F5F3F4F41E050E0B0
:10BAC0006DE11DDF898190E00F90DF91CF910895A6
:10BAD000AF92BF92CF92DF92EF92FF920F931F939C
:10BAE000CF93DF931F92CDB7DEB78C015B016A0164
:10BAF00079019E012F5F3F4F41E050E06EE1FFDE94
:10BB0000898190E0F501918380839E012F5F3F4FF3
:10BB100041E050E06FE1C801F2DE898190E0F6017A
:10BB2000918380839E012F5F3F4F41E050E060E2B0
:10BB3000C801E5DE898190E0F701918380830F9051
:10BB4000DF91CF911F910F91FF90EF90DF90CF90F9
:10BB5000BF90AF900895CF93DF931F92CDB7DEB71C
:10BB60009E012F5F3F4F41E050E061E2C8DE8981D6
:10BB700090E00F90DF91CF910895CF93DF931F92C4
:10BB8000CDB7DEB79E012F5F3F4F41E050E062E24C
:10BB9000B6DE898190E00F90DF91CF910895CF9329
:10BBA000DF931F92CDB7DEB79E012F5F3F4F41E07D
:10BBB00050E063E2A4DE898190E00F90DF91CF91A5
:10BBC0000895CF93DF931F92CDB7DEB79E012F5F0D
:10BBD0003F4F41E050E064E292DE898190E00F90B7
:10BBE000DF91CF910895CF93DF931F92CDB7DEB74A
:10BBF0009E012F5F3F4F41E050E065E280DE89818A
:10BC000090E00F90DF91CF910895CF93DF931F9233
:10BC1000CDB7DEB79E012F5F3F4F41E050E066E2B7
:10BC20006EDE898190E00F90DF91CF910895CF93E0
:10BC3000DF931F92CDB7DEB79E012F5F3F4F41E0EC
:10BC400050E068E25CDE898190E00F90DF91CF9157
:10BC50000895CF93DF931F92CDB7DEB79E012F5F7C
:10BC60003F4F41E050E069E24ADE898190E00F9069
:10BC7000DF91CF910895CF93DF931F92CDB7DEB7B9
:10BC80009E012F5F3F4F41E050E06CE238DE69815A
:10BC90006F7070E066507109882777FD8095982F46
:10BCA0000E94617B9B01AC0160E070E080E090E469
:10BCB0000E94587D20E030E048EC50E40E94F57C82
:10BCC0000F90DF91CF910895EF92FF920F931F9302
:10BCD000CF93DF931F92CDB7DEB78C01CB01BA01B2
:10BCE00020E030E048EC50E40E94957A0E942E7BE0
:10BCF000E12CF12C759567956115710521F08FEF99
:10BD0000E81AF80AF7CF8AE0E816F10484F49E01F5
:10BD10002F5F3F4F41E050E06CE2C801F0DD46E0AC
:10BD20004E0D8981807F482B6CE2C8012ADD0F907F
:10BD3000DF91CF911F910F91FF90EF900895CF93D6
:10BD4000DF931F92CDB7DEB79E012F5F3F4F41E0DB
:10BD500050E060E3D4DD89810F90DF91CF910895A9
:10BD6000DF92EF92FF920F931F93CF93DF931F9277
:10BD7000CDB7DEB78C01F62EE42ED22E9E012F5FBA
:10BD80003F4F41E050E0BBDD898121E030E00E2CE7
:10BD900001C0220F0A94EAF7DD2011F0282B02C01F
:10BDA00020952823298349816F2DC801EADC0F9053
:10BDB000DF91CF911F910F91FF90EF90DF90089549
:10BDC000262F47E050E061E3CBCF262F46E050E03E
:10BDD00067E2C6CF262F45E050E067E2C1CF262FAD
:10BDE00044E050E067E2BCCF262F42E050E067E23B
:10BDF000B7CF262F41E050E067E2B2CF262F40E0D8
:10BE000050E067E2ADCF262F47E050E067E2A8CFD1
:10BE1000262F43E050E067E2A3CF262F43E050E017
:10BE20006AE29ECF262F42E050E06AE299CF262FA9
:10BE300041E050E06AE294CF262F40E050E06AE211
:10BE40008FCF262F44E050E06CE28ACF242F462F7C
:10BE500050E06FE285CF242F462F50E06EE280CF76
:10BE60001F93CF93DF931F92CDB7DEB7142F9E01A0
:10BE70002F5F3F4F41E050E042DD898190E002C0FA
:10BE8000959587951A95E2F781700F90DF91CF9184
:10BE90001F91089547E050E061E3E2CF46E050E0B3
:10BEA00067E2DECF45E050E067E2DACF44E050E001
:10BEB00067E2D6CF42E050E067E2D2CF41E050E007
:10BEC00067E2CECF40E050E067E2CACF43E050E007
:10BED00067E2C6CF43E050E06AE2C2CF42E050E002
:10BEE0006AE2BECF41E050E06AE2BACF40E050E003
:10BEF0006AE2B6CF46E050E06BE2B2CF45E050E0F8
:10BF00006BE2AECF44E050E06BE2AACF42E050E0FB
:10BF10006BE2A6CF41E050E06BE2A2CF40E050E000
:10BF20006BE29ECF43E050E06BE29ACF44E050E0FA
:10BF30006CE296CF462F50E060E392CF462F50E060
:10BF40006FE28ECF462F50E06EE28ACFEF92FF92E3
:10BF50000F931F93CF93DF931F92CDB7DEB77C0172
:10BF60006AE772E187E996E10E9420739E012F5FE4
:10BF70003F4F41E050E060E0C701C1DC8981DDDB7B
:10BF800066E972E187E996E10E943B730DE110E0FA
:10BF900061E872E187E996E10E94207340E150E098
:10BFA000B80187E996E10E94FA736AE27BE087E9CB
:10BFB00096E10E9420739E012F5F3F4F41E050E0C9
:10BFC000602FC7019CDC8981B8DB66E972E187E9F3
:10BFD00096E10E943B730F5F1F4F0A331105C1F6B4
:10BFE0000F90DF91CF911F910F91FF90EF900895E7
:10BFF000CF92DF92EF92FF92CF93DF93EC018827ED
:10C0000077FD8095982F0E94617B6B017C0120E079
:10C0100030E040E45FE30E94F57C20E030E048E45B
:10C0200052E40E94957A0E942E7BC617D707ECF047
:10C0300020E030E040EA5FE3C701B6010E94F57CF2
:10C0400020E030E048E452E40E94957A20E030E0BD
:10C0500040E85FE30E94CB790E942E7B21E06C17C1
:10C060007D070CF420E0822F01C080E090E0DF919A
:10C07000CF91FF90EF90DF90CF900895CF92DF9215
:10C08000EF92FF92CF93DF93EC016C597F4F88279B
:10C0900077FD8095982F0E94617B6B017C0120E0E9
:10C0A00030E040E45FE30E94F57C20E030E048E4CB
:10C0B00052E40E94957A0E942E7BC617D707ECF0B7
:10C0C00020E030E040EA5FE3C701B6010E94F57C62
:10C0D00020E030E048E452E40E94957A20E030E02D
:10C0E00040E85FE30E94CB790E942E7B21E06C1731
:10C0F0007D070CF420E0822F01C080E090E0DF910A
:10C10000CF91FF90EF90DF90CF900895CF92DF9284
:10C11000EF92FF92CF93DF93EC0164567109882769
:10C1200077FD8095982F0E94617B6B017C0120E058
:10C1300030E040E45FE30E94F57C20E030E048E43A
:10C1400052E40E94957A0E942E7BC617D707ECF026
:10C1500020E030E040EA5FE3C701B6010E94F57CD1
:10C1600020E030E048E452E40E94957A20E030E09C
:10C1700040E85FE30E94CB790E942E7B21E06C17A0
:10C180007D070CF420E0822F01C080E090E0DF9179
:10C19000CF91FF90EF90DF90CF9008951F920F9274
:10C1A0000FB60F9211240BB60F922F933F934F931C
:10C1B0005F936F937F938F939F93AF93BF93EF930F
:10C1C000FF938091BE150E941A6F2091C115309186
:10C1D000C2152F5F3F4F3093C2152093C115909128
:10C1E000C015953618F096E09093BD159091BD1549
:10C1F0009430C9F128F4923069F09330D1F05EC0E8
:10C20000953009F451C0963009F058C091E09093F0
:10C210008D1651C0811152C02091C1153091C215A7
:10C220002436310508F442C010928D161092C015C4
:10C230001CC0813009F042C0E091C01591E09E0F12
:10C240009093C015F0E02091C1153091C215EE0F0A
:10C25000FF1FED53FA4E318320831092C2151092C6
:10C26000C11594E029C0811117C0E091C01591E07B
:10C270009E0F9093C015F0E02091C1153091C2152A
:10C28000EE0FFF1FED53FA4E318320831092C2153B
:10C290001092C11593E010C02091C1153091C215C4
:10C2A0002536310558F007C0811108C01092C2151B
:10C2B0001092C11503C095E09093BD159091BF15E4
:10C2C000992329F0811102C02F9A01C02F98FF9164
:10C2D000EF91BF91AF919F918F917F916F915F91FE
:10C2E0004F913F912F910F900BBE0F900FBE0F906B
:10C2F0001F9018956093BE151092BF150895F8947D
:10C3000082E08093B0008093B10094E69093B300F4
:10C310001092B2008093700078948093BD151092B3
:10C32000C0158091BE1560E00C94AC6E82E08093E5
:10C33000BD151092C01508958F929F92AF92BF9233
:10C34000CF92DF92EF92FF927B01BA0180E090E002
:10C350000E945F7B4B015C01B70180E090E00E948E
:10C360005F7B6B017C012DEC3CEC4CE45FE30E94B5
:10C37000F57C9B01AC01C501B4010E94917A87FD57
:10C3800017C02DEC3CEC4CE45FE3C501B4010E9406
:10C39000F57C9B01AC01C701B6010E94917A9927F7
:10C3A00087FD90958827990F881F9927019602C0CD
:10C3B00080E090E0FF90EF90DF90CF90BF90AF9043
:10C3C0009F908F9008958F929F92AF92BF92CF923D
:10C3D000DF92EF92FF920F931F93CF93DF936C0145
:10C3E000EB01EC84FD8486E0E816F1040CF443C014
:10C3F000EE0CFF1C06E010E045EC842E4DE9942E77
:10C400004CE1A42E41E8B42E8A859B85FC01E00F07
:10C41000F11F40815181F8013497E80FF91F6081C5
:10C420007181C60189DFFC01A501940163E971E016
:10C4300080E091E00E94027E4F01AA2497FCA09424
:10C44000BA2C86269726A826B9260E5F1F4F0E15F2
:10C450001F05D1F68C829D82AE82BF8280E290E081
:10C46000998788878FEF9FEF9983888361E070E0D9
:10C4700080E090E003C060E070E0CB01DF91CF91FD
:10C480001F910F91FF90EF90DF90CF90BF90AF90F2
:10C490009F908F9008950F931F93CF93DF938C01FC
:10C4A000EB0183EC95E19B878A878091C01590E032
:10C4B0009D878C8780918D1690E09F878E878091D5
:10C4C000BD15853009F051C0C8011BD3882319F070
:10C4D00081E090E04CC0BE01C801B0D78111F8CF17
:10C4E000BE01C80107D78111F3CFBE01C8017ED2BA
:10C4F0008111EECFBE01C801CCD48111E9CFBE01BC
:10C50000C80169D58111E4CFBE01C80192D3811160
:10C51000DFCFBE01C801E3D18111DACFBE01C8016E
:10C520002DD18111D5CFBE01C80145D68111D0CF03
:10C53000BE01C8010E94B96A8111CACFBE01C801FB
:10C540001BD08111C5CFBE01C801A2D08111C0CFBF
:10C55000BE01C80138DF672B682B692B09F0B8CF03
:10C5600082E08093BD151092C01580E090E0DF91CD
:10C57000CF911F910F910895AF92BF92CF92DF920A
:10C58000EF92FF920F931F93CF93DF93EB01809174
:10C59000C015883510F480E070C0EA85FB85828183
:10C5A000938160E672E26ADD892BA9F3EA85FB8557
:10C5B0008481958164E971E1A9DD892B61F3BEE194
:10C5C000CB2ED12C1DE1E12EF12C00E010E080916A
:10C5D000C01590E00497E816F906ACF5EA85FB85EE
:10C5E000C701880F991FE80FF91F8081918164EFBF
:10C5F00071E044DD892B79F25601AA0CBB1CEA8557
:10C60000FB85EA0DFB1D8081918168E572E07EDD8E
:10C61000892B21F0000F111F01600DC0EA85FB85F9
:10C62000EA0DFB1D8081918164EA76E06FDD892B44
:10C6300049F0000F111F82E0E80EF11C82E0C80EE5
:10C64000D11CC5CF760181E0E81AF108F594E79492
:10C65000F986E8868AE2E816F1040CF49CCFC8015A
:10C66000AA2797FDA095BA2F8C839D83AE83BF83A5
:10C6700089E090E09983888381E0DF91CF911F91D9
:10C680000F91FF90EF90DF90CF90BF90AF90089503
:10C69000AF92BF92CF92DF92EF92FF920F931F93D0
:10C6A000CF93DF93EB018091C015803211F080E0D1
:10C6B0005AC0EA85FB85828193816CE271E0DEDC01
:10C6C000892BA9F3EA85FB85848195816EEE72E062
:10C6D0001DDD892B61F306E010E0C12CD12C760121
:10C6E000EA85FB85E00FF11F808191816CE271E0AA
:10C6F000C5DC892BE1F2580182E0A80EB11CEA8565
:10C70000FB85EA0DFB1D8081918168E077E0FEDC0E
:10C71000892B39F0CC0CDD1CEE1CFF1C6894C0F892
:10C7200010C0EA85FB85EA0DFB1D808191816EEECC
:10C7300072E0ECDC892B09F4BACFCC0CDD1CEE1CCA
:10C74000FF1C0C5F1F4F0E33110551F68EE090E079
:10C7500099878887CC82DD82EE82FF828FE090E02D
:10C760009983888381E0DF91CF911F910F91FF9092
:10C77000EF90DF90CF90BF90AF900895AF92BF92AF
:10C78000CF92DF92EF92FF920F931F93CF93DF939D
:10C79000EB018091C015823251F5EA85FB858281DB
:10C7A000938168E572E06ADC892B09F18091C015FC
:10C7B00090E081509048880F991FEA85FB85E80F2B
:10C7C000F91F8081918168E572E058DC892B79F04E
:10C7D000198618868FEF9FEFDC018C839D83AE83D3
:10C7E000BF8386E090E09983888381E06DC0EA850D
:10C7F000FB858281938160E47FE140DC892B21F01D
:10C800008091C015813210F480E05EC0EA85FB851E
:10C810008481958160EA7FE079DC892BA9F358E077
:10C82000A52EB12C03E010E0C12CD12C7601EA85B5
:10C83000FB85C801880F991FE80FF91F808191813E
:10C8400068E572E01BDC892BF9F2EA85FB85EA0DCD
:10C85000FB1D8081918160E476E058DC892B39F002
:10C86000CC0CDD1CEE1CFF1C6894C0F810C0EA85DF
:10C87000FB85EA0DFB1D8081918166E272E046DC5A
:10C88000892B09F4C1CFCC0CDD1CEE1CFF1C0E5F04
:10C890001F4F84E0A80EB11C0332110541F6EA8552
:10C8A000FB85EA5BFF4F8081918168E572E0E6DB02
:10C8B000892B09F4A9CF80E190E099878887CC8201
:10C8C000DD82EE82FF828DCFDF91CF911F910F919C
:10C8D000FF90EF90DF90CF90BF90AF900895AF9210
:10C8E000BF92CF92DF92EF92FF920F931F93CF935D
:10C8F000DF93EB018091C015893310F480E06BC0A9
:10C90000EA85FB858281938160E47FE1B7DB892B37
:10C91000A9F3EA85FB858481958160EA7FE0F6DBF7
:10C92000892B61F338E0A32EB12C03E010E0C12C79
:10C93000D12C7601EA85FB85C801880F991FE80F85
:10C94000F91F8081918168E572E098DB892BB1F253
:10C95000EA85FB85EA0DFB1D8081918160E476E02C
:10C96000D5DB892B39F0CC0CDD1CEE1CFF1C689448
:10C97000C0F810C0EA85FB85EA0DFB1D808191811E
:10C9800066E272E0C3DB892B09F4B8CFCC0CDD1C66
:10C99000EE1CFF1C0E5F1F4F84E0A80EB11C0B3372
:10C9A000110541F6EA85FB85EA58FF4F80819181A8
:10C9B00068E572E063DB892B09F4A0CF8CE190E09D
:10C9C00099878887CC82DD82EE82FF828AE090E0C0
:10C9D0009983888381E0DF91CF911F910F91FF9020
:10C9E000EF90DF90CF90BF90AF9008956F927F92BD
:10C9F0008F929F92AF92BF92CF92DF92EF92FF926F
:10CA00000F931F93CF93DF93EB018091C015823278
:10CA100008F45DC0EA85FB85828193816EE571E053
:10CA20002DDB892B09F453C063E0A62EB12C02E064
:10CA300010E0C12CD12C760135018091C01590E019
:10CA4000A816B906CCF54801880C991CEA85FB8527
:10CA5000E80DF91D808191816EE977E00FDB892B6C
:10CA600039F0CC0CDD1CEE1CFF1C6894C0F80FC024
:10CA7000EA85FB85E80DF91D808191816EEE72E0FB
:10CA8000FDDA892B21F1CC0CDD1CEE1CFF1CC5014D
:10CA9000880F991FEA85FB85E80FF91F8081918136
:10CAA0006EE571E033DB22E0A20EB11C892B19F098
:10CAB0000E5F1F4FC1CF83010150110915950795D6
:10CAC000198708870031110524F41986188680E03B
:10CAD00009C0CC82DD82EE82FF828CE090E09983F7
:10CAE000888381E0DF91CF911F910F91FF90EF90AC
:10CAF000DF90CF90BF90AF909F908F907F906F907E
:10CB00000895AF92BF92CF92DF92EF92FF920F9370
:10CB10001F93CF93DF93EB01EA85FB85828193819D
:10CB200068E273E2ABDA892B11F480E077C0809180
:10CB3000C015843009F5EA85FB85848195816AEC0E
:10CB400078E0E4DA892BC1F0EA85FB85868197815C
:10CB500060E372E093DA892B79F0198618868FEFFB
:10CB60009FEFDC018C839D83AE83BF8383E090E0E5
:10CB70009983888381E052C08091C0158434A8F2E3
:10CB8000EA85FB858481958164E971E1BFDA892BAF
:10CB900061F206E010E0C12CD12C7601EA85FB851C
:10CBA000E00FF11F8081918160E372E067DA892BE9
:10CBB00009F4BBCF580182E0A80EB11CEA85FB85C1
:10CBC000EA0DFB1D808191816AE976E09FDA892B6D
:10CBD00039F0CC0CDD1CEE1CFF1C6894C0F810C0B2
:10CBE000EA85FB85EA0DFB1D8081918160E372E09F
:10CBF0008DDA892B09F499CFCC0CDD1CEE1CFF1CBF
:10CC00000C5F1F4F0638110549F680E290E09987C6
:10CC10008887CC82DD82EE82FF82A8CFDF91CF9120
:10CC20001F910F91FF90EF90DF90CF90BF90AF904A
:10CC300008958F929F92AF92BF92CF92DF92EF9220
:10CC4000FF920F931F93CF93DF9300D01F92CDB726
:10CC5000DEB74B01DB011A96ED91FC911B978281A7
:10CC600093816EEA7DE00ADA892B11F480E08FC0AF
:10CC7000D4011A96ED91FC911B978481958166ED04
:10CC800076E0FCD9892B91F3E6E0EE2EF12C20E042
:10CC900030E040E050E0A12CB12CC12CD12CD401CB
:10CCA0001A96ED91FC911B97EE0DFF1D80819181ED
:10CCB00066EF71E029833A834B835C83DFD9892B4C
:10CCC000A9F287010E5F1F4FD4011A96ED91FC91D6
:10CCD0001B97E00FF11F808191816CED74E016DAF3
:10CCE00029813A814B815C81892B39F0B501C601DC
:10CCF00001E00E94907E21601CC0D4011A96ED9143
:10CD0000FC911B97E00FF11F8081918160E971E038
:10CD100029833A834B835C83F9D929813A814B81FA
:10CD20005C81892B09F4A2CFB501C60101E00E9404
:10CD3000907E5B016C01B4E0EB0EF11CE6ECEE16AC
:10CD4000F10409F0ACCFD40114962C9314971596E6
:10CD50003C93159716964C93169717965C931797D6
:10CD6000B501C60100E20E94AB7E12962C93129789
:10CD700013963C93139785E090E011969C938E93C5
:10CD800080E390E019969C938E93189781E00F9022
:10CD90000F900F900F90DF91CF911F910F91FF9007
:10CDA000EF90DF90CF90BF90AF909F908F900895BD
:10CDB0008F929F92AF92BF92CF92DF92EF92FF92AB
:10CDC0000F931F93CF93DF937A016901DA01CD911D
:10CDD000DC91FB0184859585C817D9070CF047C005
:10CDE000CE01880F991F0284F385E02DE80FF91F0B
:10CDF000A080B180C170DD27F1E0CF27209719F422
:10CE000084E690E002C08CE99FEF4801880E991EED
:10CE1000B401C501EDD8892B89F4800E911EB401AF
:10CE2000C501E6D8892B69F4B401600F711FC501F3
:10CE3000DFD8892BF9F023E030E005C021E030E0B5
:10CE400002C022E030E0D6018D919C9111970196AD
:10CE50008217930744F0F60111821082D7018D9159
:10CE60009C91119701968D939C93CE0105C081E012
:10CE700090E002C08FEF9FEFDF91CF911F910F9154
:10CE8000FF90EF90DF90CF90BF90AF909F908F90EA
:10CE900008954F925F926F927F928F929F92AF927E
:10CEA000BF92CF92DF92EF92FF920F931F93CF9397
:10CEB000DF9300D01F92CDB7DEB76C017B011C82DF
:10CEC0001B8281E090E09A8389838091C0158D3028
:10CED00010F480E06BC009E713E09E012D5F3F4F27
:10CEE000AE014F5F5F4FC60163DF892B91F79E0153
:10CEF0002D5F3F4FAE014F5F5F4FB701C60158DF57
:10CF0000019739F79E012D5F3F4FAE014F5F5F4F95
:10CF1000B701C6014DDF892BE1F6412C512C3201BE
:10CF2000A12CB12C8091C01590E029813A8128175D
:10CF300039078CF509E713E09E012D5F3F4FAE01E5
:10CF40004F5F5F4FB701C60133DF4C019E012D5F7C
:10CF50003F4FAE014F5F5F4FB701C60129DF21E0B0
:10CF60008216910451F4892B09F0B3CF440C551C5F
:10CF7000661C771C689440F80AC0892809F0A9CF7C
:10CF8000019709F0A6CF440C551C661C771C8FEF47
:10CF9000A81AB80AC7CFF701B186A0864482558285
:10CFA0006682778281E090E0918380830F900F907A
:10CFB0000F900F90DF91CF911F910F91FF90EF9005
:10CFC000DF90CF90BF90AF909F908F907F906F90A9
:10CFD0005F904F9008952F923F924F925F926F9281
:10CFE0007F928F929F92AF92BF92CF92DF92EF92F9
:10CFF000FF920F931F93CF93DF9300D01F92CDB773
:10D00000DEB76C017B011C821B82DB011C968D91BB
:10D010009C911D971816190614F080E0B5C0DB012D
:10D020001A96ED91FC911B9782E090E09A83898398
:10D03000828193816AE67AE021D8892B71F3D70146
:10D040001A96ED91FC911B9789819A819C012F5F23
:10D050003F4F3A832983880F991FE80FF91F80817A
:10D06000918169E773E052D8892BB9F20CEB11E09A
:10D070009E012D5F3F4FAE014F5F5F4FB701C6016D
:10D0800097DE892B51F69E012D5F3F4FAE014F5F1A
:10D090005F4FB701C6018CDE019709F0BECF212C8E
:10D0A000312C2101A12CB12C29813A81F7018485F1
:10D0B0009585281739070CF05CC00CEB11E09E0138
:10D0C0002D5F3F4FAE014F5F5F4FB701C60170DE6E
:10D0D0003C01B3E0AB16B10489F00CEB11E09E010A
:10D0E0002D5F3F4FAE014F5F5F4FB701C60160DE5E
:10D0F0004C01E3E0AE16B104F9F40FC00CEB11E003
:10D100009E012D5F3F4FAE014F5F5F4FB701C601DC
:10D110004FDE6816790609F380CF0CEB11E09E0113
:10D120002D5F3F4FAE014F5F5F4FB701C60140DE3D
:10D130008816990609F071CF6114710459F48A9424
:10D14000892809F06ACF220C331C441C551C6894B2
:10D1500020F80BC06A94672809F05FCF892809F08E
:10D160005CCF220C331C441C551CAFEFAA1ABA0A20
:10D170009BCFB186A086248235824682578282E088
:10D1800090E09183808381E00F900F900F900F903B
:10D19000DF91CF911F910F91FF90EF90DF90CF9093
:10D1A000BF90AF909F908F907F906F905F904F90C7
:10D1B0003F902F900895AF92BF92CF92DF92EF925F
:10D1C000FF920F931F93CF93DF93EB01EA85FB85CB
:10D1D0008281938168E873E10E943E60892B11F49B
:10D1E00080E07DC08091C015843019F5EA85FB850B
:10D1F000848195816AEC78E00E948660892BC9F071
:10D20000EA85FB858681978160E372E00E943E603B
:10D21000892B79F0198618868FEF9FEFDC018C83BC
:10D220009D83AE83BF8387E090E09983888381E00C
:10D2300056C08091C015843498F2EA85FB858481BC
:10D24000958168E873E10E948660892B49F206E0C7
:10D2500010E0C12CD12C7601EA85FB85E00FF11F8F
:10D260008081918160E372E00E943E60892B09F425
:10D27000B7CF580182E0A80EB11CEA85FB85EA0D04
:10D28000FB1D8081918160E476E00E948660892B9D
:10D2900039F0CC0CDD1CEE1CFF1C6894C0F811C0EA
:10D2A000EA85FB85EA0DFB1D8081918160E372E0D8
:10D2B0000E948660892B09F493CFCC0CDD1CEE1CF8
:10D2C000FF1C0C5F1F4F0638110531F680E290E01D
:10D2D00099878887CC82DD82EE82FF82A4CFDF919E
:10D2E000CF911F910F91FF90EF90DF90CF90BF9063
:10D2F000AF9008958F929F92AF92BF92CF92DF929C
:10D30000EF92FF920F931F93CF93DF93EB018091E6
:10D31000C0158A3108F47AC0EA85FB858081918145
:10D320008032934050F4198618868FEF9FEFDC010E
:10D330008C839D83AE83BF836FC0828193816CEAAF
:10D340007DE00E943E60892B09F460C0EA85FB8580
:10D35000848195816CEA7DE00E943E60892B09F40E
:10D3600055C054E0A52EB12C03E010E0C12CD12C07
:10D3700076018091C01590E0A816B906E4F5EA851B
:10D38000FB85C801880F991FE80FF91F80819181E3
:10D3900066EB73E00E948660892B61F14501880C81
:10D3A000991CEA85FB85E80DF91D8081918160E675
:10D3B00079E00E943E60892B39F0CC0CDD1CEE1C1C
:10D3C000FF1C6894C0F810C0EA85FB85E80DF91DC4
:10D3D000808191816CEB72E00E943E60892BB1F0FC
:10D3E000CC0CDD1CEE1CFF1C0E5F1F4F82E0A80E54
:10D3F000B11CBFCF850101501109159507951987FB
:10D4000008870C30110524F41986188680E009C0BD
:10D41000CC82DD82EE82FF828BE090E0998388836C
:10D4200081E0DF91CF911F910F91FF90EF90DF90FE
:10D43000CF90BF90AF909F908F9008958F929F92C2
:10D44000AF92BF92CF92DF92EF92FF920F931F9312
:10D45000CF93DF93EB018091C0158A3108F471C03E
:10D46000EA85FB8580819181843F914060F4198633
:10D4700018868FEF9FEFDC018C839D83AE83BF8383
:10D480008BE090E066C08281938160E679E00E9443
:10D490003E60892B09F455C073E0A72EB12C02E041
:10D4A00010E0C12CD12C76018091C01590E0A81617
:10D4B000B906E4F5EA85FB85C801880F991FE80FD6
:10D4C000F91F8081918168E572E00E948660892B56
:10D4D00061F14501880C991CEA85FB85E80DF91D71
:10D4E0008081918160EB74E00E943E60892B39F06D
:10D4F000CC0CDD1CEE1CFF1C6894C0F810C0EA8543
:10D50000FB85E80DF91D8081918168E572E00E943C
:10D510003E60892BB1F0CC0CDD1CEE1CFF1C0E5FB5
:10D520001F4F82E0A80EB11CBFCF85010150110929
:10D5300015950795198708870C30110524F419866D
:10D54000188680E009C0CC82DD82EE82FF8284E012
:10D5500090E09983888381E0DF91CF911F910F91B3
:10D56000FF90EF90DF90CF90BF90AF909F908F9003
:10D570000895AF92BF92CF92DF92EF92FF920F93F6
:10D580001F93CF93DF93EB018091C015863410F485
:10D5900080E086C0EA85FB85828193816EEE72E031
:10D5A0000E943E60892BA1F3EA85FB8584819581E9
:10D5B0006EEE72E00E948660892B51F3EA85FB854E
:10D5C0008681978162E27BE00E943E60892B01F3B5
:10D5D000EA85FB858085918562E27BE00E9486601A
:10D5E000892BB1F25CE0A52EB12C05E010E0C12C36
:10D5F000D12C7601EA85FB85C801880F991FE80FB9
:10D60000F91F808191816EEE72E00E943E60892B4D
:10D6100009F4BECFEA85FB85EA0DFB1D808191816F
:10D6200066E678E00E948660892B39F0CC0CDD1C20
:10D63000EE1CFF1C6894C0F811C0EA85FB85EA0D5A
:10D64000FB1D808191816EEE72E00E948660892BC5
:10D6500009F49ECFCC0CDD1CEE1CFF1C0E5F1F4F8F
:10D6600084E0A80EB11C0534110521F6EA85FB857E
:10D67000E657FF4F808191816EEE72E00E943E601E
:10D68000892B09F485CF80E290E099878887CC8246
:10D69000DD82EE82FF8288E090E09983888381E0DA
:10D6A000DF91CF911F910F91FF90EF90DF90CF907E
:10D6B000BF90AF9008953F924F925F926F927F928A
:10D6C0008F929F92AF92BF92CF92DF92EF92FF9292
:10D6D0000F931F93CF93DF9300D01F921F92CDB76C
:10D6E000DEB75C01562E19821A821B821C821D82B3
:10D6F00061E0852D31D360E0852D67D362E170E074
:10D7000080E090E01AD261E0852D5FD388E290E05E
:10D710003AD260E0852D20D301E117E2852D8AD32E
:10D72000892B31F401501109C9F78EEF9FEF69C0C1
:10D7300001E117E2852D7ED3019721F401501109F3
:10D74000C9F7F3CF08E210E0312C37E0432E8824EC
:10D750008394912C21E1E22E27E2F22E852D6AD3CB
:10D76000892B29F481E0E81AF108C1F7DECFC2D194
:10D770006B017C0191E1692E97E2792E852D5AD3B8
:10D78000019729F4E1E06E1A7108C1F7CECFB2D14A
:10D790006C197D098E099F09693271058105910512
:10D7A00078F0E1E0F0E0EC0FFD1FE30DF11D2081CA
:10D7B000C401042C01C0880F0A94EAF7282B2083A7
:10D7C000411004C0339487E0482E01C04A940150B0
:10D7D000110909F0BFCF2981822F90E0F5019183D3
:10D7E00080833B81832F90E093838283230F81E0AA
:10D7F00090E03D81321302C080E090E091958195E8
:10D8000091090F900F900F900F900F90DF91CF9193
:10D810001F910F91FF90EF90DF90CF90BF90AF904E
:10D820009F908F907F906F905F904F903F90089562
:10D83000FB016181828170E0762F6627680F711D80
:10D84000882777FD8095982F0E94617B20E030E04B
:10D8500040E85DE30E94F57C23E333E948E853E4C4
:10D860000C94CA79089521E06227FC018081ADC241
:10D87000CF93DF93EC01862F688349832A8361E08D
:10D880006BD261E08881A1D260E0898165D260E0DD
:10D890008A8162D261E0898198D261E08A8195D2E1
:10D8A00060E0CE01DF91CF91DECFFB0181819081DD
:10D8B000890F9281890F9381981304C081E094812C
:10D8C0009D3009F080E008952F923F924F925F9231
:10D8D0006F927F928F929F92AF92BF92CF92DF9280
:10D8E000EF92FF920F931F93CF93DF9300D000D05E
:10D8F000CDB7DEB78C013B014E83F0D01B012C016C
:10D9000080ED280E87E0381E411C511C61E0C801E3
:10D91000AADFFE0131966F014E01F6E08F0E911CD9
:10D92000F60185E011928A95E9F7760127E0A22EAB
:10D93000B12CF80181817ED2019731F4CFD06215EC
:10D94000730584059505A8F3F801818173D2892BAD
:10D9500031F4C4D06215730584059505A8F3F80168
:10D96000828168D2892B59F0F701208181E090E013
:10D970000A2C01C0880F0A94EAF7282B2083F1E0D3
:10D98000AF1AB108B0F69FEFE91AF90AE814F904E2
:10D9900069F6A4D0621573058405950540F060E032
:10D9A000C80161DF20E030E040EC5FE72EC08981F4
:10D9B000EE818E13B5CFB601C80177DF882309F455
:10D9C000AFCF60E0C8014FDFB601C80131DFFB0116
:10D9D000DC016A946728B9F420E030E040E151E4CA
:10D9E000BF01CD010E94F57C20E030E040EA50E428
:10D9F0000E94957A20E030E040E052E40E94CB792A
:10DA00009B01AC0102C09F01AD01B901CA0126967C
:10DA10000FB6F894DEBF0FBECDBFDF91CF911F913F
:10DA20000F91FF90EF90DF90CF90BF90AF909F90BD
:10DA30008F907F906F905F904F903F902F900895C0
:10DA400046E642CF4CE440CF1F920F920FB60F92A2
:10DA500011242F933F938F939F93AF93BF93809104
:10DA60008F1690919016A0919116B09192163091C8
:10DA70008E1623E0230F2D3720F40196A11DB11D32
:10DA800005C026E8230F0296A11DB11D20938E1616
:10DA900080938F1690939016A0939116B093921640
:10DAA0008091931690919416A0919516B091961628
:10DAB0000196A11DB11D8093931690939416A09387
:10DAC0009516B0939616BF91AF919F918F913F910C
:10DAD0002F910F900FBE0F901F9018952FB7F894AD
:10DAE00060918F1670919016809191169091921678
:10DAF0002FBF08953FB7F894809193169091941694
:10DB0000A0919516B091961626B5A89B05C02F3FFB
:10DB100019F00196A11DB11D3FBF6627782F892FEF
:10DB20009A2F620F711D811D911D42E0660F771FB4
:10DB3000881F991F4A95D1F70895CF92DF92EF92EF
:10DB4000FF92CF93DF936B017C01D4DFEB01C11413
:10DB5000D104E104F10481F00E94C979CBDF6C1B90
:10DB60007D0B683E734098F381E0C81AD108E10844
:10DB7000F108C851DC4FEBCFDF91CF91FF90EF90D0
:10DB8000DF90CF9008958230910538F0880F991F6B
:10DB9000880F991F05970197F1F70895789484B538
:10DBA000826084BD84B5816084BD85B5826085BD99
:10DBB00085B5816085BDEEE6F0E08081816080837F
:10DBC000E1E8F0E010828081826080838081816062
:10DBD0008083E0E8F0E0808181608083E1EBF0E029
:10DBE000808184608083E0EBF0E0808181608083CD
:10DBF000E1E9F0E0808182608083808181608083C0
:10DC0000E0E9F0E0808181608083E1EAF0E08081FA
:10DC100082608083808181608083E0EAF0E080819F
:10DC200081608083E1E2F1E0808182608083808195
:10DC300081608083E0E2F1E0808181608083EAE7B7
:10DC4000F0E0808184608083808182608083808135
:10DC5000816080838081806880831092C1000895F4
:10DC600080939F040895863308F0865320917B00AB
:10DC7000982F9870277F922B90937B00877020912C
:10DC80009F0490E4299F90011124822B80937C00B3
:10DC900080917A00806480937A0080917A0086FD7A
:10DCA000FCCF809178002091790090E0922B08952C
:10DCB00090E0FC013197E231F10508F04CC0EB56E1
:10DCC000FF4F0C94767E809180008F7703C0809107
:10DCD00080008F7D80938000089580918000877FF1
:10DCE000F9CF84B58F7702C084B58F7D84BD089548
:10DCF0008091B0008F7703C08091B0008F7D8093BA
:10DD0000B0000895809190008F7707C080919000B7
:10DD10008F7D03C080919000877F8093900008954D
:10DD20008091A0008F7707C08091A0008F7D03C0F5
:10DD30008091A000877F8093A000089580912001AA
:10DD40008F7707C0809120018F7D03C080912001D3
:10DD5000877F809320010895CF93DF9390E0FC01AB
:10DD6000EC5BFD4F2491FC01E657FD4F8491882325
:10DD700049F190E0880F991FFC01EC5FFC4FA591E1
:10DD8000B49186519D4FFC01C591D4919FB761110B
:10DD900008C0F8948C91209582238C9388818223EB
:10DDA0000AC0623051F4F8948C91322F309583235D
:10DDB0008C938881822B888304C0F8948C91822B69
:10DDC0008C939FBFDF91CF9108950F931F93CF93B3
:10DDD000DF931F92CDB7DEB7282F30E0F901E25074
:10DDE000FE4F8491F901EC5BFD4F1491F901E65768
:10DDF000FD4F04910023C1F0882319F0698358DF97
:10DE00006981E02FF0E0EE0FFF1FE651FD4FA59175
:10DE1000B4919FB7F8948C91611103C01095812340
:10DE200001C0812B8C939FBF0F90DF91CF911F91E9
:10DE30000F910895CF93DF93282F30E0F901E2503E
:10DE4000FE4F8491F901EC5BFD4FD491F901E65747
:10DE5000FD4FC491CC2389F081112ADFEC2FF0E033
:10DE6000EE0FFF1FE053FD4FA591B4912C912D2390
:10DE700081E090E021F480E002C080E090E0DF915A
:10DE8000CF910895FC01818D228D90E0805C9F4FA1
:10DE9000821B91098F7399270895FC01918D828DC2
:10DEA000981731F0828DE80FF11D858D90E008956F
:10DEB0008FEF9FEF0895FC01918D828D981761F08F
:10DEC000828DDF01A80FB11D5D968C91928D9F5FB1
:10DED0009F73928F90E008958FEF9FEF089582E3F4
:10DEE00091E7892B39F080E090E0892B19F0BAD1C5
:10DEF000811123C080E090E0892B41F080E090E028
:10DF0000892B21F00E94000081111AC08DED91E74C
:10DF1000892B39F080E090E0892B19F04ED28111E5
:10DF200012C088E892E7892B99F080E090E0892B75
:10DF300079F0EED281110AC008950E940000DACF74
:10DF40000E940000E3CF0E940000EBCF0C94000081
:10DF50000895FC01848DDF01A80FB11DA35ABF4FA6
:10DF60002C91848D90E001968F739927848FA689D8
:10DF7000B7892C93A089B1898C9180648C93938DFF
:10DF8000848D981306C00288F389E02D80818F7DEF
:10DF900080830895CF93DF93EC01888D8823C1F0AF
:10DFA000EA89FB89808185FD05C0A889B9898C91A2
:10DFB00086FD0EC00FB607FCF5CF808185FFF2CF3E
:10DFC000A889B9898C9185FFEDCFCE01C2DFE8CF5A
:10DFD000DF91CF910895CF92DF92FF920F931F931D
:10DFE000CF93DF931F92CDB7DEB76C0181E0D601EE
:10DFF00058968C9358975B969C915B975C968C9106
:10E000005C97981307C05096ED91FC9151978081D1
:10E0100085FD2DC0F601038D10E00F5F1F4F0F73BC
:10E020001127F02EF601848DF81210C00FB607FCF0
:10E03000F9CFD6015096ED91FC915197808185FFE3
:10E04000F1CFC601698385DF6981ECCF838DE80F4D
:10E05000F11DE35AFF4F6083D6015B960C935B97EB
:10E060005296ED91FC915397808180620CC0D6014D
:10E070005696ED91FC91579760835096ED91FC91E7
:10E08000519780818064808381E090E00F90DF91E0
:10E09000CF911F910F91FF90DF90CF900895BF9285
:10E0A000CF92DF92EF92FF92CF93DF93EC016A0160
:10E0B0007B01B22EE889F98982E08083411581EEE7
:10E0C000580761057105A1F060E079E08DE390E00B
:10E0D000A70196010E94387E21503109410951095A
:10E0E0005695479537952795211580E1380798F083
:10E0F000E889F989108260E874E88EE190E0A70170
:10E1000096010E94387E21503109410951095695E6
:10E11000479537952795EC85FD853083EE85FF85FE
:10E120002083188EEC89FD89B082EA89FB89808181
:10E1300080618083EA89FB89808188608083EA89A5
:10E14000FB89808180688083EA89FB8980818F7D5B
:10E150008083DF91CF91FF90EF90DF90CF90BF90C1
:10E160000895CF93DF93EC01E881F9810284F38570
:10E17000E02D1995EA89FB8980818F7E8083EA8969
:10E18000FB898081877F8083EA89FB8980818F7703
:10E190008083EA89FB8980818F7D80838A8D898F46
:10E1A000DF91CF9108951F920F920FB60F92112415
:10E1B0000BB60F922F938F939F93EF93FF93E09162
:10E1C000A716F091A8168081E091AD16F091AE16D9
:10E1D00082FD12C090818091B0168F5F8F73209165
:10E1E000B116821751F0E091B016F0E0E956F94E01
:10E1F000958F8093B01601C08081FF91EF919F9120
:10E200008F912F910F900BBE0F900FBE0F901F900C
:10E2100018951F920F920FB60F9211240BB60F9202
:10E220002F933F934F935F936F937F938F939F931E
:10E23000AF93BF93EF93FF9387E996E18ADEFF9157
:10E24000EF91BF91AF919F918F917F916F915F916E
:10E250004F913F912F910F900BBE0F900FBE0F90DB
:10E260001F90189587E996E10DDE21E0892B09F4CE
:10E2700020E0822F089510929A161092991688EE37
:10E2800093E0A0E0B0E080939B1690939C16A0933F
:10E290009D16B0939E1688E892E19093981680930D
:10E2A000971685EC90E09093A4168093A31684ECC7
:10E2B00090E09093A6168093A51680EC90E0909342
:10E2C000A8168093A71681EC90E09093AA168093ED
:10E2D000A91682EC90E09093AC168093AB1686EC76
:10E2E00090E09093AE168093AD161092B0161092F7
:10E2F000B1161092B2161092B31608951F920F9293
:10E300000FB60F9211240BB60F922F938F939F93FA
:10E31000EF93FF93E0914417F09145178081E091CE
:10E320004A17F0914B1782FD12C0908180914D17D2
:10E330008F5F8F7320914E17821751F0E0914D1728
:10E34000F0E0EC5CF84E958F80934D1701C0808112
:10E35000FF91EF919F918F912F910F900BBE0F9096
:10E360000FBE0F901F9018951F920F920FB60F922D
:10E3700011240BB60F922F933F934F935F936F939C
:10E380007F938F939F93AF93BF93EF93FF9384E318
:10E3900097E1DFDDFF91EF91BF91AF919F918F9159
:10E3A0007F916F915F914F913F912F910F900BBE95
:10E3B0000F900FBE0F901F90189584E397E162DDD8
:10E3C00021E0892B09F420E0822F0895109237175D
:10E3D0001092361788EE93E0A0E0B0E080933817F3
:10E3E00090933917A0933A17B0933B1788E892E1BE
:10E3F000909335178093341785ED90E090934117F3
:10E400008093401784ED90E09093431780934217D8
:10E4100080ED90E0909345178093441781ED90E054
:10E42000909347178093461782ED90E09093491799
:10E430008093481786ED90E090934B1780934A178E
:10E4400010924D1710924E1710924F1710925017AE
:10E4500008951F920F920FB60F9211240BB60F92D0
:10E460002F938F939F93EF93FF93E091E117F09198
:10E47000E2178081E091E717F091E81782FD12C062
:10E4800090818091EA178F5F8F732091EB1782172D
:10E4900051F0E091EA17F0E0EF52F84E958F80933B
:10E4A000EA1701C08081FF91EF919F918F912F9189
:10E4B0000F900BBE0F900FBE0F901F9018951F92DC
:10E4C0000F920FB60F9211240BB60F922F933F931A
:10E4D0004F935F936F937F938F939F93AF93BF936C
:10E4E000EF93FF9381ED97E134DDFF91EF91BF91C1
:10E4F000AF919F918F917F916F915F914F913F91DC
:10E500002F910F900BBE0F900FBE0F901F9018957C
:10E5100081ED97E1B7DC21E0892B09F420E0822F1F
:10E5200008951092D4171092D31788EE93E0A0E0CC
:10E53000B0E08093D5179093D617A093D717B093D8
:10E54000D81788E892E19093D2178093D11785E38A
:10E5500091E09093DE178093DD1784E391E0909330
:10E56000E0178093DF1780E391E09093E2178093A8
:10E57000E11781E391E09093E4178093E31782E33E
:10E5800091E09093E6178093E51786E391E09093EE
:10E59000E8178093E7171092EA171092EB17109282
:10E5A000EC171092ED170895CF92DF92EF92FF9241
:10E5B0000F931F93CF93DF937C016A01EB0100E07F
:10E5C00010E00C151D0571F06991D701ED91FC91DA
:10E5D0000190F081E02DC7011995892B19F00F5F8B
:10E5E0001F4FEFCFC801DF91CF911F910F91FF9087
:10E5F000EF90DF90CF9008956115710581F0DB01F8
:10E600000D900020E9F7AD0141505109461B570B11
:10E61000DC01ED91FC910280F381E02D199480E002
:10E6200090E00895DC01ED91FC91DB0114964D9191
:10E630005C9115976D917C910280F381E02D199486
:10E64000DBCFDC01ED91FC910190F081E02D19947C
:10E6500064E972E1D1CF0F931F93CF93DF93EC0165
:10E66000E1DF8C01CE01F4DF800F911FDF91CF91AC
:10E670001F910F9108950F931F93CF93DF93EC0198
:10E68000BBDF8C01CE01E4DF800F911FDF91CF91C2
:10E690001F910F9108950F931F93CF93DF93EC0178
:10E6A000D0DF8C01CE01D4DF800F911FDF91CF919D
:10E6B0001F910F9108958F929F92AF92BF92CF9228
:10E6C000DF92EF92FF920F931F93CF93DF93CDB71B
:10E6D000DEB7A1970FB6F894DEBF0FBECDBF7C01A9
:10E6E000C42EE52FCB01D22E19A221E02D1510F05A
:10E6F0002AE0D22E8E010F5D1F4F8D2C912CA12C64
:10E70000B12C6C2D7E2FA50194010E94387E8C2D9A
:10E71000D29E80191124015011098A3014F4805DB1
:10E7200001C0895CF801808321153105410551053F
:10E7300021F0C22EE32FCA01E4CFB801C7015CDF8C
:10E74000A1960FB6F894DEBF0FBECDBFDF91CF917B
:10E750001F910F91FF90EF90DF90CF90BF90AF90FF
:10E760009F908F900895CF92DF92EF92FF920F9338
:10E770001F93CF93DF93EC016A017B0121153105D3
:10E7800079F4E881F9810190F081E02D642FDF9127
:10E79000CF911F910F91FF90EF90DF90CF90199440
:10E7A0002A303105D9F477FF18C06DE24ADF8C01B9
:10E7B00044275527BA014C195D096E097F092AE0E3
:10E7C000CE0179DF800F911FDF91CF911F910F91C3
:10E7D000FF90EF90DF90CF9008952AE0B701A60157
:10E7E000CE01DF91CF911F910F91FF90EF90DF90BD
:10E7F000CF9061CF9A01AB01662757FD6095762FC8
:10E80000B2CF0F931F93CF93DF93EC019A01AB012B
:10E81000662757FD6095762FA6DF8C01CE0118DFA5
:10E82000800F911FDF91CF911F910F9108950F934A
:10E830001F93CF93DF93EC0196DF8C01CE0108DFAD
:10E84000800F911FDF91CF911F910F910895211596
:10E85000310541F4DC01ED91FC910190F081E02D56
:10E86000642F199428CF0F931F93CF93DF93EC015C
:10E870009A01462F50E060E070E0E9DF8C01CE01A4
:10E88000E7DE800F911FDF91CF911F910F910895C7
:10E890000F931F93CF93DF93EC01D9DF8C01CE014F
:10E8A000D7DE800F911FDF91CF911F910F910895B7
:10E8B0004F925F926F927F928F929F92AF92BF9290
:10E8C000CF92DF92EF92FF920F931F93CF93DF933C
:10E8D000EC016A017B01B22E9A01AB01C701B601BE
:10E8E0000E94E97D882319F067E972E125C02601BD
:10E8F0003701E89477F82FEF3FEF4FE75FE7C30169
:10E90000B2010E94E97D81110CC02FEF3FEF4FE76C
:10E910005FE7C301B20105D618161CF46BE972E17A
:10E920000BC02FEF3FEF4FE75FE4C701B6019ED763
:10E930001816A4F46FE972E1CE01DF91CF911F9117
:10E940000F91FF90EF90DF90CF90BF90AF909F908E
:10E950008F907F906F905F904F904ECE2FEF3FEF54
:10E960004FE75FECC701B601DCD587FDE3CF20E0C0
:10E9700030E0A901C701B601D4D587FF09C06DE217
:10E98000CE015FDE8C01F7FAF094F7F8F09402C044
:10E9900000E010E0A12C60E070E080E09FE3AB14A9
:10E9A00039F020E030E040E251E4BFD5A394F7CF46
:10E9B0009B01AC01C701B601EED46B017C0153D6BB
:10E9C0002B013C017CD69B01AC01C701B601E2D40E
:10E9D0006B017C012AE0B301A201CE016CDE080FBD
:10E9E000191FBB2031F06AE57CE0CE0105DE080F7F
:10E9F000191F7B2C772019F120E030E040E251E430
:10EA0000C701B601F2D76B017C0128D64B01AA24BD
:10EA100097FCA094BA2C2AE030E0B501A401CE0105
:10EA2000A2DE080F191FC501B4014BD69B01AC0132
:10EA3000C701B601AFD46B017C017A94DBCFC8016A
:10EA4000DF91CF911F910F91FF90EF90DF90CF90CA
:10EA5000BF90AF909F908F907F906F905F904F90FE
:10EA6000089526CF0F931F93CF93DF93EC0120DF00
:10EA70008C01CE01EDDD800F911FDF91CF911F91B1
:10EA80000F9108950F931F93CF93DF93EC0126D836
:10EA9000688779878A879B87E881F9810680F78173
:10EAA000E02DCE01199597FF14C018D80885198557
:10EAB0002A853B85601B710B820B930B0C811D819A
:10EAC0002E813F81601771078207930728F38FEF2C
:10EAD0009FEFDF91CF911F910F910895FC01448327
:10EAE0005583668377830895CF92DF92EF92FF92EA
:10EAF0000F931F93CF93DF937C016A01EB0100E03A
:10EB000010E00C151D0541F0C701BCDF97FD04C0E6
:10EB100089930F5F1F4FF5CFC801DF91CF911F91F0
:10EB20000F91FF90EF90DF90CF9008954F925F92FA
:10EB30006F927F928F929F92AF92BF92CF92DF920D
:10EB4000EF92FF920F931F93CF93DF934C01EB0152
:10EB500086E0849F8001859F100D1124060F171FEA
:10EB6000FB01E017F10708F582819381892B19F1E8
:10EB70003696F7CF4081518164817581DA01A60F05
:10EB8000B71F2C91332727FD30958217930709F57E
:10EB90006F5F7F4F758364832281338162177307B0
:10EBA00051F03696E017F10728F3C4016BDF97FDAB
:10EBB00046C0FE01F7CFEC1BFD0BF595E7952BEA60
:10EBC0003AEAE29FC001E39F900DF29F900D11245D
:10EBD00038C06115710529F3A480B58095012150D5
:10EBE000310935832483DA01A20FB31FAC91BB270F
:10EBF000A7FDB0958A179B07F9F421153105C9F0D7
:10EC00006A017B01E21AF30AE40EF51E412C512C35
:10EC1000D6016D906D01D7017D907D01671006C012
:10EC2000BFEF4B1A5B0A4216530690F34216530687
:10EC300099F6B582A482B5CF232B71F6B2CF8FEFB0
:10EC40009FEFDF91CF911F910F91FF90EF90DF9099
:10EC5000CF90BF90AF909F908F907F906F905F907C
:10EC60004F900895CF93DF9300D000D0CDB7DEB79B
:10EC7000FE01319626E0DF011D922A95E9F77A839D
:10EC800069835C834B8341E050E0BF014FDF21E0AB
:10EC9000892B09F020E0822F26960FB6F894DEBF6C
:10ECA0000FBECDBFDF91CF910895DCCFFC018081F5
:10ECB00091810C948E7FCF93DF93EC0188819981B1
:10ECC000009711F00E948E7F198218821D821C828B
:10ECD0001B821A82DF91CF9108950F931F93CF93D8
:10ECE000DF93EC018B016F5F7F4F888199810E94D8
:10ECF0001D80009731F0998388831B830A8381E00C
:10ED000001C080E0DF91CF911F910F910895CF93C3
:10ED1000DF93EC0188819981892B29F08A819B817D
:10ED20008617970758F4CE01D8DF882341F08C81ED
:10ED30009D81892B19F4E881F981108281E0DF91AE
:10ED4000CF910895EF92FF920F931F93CF93DF938C
:10ED5000EC017B018A01BA01DADF811103C0CE0127
:10ED6000AADF07C01D830C83B701888199810E94A7
:10ED70003F81CE01DF91CF911F910F91FF90EF90D6
:10ED80000895FC011182108213821282158214826E
:10ED90006115710551F0FB0101900020E9F7AF0109
:10EDA00041505109461B570BCDCF08950F931F9328
:10EDB000CF93DF938C01EB01FC018081918100975F
:10EDC00099F0428153812C813D814217530750F0C5
:10EDD000688179810E943F818C819D81F8019583B2
:10EDE000848313C00E948E7F88819981F80191836A
:10EDF00080838A819B81938382838C819D8195838B
:10EE00008483198218821B821A821D821C82DF91E0
:10EE1000CF911F910F910895CF93DF93EC01FB01E8
:10EE20008617970751F0608171816115710521F096
:10EE30004481558187DF01C03EDFCE01DF91CF9154
:10EE40000895FC01118210821382128215821482AD
:10EE5000E3CFCF93DF93EC018617970709F0A6DF86
:10EE6000CE01DF91CF910895CF93DF93EC01861708
:10EE7000970709F09BDFCE01DF91CF910895CF93E3
:10EE8000DF93EC016115710559F0FB010190002041
:10EE9000E9F7AF0141505109461B570B53DF01C041
:10EEA0000ADFCE01DF91CF910895CF93DF931F92B8
:10EEB0001F92CDB7DEB7FC0111821082138212823D
:10EEC0001582148269831A82BE016F5F7F4FD7DF7C
:10EED0000F900F90DF91CF9108950F931F93CF93D1
:10EEE000DF93CDB7DEB762970FB6F894DEBF0FBEE3
:10EEF000CDBF8C01CB01F8011182108213821282E6
:10EF00001582148250E0BE016F5F7F4F0E947D81A9
:10EF1000BE016F5F7F4FC801B2DF62960FB6F894F3
:10EF2000DEBF0FBECDBFDF91CF911F910F9108952E
:10EF30000F931F93CF93DF93CDB7DEB7A2970FB692
:10EF4000F894DEBF0FBECDBF8C01CB01BA01F80132
:10EF500011821082138212821582148230E0AE0177
:10EF60004F5F5F4F0E949181BE016F5F7F4FC8016D
:10EF700086DFA2960FB6F894DEBF0FBECDBFDF913D
:10EF8000CF911F910F910895EF92FF920F931F93CE
:10EF9000CF93DF93CDB7DEB7A1970FB6F894DEBF5E
:10EFA0000FBECDBF7C01CB01BA01F70111821082E7
:10EFB000138212821582148242E0420F8E010F5F8B
:10EFC0001F4FF4D6BC01C7015ADFA1960FB6F894C3
:10EFD000DEBF0FBECDBFDF91CF911F910F91FF908C
:10EFE000EF900895EF92FF920F931F93CF93DF93CB
:10EFF000CDB7DEB7A1970FB6F894DEBF0FBECDBF79
:10F000007C01CB01BA01F7011182108213821282B6
:10F010001582148242E0420F8E010F5F1F4FC6D649
:10F02000BC01C7012CDFA1960FB6F894DEBF0FBE5E
:10F03000CDBFDF91CF911F910F91FF90EF90089579
:10F04000EF92FF920F931F93CF93DF93EC017B011D
:10F050000C811D816115710511F480E015C0411509
:10F06000510589F0040F151FB80151DE8823A9F35B
:10F07000288139818C819D81B701820F931F0E9465
:10F080003F811D830C8381E0DF91CF911F910F9110
:10F09000FF90EF900895FB0144815581608171815B
:10F0A000CFCF6115710551F0FB0101900020E9F708
:10F0B000AF0141505109461B570BC2CF80E0089564
:10F0C000CF93DF931F921F92CDB7DEB769831A8269
:10F0D00041E050E0BE016F5F7F4FB2DF0F900F90B5
:10F0E000DF91CF910895CF93DF93EC01FB01448131
:10F0F000558160817181A4DF811102C0CE01DBDD09
:10F10000CE01DF91CF910895CF93DF93EC0161158C
:10F11000710561F0FB0101900020E9F7AF0141505A
:10F120005109461B570B8CDF811102C0CE01C3DD94
:10F13000CE01DF91CF910895FA01DB0114964D9134
:10F140005C911597DC0114962D913C911597241B29
:10F15000350B2E173F0788F08D919C91009769F031
:10F16000DB016D917C916115710539F08E0F9F1F48
:10F170000E94468121E0892B09F020E0822F08952A
:10F18000FC0144815581FB012481358142175307DD
:10F1900018F040E050E0D0CF80E00895FC012481D9
:10F1A00035816217730748F480819181009729F0B7
:10F1B000FC01E60FF71F8081089580E00895EECFEF
:10F1C0000F931F93CF93DF93EB0141155105E9F0A6
:10F1D0002097D9F0FC016481758126173707A0F4C8
:10F1E000621B730B8A01015011096017710708F443
:10F1F0008B01FC0160817181620F731FA801CE0138
:10F200000E945481C00FD11F1882DF91CF911F91AE
:10F210000F910895AF92BF92CF92DF92EF92FF923B
:10F220000F931F93CF93DF937B01EA01FB0144818E
:10F2300055814115510569F1FC0124813581211564
:10F24000310539F12417350720F1C217D30710F023
:10F25000E9012197FC0100811181C801AA24AA9427
:10F26000BB24BA946801CC0EDD1EC816D906A0F0E6
:10F27000F701608171810E946381009769F09C01B0
:10F28000201B310BC217D30708F4950101965901D1
:10F29000ECCF8FEF9FEF01C0C501DF91CF911F91A0
:10F2A0000F91FF90EF90DF90CF90BF90AF900895B7
:10F2B000FC0144815581FB0124813581421B530BA4
:10F2C000A9CFBF92CF92DF92EF92FF920F931F933D
:10F2D000CF93DF936C017B01EA0189012417350785
:10F2E00020F48D2FE901042F182F66E972E1C60181
:10F2F00048DDD70114968D919C911597C817D907B1
:10F30000C0F48017910708F48C01D701ED91FC91AE
:10F310001197E00FF11FB08010826D917C916C0FFE
:10F320007D1FC601ACDDD701ED91FC91E00FF11F0F
:10F33000B082C601DF91CF911F910F91FF90EF90A6
:10F34000DF90CF90BF900895FC018081918100975C
:10F3500009F05EC760E070E0CB010895FC01808198
:10F360009181009709F051C760E070E0CB010895EA
:10F3700048D708950E94CE6DFCDF0E94C42CCFE6D2
:10F38000DFE60E947B3B2097E1F30E946F6FF9CF8D
:10F39000C5C508955058BB27AA270ED02DC21ED22E
:10F3A00030F023D220F031F49F3F11F41EF4EEC16F
:10F3B0000EF4E095E7FBE4C1E92F2FD280F3BA17F2
:10F3C000620773078407950718F071F49EF547C22A
:10F3D0000EF4E0950B2EBA2FA02D0B01B901900170
:10F3E0000C01CA01A0011124FF27591B99F0593FB4
:10F3F00050F4503E68F11A16F040A22F232F342FFC
:10F400004427585FF3CF469537952795A795F04049
:10F410005395C9F77EF41F16BA0B620B730B840B5E
:10F42000BAF09150A1F0FF0FBB1F661F771F881F16
:10F43000C2F70EC0BA0F621F731F841F48F487956E
:10F4400077956795B795F7959E3F08F0B3CF93955D
:10F45000880F08F09927EE0F979587950895BED1EC
:10F4600058F080E891E009F49EEFBFD128F040E821
:10F4700051E059F45EEF09C089C1F1C1E92FE0788C
:10F48000CCD168F3092E052AC1F3261737074807A0
:10F49000590738F00E2E07F8E02569F0E025E06402
:10F4A0000AC0EF6307F8009407FADB01B9019D0178
:10F4B000DC01CA01AD01EF9347D09ED10AD05F9124
:10F4C000552331F02BED3FE049E450FD49EC63CF8B
:10F4D0000895DF93DD27B92FBF7740E85FE3161665
:10F4E000170648075B0710F4D92FC4D19F938F9359
:10F4F0007F936F936BD3EEE4F1E04BD17DD12F91ED
:10F500003F914F915F917DD2DD2349F09058A2EA5F
:10F510002AED3FE049EC5FE3D0785D274DDFDF91D6
:10F520006BC10AD108F481E008950CD065C15DD1AA
:10F5300040F054D130F021F45F3F19F021C1511156
:10F540008FC124C16AD198F39923C9F35523B1F32C
:10F55000951B550BBB27AA2762177307840738F042
:10F560009F5F5F4F220F331F441FAA1FA9F333D0A1
:10F570000E2E3AF0E0E830D091505040E695001C55
:10F58000CAF729D0FE2F27D0660F771F881FBB1F11
:10F59000261737074807AB07B0E809F0BB0B802DEB
:10F5A000BF01FF2793585F4F2AF09E3F510568F037
:10F5B000E7C056C15F3FECF3983EDCF38695779544
:10F5C0006795B795F7959F5FC9F7880F911D969539
:10F5D000879597F90895E1E0660F771F881FBB1F95
:10F5E000621773078407BA0720F0621B730B840B42
:10F5F000BA0BEE1F88F7E095089519F40EF0C0C01D
:10F600002EC1C4C012D1C8F39638C0F707F80F92C4
:10F61000E8942BE33AEA48EB5FE7F5D10F920F92BB
:10F620000F924DB75EB70F92ADD1EBE7F1E0B1D0DD
:10F630004F915F91EF91FF91E595EE1FFF1F49F00C
:10F64000FE57E0684427EE0F441FFA95E1F7419515
:10F65000550B19D10F9007FE0DC1089504D0689481
:10F66000B111FEC00895E1D088F09F5790F0B92FF6
:10F670009927B751A0F0D1F0660F771F881F991F07
:10F680001AF0BA95C9F712C0B13081F0E8D0B1E0F4
:10F690000895E5C0672F782F8827B85F39F0B93F04
:10F6A000CCF3869577956795B395D9F73EF4909509
:10F6B0008095709561957F4F8F4F9F4F0895E89487
:10F6C00009C097FB3EF490958095709561957F4FAA
:10F6D0008F4F9F4F9923A9F0F92F96E9BB27939558
:10F6E000F695879577956795B795F111F8CFFAF468
:10F6F000BB0F11F460FF1BC06F5F7F4F8F4F9F4F99
:10F7000016C0882311F096E911C0772321F09EE8F6
:10F71000872F762F05C0662371F096E8862F70E05C
:10F7200060E02AF09A95660F771F881FDAF7880F36
:10F730009695879597F90895990F0008550FAA0B8C
:10F74000E0E8FEEF16161706E807F907C0F01216F4
:10F750001306E407F50798F0621B730B840B950BF7
:10F7600039F40A2661F0232B242B252B21F408954C
:10F770000A2609F4A140A6958FEF811D811D0895E9
:10F7800097F99F6780E870E060E008959FEF80EC54
:10F790000895DF93CF931F930F93FF92EF92DF9221
:10F7A0007B018C01689405C0DA2EEF012AD1FE019D
:10F7B000E894A5912591359145915591AEF3EF01CE
:10F7C000FBDDFE019701A801DA9479F7DF90EF9055
:10F7D000FF900F911F91CF91DF91089500240A941B
:10F7E0001616170618060906089500240A9412161C
:10F7F0001306140605060895092E0394000C11F44F
:10F80000882352F0BB0F40F4BF2B11F460FF04C0FB
:10F810006F5F7F4F8F4F9F4F089557FD9058440F54
:10F82000551F59F05F3F71F04795880F97FB991F5F
:10F8300061F09F3F79F0879508951216130614061C
:10F84000551FF2CF4695F1DF08C0161617061806A9
:10F85000991FF1CF86957105610508940895E89484
:10F86000BB2766277727CB0197F9089565DF08F452
:10F870008FEF08959B01AC0160E070E080E89FE3AA
:10F8800054CE7ECFAAC1D1DFE8F39923D9F3940FE8
:10F89000511DBBF39150504094F059F0882332F041
:10F8A000660F771F881F91505040C1F79E3F51054A
:10F8B00044F7880F911D9695879597F908955F3FB6
:10F8C000ACF0983E9CF0BB27869577956795B795E9
:10F8D00008F4B1609395C1F7BB0F58F711F460FFBE
:10F8E000E8CF6F5F7F4F8F4F9F4FE3CFB9CF0AD0E5
:10F8F00029ED3BE54EED5EE378C00EF06EC146CFDC
:10F9000068943ECF92DFC8F39923D1F3C6F3DF9317
:10F91000CF931F930F93FF92C92FDD2788232AF0DF
:10F920002197660F771F881FDAF720E030E040E864
:10F930005FEB9FE3883920F0803E30F021968F778F
:10F940002ADDE3EAF1E003C026DDE0EDF1E021DFAE
:10F950008B01BE01EC01FB2E6F5771097595771F66
:10F96000880B990BAEDE28E132E741E35FE349D033
:10F97000AF2D9801AE01FF900F911F91CF91DF91B4
:10F980001BDD3ACFFA01DC01AA0FBB1F9B01AC01C2
:10F99000BF5728F422273327442750781FC0B75178
:10F9A00088F4AB2F0024469537952795011CA39525
:10F9B000D2F3002069F0220F331F441FB395DAF30E
:10F9C0000DD0E8CC61307105A0E88A07B94630F463
:10F9D0009B01AC016627772788279078309621F025
:10F9E000208331834283538308950BD005CFF6DE05
:10F9F00028F0FBDE18F0952309F0C2CEC7CE112403
:10FA00002FCF0BDFA0F3959FD1F3950F50E0551F3B
:10FA1000629FF001729FBB27F00DB11D639FAA2763
:10FA2000F00DB11DAA1F649F6627B00DA11D661FB2
:10FA3000829F2227B00DA11D621F739FB00DA11DD3
:10FA4000621F839FA00D611D221F749F3327A00D8D
:10FA5000611D231F849F600D211D822F762F6A2F29
:10FA600011249F5750408AF0E1F088234AF0EE0FAE
:10FA7000FF1FBB1F661F771F881F91505040A9F7BB
:10FA80009E3F510570F07CCEEBCE5F3FECF3983E8D
:10FA9000DCF3869577956795B795F795E7959F5F22
:10FAA000C1F7FE2B880F911D9695879597F90895BC
:10FAB000FA01EE0FFF1F30962105310599F161150E
:10FAC000710561F48038BFE39B0749F16894903871
:10FAD000810561F08038BFEF9B0741F0992342F523
:10FAE000FF3FE1053105210511F1E8940894E79500
:10FAF000D901AA2329F4AB2FBE2FF85FD0F310C091
:10FB0000FF5F70F4A695E0F7F73950F019F0FF3A6F
:10FB100038F49F779F930CD00F9007FC905808956E
:10FB20003EF034CE60E070E080E89FE308954FE758
:10FB30009F775F934F933F932F93E4DE2F913F91F5
:10FB40004F915F9152DF5ECD11F40EF41FCE45C090
:10FB50006CDED0F39923D9F3CEF39F57550B87FF73
:10FB60004AD00024A0E640EA900180585695979527
:10FB700028F4805C660F771F881F20F02617370750
:10FB8000480730F4621B730B840B202931294A2B60
:10FB9000A69517940794202531254A2758F7660F14
:10FBA000771F881F20F026173707480730F4620BAD
:10FBB000730B840B200D311D411DA09581F7B901F8
:10FBC000842F9158880F9695879508959B01AC01D5
:10FBD0000CCFB2DD880B990B08959F3F31F0915007
:10FBE00020F4879577956795B795880F911D969521
:10FBF000879597F9089591505040660F771F881F99
:10FC0000D2F70895DB018F939F9376D0BF91AF9188
:10FC1000A29F800D911DA39F900DB29F900D112466
:10FC20000895AA1BBB1B51E107C0AA1FBB1FA61743
:10FC3000B70710F0A61BB70B881F991F5A95A9F795
:10FC400080959095BC01CD01089597FB072E16F481
:10FC5000009406D077FD08D0E4DF07FC05D03EF421
:10FC6000909581959F4F0895709561957F4F089568
:10FC7000A1E21A2EAA1BBB1BFD010DC0AA1FBB1FB0
:10FC8000EE1FFF1FA217B307E407F50720F0A21B22
:10FC9000B30BE40BF50B661F771F881F991F1A948F
:10FCA00069F760957095809590959B01AC01BD01B9
:10FCB000CF010895052E97FB16F400940FD057FD41
:10FCC00005D0D6DF07FC02D046F408C05095409519
:10FCD000309521953F4F4F4F5F4F089590958095F8
:10FCE000709561957F4F8F4F9F4F0895EE0FFF1FC7
:10FCF0000590F491E02D19944AD0A59F900DB49FE2
:10FD0000900DA49F800D911D11240895B7FFF4CF8D
:10FD1000F3DF821B930B08950790F691E02D199461
:10FD20000F93083090F0982F872F762F652F542F40
:10FD3000432F322F22270850F4CF220F331F441FA6
:10FD4000551F661F771F881F991F0A95B2F70F91DD
:10FD5000089597FB10F8169400080F93083098F058
:10FD60000850232F342F452F562F672F782F892F98
:10FD7000902DF4CF0594979587957795679557952E
:10FD80004795379527950A95AAF70F910895A29F51
:10FD9000B001B39FC001A39F700D811D1124911D5F
:10FDA000B29F700D811D1124911D0895EF920F9344
:10FDB0001F93CF93DF93E80147FF02C034E101C0F6
:10FDC00034E0E42FFF27E7FDF095F7FF03C0F1953E
:10FDD000E195F109E32E022F2E2FAE011FD3CE01A4
:10FDE000DF91CF911F910F91EF900895CF93DF9303
:10FDF0008230910510F482E090E0E0917018F0916B
:10FE0000711820E030E0A0E0B0E0309739F1408197
:10FE1000518148175907B8F04817590771F4828182
:10FE20009381109729F013969C938E9312972CC070
:10FE3000909371188093701827C02115310531F007
:10FE40004217530718F0A901DB0101C0EF019A0125
:10FE5000BD01DF010280F381E02DD7CF21153105EF
:10FE6000F9F0281B390B2430310580F48A819B81FD
:10FE70006115710521F0FB019383828304C0909387
:10FE8000711880937018FE01329644C0FE01E20F93
:10FE9000F31F8193919322503109398328833AC00B
:10FEA00020916E1830916F18232B41F4209102029B
:10FEB0003091030230936F1820936E182091000246
:10FEC000309101022115310541F42DB73EB7409123
:10FED000040250910502241B350BE0916E18F0913D
:10FEE0006F18E217F307A0F42E1B3F0B28173907F2
:10FEF00078F0AC014E5F5F4F2417350748F04E0F86
:10FF00005F1F50936F1840936E188193919302C0B6
:10FF1000E0E0F0E0CF01DF91CF910895CF93DF9340
:10FF2000009709F487C0FC01329713821282C091B6
:10FF30007018D0917118209781F420813181280F99
:10FF4000391F80916E1890916F188217930779F579
:10FF5000F0936F18E0936E186DC0DE0120E030E082
:10FF6000AE17BF0750F412964D915C9113979D0107
:10FF70004115510509F1DA01F3CFB383A283408122
:10FF80005181840F951F8A179B0771F48D919C9165
:10FF90001197840F951F02969183808312968D91FD
:10FFA0009C911397938382832115310529F4F09353
:10FFB0007118E09370183EC0D9011396FC93EE932C
:10FFC00012974D915D91A40FB51FEA17FB0779F4C5
:10FFD00080819181840F951F0296D90111969C937F
:10FFE0008E938281938113969C938E931297E0E077
:10FFF000F0E08A819B81009719F0FE01EC01F9CFB6
:020000021000EC
:10000000CE01029628813981820F931F20916E18AC
:1000100030916F182817390769F4309729F4109236
:1000200071181092701802C013821282D0936F1848
:10003000C0936E18DF91CF9108956F927F928F9247
:100040009F92AF92BF92CF92DF92EF92FF920F9367
:100050001F93CF93DF93EC01CB01209779F4DF91CD
:10006000CF911F910F91FF90EF90DF90CF90BF90B5
:10007000AF909F908F907F906F90B8CEFE01E60F6B
:10008000F71F9E0122503109E217F30708F4A8C0B8
:10009000D9010D911C91119706171707B0F0053083
:1000A000110508F49BC0A801445051094617570791
:1000B00008F494C002501109061B170B0193119309
:1000C0006D937C93CF012ADF89C05B01A01AB10A2E
:1000D0004E01800E911EA0917018B0917118612C84
:1000E000712C60E070E0109709F449C0A815B905BB
:1000F000C9F5ED90FC901197670142E0C40ED11C48
:10010000CA14DB0478F147018A189B08640142E0B5
:10011000C40ED11C1296BC9012971396AC91B5E008
:10012000CB16D10440F0B282A38391828082D901A0
:100130008D939C9309C00E5F1F4F0E0D1F1DF9017B
:1001400011830083EB2DFA2F6115710531F0DB016E
:100150001396FC93EE93129741C0F0937118E093BD
:1001600070183CC06D917C9111976616770608F463
:100170003B01BD0112960D90BC91A02DB4CF6091B2
:100180006E1870916F1868157905E9F4681679068C
:10019000D0F440910002509101024115510541F403
:1001A0004DB75EB76091040270910502461B570B74
:1001B000E417F507A8F4F0936F18E0936E18F901AF
:1001C000918380830BC012DE7C01009749F0A80167
:1001D000BE014CD0CE01A2DEC70104C0CE0102C0D8
:1001E00080E090E0DF91CF911F910F91FF90EF9011
:1001F000DF90CF90BF90AF909F908F907F906F9047
:10020000089581E090E0F894F4C46627772783C2CC
:100210001F93FC0199278827BC01E89411911032A3
:10022000E9F3193010F01E30C8F31B3249F01D32CB
:1002300041F4689405C08DD0610F711D811D911D21
:10024000119110531A30B8F33EF490958095709543
:1002500061957F4F8F4F9F4F1F91089591119EC4BD
:10026000803219F089508550D0F70895FB01DC01E8
:1002700002C001900D9241505040D8F70895FB0103
:10028000DC0101900D920020E1F70895FB01DC01F3
:100290004150504030F08D910190801919F40020A8
:1002A000B9F7881B990B0895FB01DC0141505040C0
:1002B00048F001900D920020C9F701C01D924150F5
:1002C0005040E0F70895FB0151915523A9F0BF017B
:1002D000DC014D9145174111E1F759F4CD01019031
:1002E000002049F04D9140154111C9F3FB01411126
:1002F000EFCF81E090E0019708954532510518F461
:10030000423008F004C0FB011082CB010895BB27E6
:100310004A3031F4992322F4BDE2909581959F4FA4
:100320004FC02532310518F4223008F004C0FA011C
:100330001082CA010895BB272A3051F4992342F450
:10034000BDE290958095709561957F4F8F4F9F4F3F
:1003500016C0592F482F372F262F660F771F881F5B
:10036000991F660F771F881F991F620F731F841FC5
:10037000951F660F771F881F991F0895BB27FA01E5
:10038000A62F6217710581059105330B30FB66F0CE
:10039000AA27660F771F881F991FAA1FA21710F0A0
:1003A000A21B63953850A9F7A05DAA3308F0A95D98
:1003B000A19336F7B111B1931082CA010AC4BB27C9
:1003C000FB015527AA27880F991FAA1FA41710F011
:1003D000A41B83955051B9F7A05DAA3308F0A95D1D
:1003E000A193009779F7B111B1931192CB01F1C3A9
:1003F000F999FECF92BD81BDF89A992780B50895ED
:10040000262FF999FECF1FBA92BD81BD20BD0FB630
:10041000F894FA9AF99A0FBE019608956F927F9216
:100420009F92AF92BF92CF92DF92EF92FF920F9383
:100430001F93CF93DF93CDB7DEB729970FB6F8940C
:10044000DEBF0FBECDBF6A01B22E102F0C3320F4D9
:10045000FF24F394F00E02C04CE3F42E0F2D27E09E
:10046000AE014F5F5F4FC2D27981272F29702130B3
:1004700031F0E1FC06C0E0FC06C060E005C06DE2C2
:1004800003C06BE201C060E2AE2DA07173FF36C005
:10049000662311F084E001C083E08B1510F4B81AD4
:1004A00001C0B12CA1110BC0F6018B2D90E2882365
:1004B00019F091938150FBCFCB0CD11CB12C66234A
:1004C00031F0F601608396012F5F3F4F6901C6014D
:1004D0000396E2FE05C02EE4F601208331E404C059
:1004E0002EE6F601208331E631832283FC012B2D99
:1004F00030E22223F1F131932150FBCF72FF40C053
:10050000662311F084E001C083E08B1510F4B81A63
:1005100001C0B12CA1110BC0F6018B2D90E28823F4
:1005200019F091938150FBCFCB0CD11CB12C6623D9
:1005300031F0F601608396012F5F3F4F6901C601DC
:100540000396E2FE07C029E4F60120832EE421830E
:1005500026E406C029E6F60120832EE6218326E65E
:100560002283FC012B2D30E2222319F031932150FC
:10057000FBCFFC01EB0DF11D10828EEF9FEFB7C09A
:10058000B1E0611101C0B0E04B2F50E01816190620
:1005900024F49C012F5F3F4F02C021E030E0240F84
:1005A000351F112329F0412F50E04F5F5F4F02C0EC
:1005B00040E050E0420F531F2B2D30E0421753070D
:1005C00014F4B41A01C0B12C2E2D287159F4F6017F
:1005D0002B2D30E2222319F031932150FBCFCB0C8D
:1005E000D11CB12CBB2331F0F601608396012F5F43
:1005F0003F4F6901A1110BC0F6012B2D30E32223DF
:1006000019F031932150FBCFCB0CD11CB12CF80E3B
:100610000A81372F3071A32E74FF03C0013309F410
:10062000FA941F142CF42F2D293018F028E001C063
:1006300021E0682F392F97FF02C060E030E0462F9D
:10064000532F612C712C3EE2932EBC01621B710969
:100650009B01DC01A41BB50BE1E0F0E0EC0FFD1FFA
:10066000AE0FBF1FE12EF12CF194E194F1084F3F42
:10067000FFEF5F0731F4F6019082B6016F5F7F4FA5
:100680006B01841795074CF02417350734F4BD012E
:10069000660D771DFB01118101C010E34150510926
:1006A000FFEF6F1A7F0AB6016F5F7F4F4E155F0530
:1006B00024F0F60110836B01DACF4817590739F49B
:1006C000063320F4053319F4A11001C011E3F6013B
:1006D0001083FB018B2D90E2882319F091938150B8
:1006E000FBCFFB01EB0DF11D108280E090E029961D
:1006F0000FB6F894DEBF0FBECDBFDF91CF911F9133
:100700000F91FF90EF90DF90CF90BF90AF909F90B0
:100710007F906F9008958F929F92AF92BF92CF92E9
:10072000DF92EF92FF920F931F93CF93DF938B0192
:100730006115710521F0DB018C9311969C93EC01FE
:100740005E01BFEFAB1ABB0A7501C8808C2D90E02B
:1007500085DD892B11F0E501F3CFEDE2CE1208C063
:100760007E01F2E0EF0EF11CC980DD24D39409C0B4
:100770002BE2C21205C07E0142E0E40EF11CC980EA
:10078000D12CE701219743E050E066E273E0CE010F
:1007900008D2892BB9F4239645E050E061E273E07A
:1007A000CE01FFD1892B09F425960115110519F009
:1007B000D801CD93DC93D11003C160E070E080E8F4
:1007C0009FE707C143E050E06EE173E0CE01E9D15D
:1007D000892B59F40115110509F4F7C0B2E0EB0EAD
:1007E000F11CF801F182E082F0C0F70160E070E0F6
:1007F000CB01C0E0D0E07F01A0EDAA2EAC0C29E037
:100800002A1528F14D2D4260B42E2D2D2870D2FED0
:1008100004C0211124C0219622C021112197A5E0F6
:10082000B0E09B01AC0168DA660F771F881F991F43
:100830006A0D711D811D911D6839A9E97A078A0722
:10084000A9E19A0760F0BD2DB660BB2E08C02EEF5F
:10085000A2120AC0D3FC50C04D2D4860B42E319670
:10086000D701CC90DB2CC7CF2C2D2F7D253409F060
:1008700043C0A081AD3241F4BD2DB061DB2E7F01BC
:1008800022E0E20EF11C0CC07F01AB3231F04FEFE1
:10089000E41AF40A21E030E006C0A2E0EA0EF11CFE
:1008A000A18122E030E0A053AA3018F0E21AF30A46
:1008B00023C0F70120E030E02038BCE03B075CF4C7
:1008C000A901440F551F440F551F240F351F220F38
:1008D000331F2A0F311DAF014F5F5F4F7A01A08197
:1008E000A053AA3010F4FA01E7CFD4FE03C031952B
:1008F00021953109C20FD31FD1FE09C00115110581
:1009000031F0E1E0EE1AF108D801ED92FC920E947C
:100910005F7B2D2D2370233019F04B015C0106C045
:100920004B015C01B7FAB094B7F8B09420E030E026
:10093000A901C501B4010E94917A882309F43DC040
:10094000D7FF06C0D195C195D1090DE313E002C0D0
:1009500005E513E06801B8E1CB1AD10890E2E92E71
:10096000F12CCE15DF056CF0F801259135914591FC
:100970005491C501B40139D84B015C01CE19DF098E
:10098000F0CF04501109F594E7940C151D0549F7B3
:100990008A2D880F8B2D881F8F3F49F020E030E093
:1009A000A901C501B4010E94917A811106C082E2B9
:1009B00090E09093731880937218C501B40109C038
:1009C00060E070E080E89FEF04C060E070E080ECE1
:1009D0009FE7DF91CF911F910F91FF90EF90DF90F4
:1009E000CF90BF90AF909F908F900895283008F0DF
:1009F00027E03327DA01990F311D87FD91600096BA
:100A00006105710539F432602E5F3D9330E32A951C
:100A1000E1F708959F3F30F080387105610509F0D6
:100A20003C5F3C5F3D93913008F08068911DDF93FF
:100A3000CF931F930F93FF92EF92192F987F969564
:100A4000E92F96959695E90FFF27ED54FC4F9927CE
:100A50003327EE24FF24A701E701059008940794AB
:100A600028F4360FE71EF81E491F511D660F771F29
:100A7000881F991F0694A1F70590079428F4E70EA4
:100A8000F81E491F561FC11D770F881F991F661F2B
:100A90000694A1F70590079428F4F80E491F561FF5
:100AA000C71FD11D880F991F661F771F0694A1F7D6
:100AB0000590079420F4490F561FC71FD81F990FA0
:100AC000661F771F881F0694A9F7849110951770E9
:100AD00041F0D695C79557954795F794E7941A95A1
:100AE000C1F7E9E5F3E068941590159135916591AA
:100AF000959105907FE27395E118F10A430B560B2F
:100B0000C90BD009C0F7E10CF11E431F561FC91FC6
:100B1000D01D7EF4703311F48A95E6CFE89401502D
:100B200030F0080F0AF40027021708F4202F23954D
:100B3000022F7A3328F079E37D932A95E9F710C0E4
:100B40007D932A9589F6069497956795379517951D
:100B50001794E118F10A430B560BC90BD00998F012
:100B600023957E9173957A3308F070E37C9320137C
:100B7000B8F77E9170617D9330F0839571E37D933A
:100B800070E32A95E1F71124EF90FF900F911F91E8
:100B9000CF91DF91992787FD909508959927882710
:100BA0000895FB01DC014150504088F08D91813463
:100BB0001CF08B350CF4805E659161341CF06B3554
:100BC0000CF4605E861B611171F3990B0895881B0C
:100BD000FCCFDC01FC01672F71917723E1F732979D
:100BE00004C07C916D9370836291AE17BF07C8F308
:100BF000089514E0CEE5D4E000E005C02297010995
:100C0000FE010BBF89D8C036D10780E00807B1F7D5
:040C1000F894FFCF86
:100C14000000741880000100000000002041000062
:100C2400F041A4707D3FCDCC2C400AD78B4000808E
:100C34003B450000803F9A99F93F0AD7C3BF6666D7
:100C4400A63F0700A16733BD7C8C01000100008032
:100C540040643B5F3E21B0B23E278826400000A896
:100C64004162BE3C3993522A409352AA4017D9009C
:100C7400418C968141B73AC9418B899D3E0000A0C1
:100C8400410000204200007042133BF142ECC43AA0
:100C9400433F00566F6C74616765000000000000FC
:100CA400000000000000000054656D702B48756D55
:100CB4000000000000000000000000000049522075
:100CC400466C616D6500000000000000000000003B
:100CD40000004761730000000000000000000000F5
:100CE4000000000000000070480000000000000048
:100CF4000000000000000000000000005475726253
:100D040069646974790000000000000000000000BC
:100D140000434F320000000000000000000000000B
:100D24000000000000004F3200000000000000003E
:100D3400000000000000000000000049522054653B
:100D44006D700000000000000000000000000000C2
:100D5400536F756E64000000000000000000000086
:100D64000000000000504D000000000000000000E2
:100D740000000000000000000000434834000000B0
:100D8400000000000000000000000000000000411E
:100D94006C636F686F6C00000000000000000000CE
:100DA40000000000434F00000000000000000000AD
:100DB40000000000000000000048320000000000B5
:100DC40000000000000000000000000000004F7A56
:100DD4006F6E6500000000000000000000000000CD
:100DE4000000004832530000000000000000000032
:100DF40000000000000000004E4833000000000026
:100E040000000000000000000000000000200000BE
:100E140000000000000000000000000000000000CE
:100E2400000020000000000000000000000000009E
:100E34000000000000000055560000000000000003
:100E44000000000000000000000000000800010095
:100E54000200030004000500060008000800080062
:100E64003700380039003F003E003D0011001000FB
:100E7400380039003D003D0008003E0038003700CE
:100E840039002E3032342F31333531323341343559
:100E94003642373839432A302344640000001804AA
:100EA40008101C0000000100007544008089440102
:100EB400202020202020202020202020202020202E
:100EC4000042543A005665723A00303A536F756ED8
:100ED40064204C6576656C2A00303A536F756E64F5
:100EE400204C6576656C00313A54656D7020487508
:100EF4006D696469747900323A54656D702050727A
:100F040065737375726500323A616E642048656971
:100F140067687400333A4C6967687420496E742EAC
:100F240000343A495220466C616D6500353A476198
:100F340073204C6576656C00363A4D61676E657456
:100F44006963206669656C6400373A4952205465C8
:100F54006D702A00373A49522054656D7000383A52
:100F640070482076616C756500393A496E636C2E61
:100F740020616E672E00393A6F722033442061631A
:100F840063656C2E0044303A566F6C74616765007B
:100F940044313A5475726269646974790044323A2E
:100FA400504D28313A322E353A3130292A00443214
:100FB4003A504D28313A322E353A313029004433F3
:100FC4003A434F3220636F6E632E0044343A4F32FB
:100FD40020636F6E632E0044353A555620496E7473
:100FE400656E736974790044423A5265736574207E
:100FF4004C6F676765720044433A436C65617220C5
:101004004C4344002A3A546869732048656C700064
:10101400233A53686F77204C4344006F4320413D8B
:10102400004320006E6F20484D4335383833206D1F
:1010340061676E657469632073656E736F72202EC9
:101044002E2E20436865636B20776972696E672171
:10105400002D2D2D2D204D61676E6574696320531D
:10106400656E736F72202D2D2D2D2D2D2D2D2D2D73
:101074002D2D2D2D2D2D2D2D2D2D0053656E736FA2
:10108400723A202020202020200044726976657264
:10109400205665723A20202000556E6971756520CE
:1010A40049443A20202020004D61782056616C7517
:1010B400653A2020202000206D47004D696E20569F
:1010C400616C75653A20202020005265736F6C7541
:1010D40074696F6E3A202020002D2D2D2D2D2D2D7D
:1010E4002D2D2D2D2D2D2D2D2D2D2D2D2D2D2D2D2C
:1010F4002D2D2D2D2D2D2D2D2D2D2D2D2D00436FF1
:101104006D706173733A2000286465672920004E6E
:1011140020005320005700482D6669656C643A200E
:101124002800296D4700203D3E000A3E00482D66F8
:1011340069656C643D00536561726368204469723B
:10114400656374696F6E00482D6669656C64004C54
:101154006F6767657220446972656374696F6E00B6
:101164004C6F6767657220446972656374696F6E5A
:101174003A20004D6561737572652074656D703F2A
:10118400004D656173757265206761733F004D6939
:10119400737320796F7521006F430049742773209E
:1011A4007665727920686F74212000497427732052
:1011B400717569746520686F7421004973206169D1
:1011C400722D636F6E64206F6E3F0054656D7020E6
:1011D40069732066696E6521004974277320746FF2
:1011E4006F20636F6F6C21004F6666206169722DFA
:1011F400636F6E6421006F4320483D004E6F20539F
:10120400656E736F722100234E6F2073656E736F6A
:101214007220666F722074656D7020262068756D6B
:101224006964697479210049742773207665727939
:1012340020686F7421006761696E735F6F726967FC
:101244005B5D3A00736574206761696E735B5D3A38
:101254000058595A20434F554E54533A2000585978
:101264005A2047733A200067657454617054687259
:101274006573686F6C6428293A2000676574417847
:1012840069734F66667365742826782C2026792C3A
:1012940020267A293A200067657454617044757277
:1012A4006174696F6E28293A2000676574446F750C
:1012B400626C655461704C6174656E637928293A77
:1012C4002000676574446F75626C6554617057697A
:1012D4006E646F77282920006765744163746976AA
:1012E4006974795468726573686F6C642829200086
:1012F400676574496E616374697669747954687258
:101304006573686F6C642829200067657454696D7F
:1013140065496E616374697669747928293A200095
:101324006765744672656546616C6C546872657372
:10133400686F6C6428293A20006765744672656595
:1013440046616C6C4475726174696F6E28293A2029
:10135400006973416374697669747958456E616292
:101364006C656428293A200069734163746976695D
:10137400747959456E61626C656428293A20006964
:101384007341637469766974795A456E61626C65F8
:101394006428293A20006973496E61637469766927
:1013A400747958456E61626C656428293A20006935
:1013B40073496E616374697669747959456E6162C3
:1013C4006C656428293A20006973496E6163746905
:1013D400766974795A456E61626C656428293A208D
:1013E4000069734163746976697479416328293AA1
:1013F4002000676574537570707265737342697405
:1014040028293B20747275653F2000676574537505
:1014140070707265737342697428293B2066616C2D
:1014240073653F2000697354617044657465637427
:10143400696F6E4F6E5828293B20747275653F2082
:10144400006973546170446574656374696F6E4FA9
:101454006E5828293B2066616C73653F20006973D0
:10146400546170446574656374696F6E4F6E592876
:10147400293B20747275653F200069735461704480
:101484006574656374696F6E4F6E5928293B2066D5
:10149400616C73653F2000697354617044657465C1
:1014A4006374696F6E4F6E5A28293B207472756598
:1014B4003F20006973546170446574656374696F97
:1014C4006E4F6E5A28293B2066616C73653F20007D
:1014D40069734163746976697479536F757263656E
:1014E4004F6E5828293A2000616363656C2E697336
:1014F4004163746976697479536F757263654F6E6D
:101504005928293A2000616363656C2E697341632D
:10151400746976697479536F757263654F6E5A286E
:10152400293A2000616363656C2E697354617053BA
:101534006F757263654F6E5828293A2000616363A2
:10154400656C2E6973546170536F757263654F6E69
:101554005928293A2000616363656C2E69735461CC
:1015640070536F757263654F6E5A28293A20006173
:101574006363656C2E697341736C65657028293AE1
:101584002000616363656C2E69734C6F77506F77CD
:10159400657228293A2000676574526174652829A8
:1015A4003A20332E31343135393F00676574496E42
:1015B40074657272757074536F7572636528293A15
:1015C4002000676574496E74657272757074536F28
:1015D400757263652831293A2000676574496E7411
:1015E4006572727570744D617070696E6728312907
:1015F4003A20006973496E74657272757074456E31
:1016040061626C65642831293A200067657453650A
:101614006C665465737442697428293A20003E61EB
:1016240028782C792C7A292F673A007320613D00A1
:101634002067007320496E636C2E20616E672E282C
:10164400782079207A292F6465673A200073204135
:101654006E676C6573002F007320613A0067200089
:101664004D6561737572696E672E2E004952205460
:10167400656D7065726174757265002349522054FA
:10168400656D70204661696C6564212000495220B3
:1016940054656D703D00234E6F2054422073656E77
:1016A400736F723F0054423D004E5455005600453E
:1016B40072726F72206E756D62657220666F722031
:1016C40074686520617272617920746F206176722A
:1016D4006167696E67212F6E0070483D00234E6F6D
:1016E4002070482073656E736F722100434F32205F
:1016F400436F6E6300434F323D0070706D0044755C
:10170400737420436F6E6300447573742070696E44
:101714003D0044743D007063732F4C00206442000C
:10172400533D00206442200020572F6D0055562061
:10173400496E742E0055563D005E3220004100561D
:101744002000476173206C6576656C3D00476173CA
:10175400004C6576656C3D00466C616D65204952B0
:1017640000495220466C616D652000566F6C25005F
:101774005343493531005345533668356E00504D57
:10178400313A322E353A313000206E672F4C0050FA
:101794004D28312E302C322E352C3130293D00236A
:1017A4004E6F2073656E736F7220666F7220504D9A
:1017B400210057656C636F6D6520746F2045645517
:1017C400484B0053656E736F7220736C6F742061A5
:1017D4006E6420747970653A00203D2023004564CE
:1017E40055484B205345534C6F6767657200206D15
:1017F4006F62696C65206C6F6767657220737461D2
:101804007274656420616E6420726561647921007C
:10181400536F756E64204C6576656C2073656E73CA
:101824006F7220666F756E6400504D322E352073D2
:10183400656E736F72206C696B656C7920666F7569
:101844006E640049522054656D702073656E736F29
:101854007220666F756E6400234572726F723A70FF
:101864007265737375726520424D503038352C2083
:10187400636865636B20776972696E67210023531F
:101884006561206C6576656C20502863616C632902
:101894003D002343616C6962726174696F6E20500C
:1018A400726573737572653D00234E6F2073656EA8
:1018B400736F72210073657269616C3A200042543F
:1018C4003A200053004C6967687420496E74656E51
:1018D4007369747900206C78004C3D00206C78208A
:1018E400007265706C6965733D00496E76616C6960
:1018F40064206B657921006B6579323D002D3500DC
:101904002D34002D33002D32002D31002D37002DC4
:1019140038002D39002D3130002D313100616E6FCA
:101924007468657220495220696E7075743D007345
:101934006574005345540023506172616D6574658C
:10194400727300235365612D6C6576656C2050724B
:101954006573737572653D00234D61676E657469C7
:1019640063206465636C696E6174696F6E20416E97
:10197400676C653D002354757262696469747920EB
:10198400766F6C74616765733A005640004E545527
:101994002C20004E5455200023426C7565746F6FE3
:1019A4007468204E616D653D0023434F32207A6593
:1019B400726F20766F6C74616765280070706D2992
:1019C4003D0023434F32206D617820766F6C746143
:1019D40067652028002343616C69627261746564E1
:1019E400204F3220636F6E63203D0020766F6C259C
:1019F4002000235556207A65726F20766F6C7461CF
:101A04006765203D0023736C6F74202300292069CF
:101A14007320002354696D6520696E746572766164
:101A24006C3D002354696D65206475726174696F3F
:101A34006E3D00476976656E20736561206C65763E
:101A4400656C20503D00506120697320756E6C698F
:101A54006B656C792100536561206C6576656C203B
:101A6400503D002068506100736C6F743D00534C0E
:101A74004F543D0072736C6F740052534C4F5400BA
:101A840076657273696F6E0056455253494F4E0026
:101A940056657273696F6E3A200042543D00627459
:101AA4003D0041542B4E414D450050494E3D0041AF
:101AB400542B50494E007068007048005048007024
:101AC40068340070483400566F6C74616765287020
:101AD400483D34293A007068313000704831300094
:101AE400566F6C746167652870483D3130293A003F
:101AF40074696D65693D0074696D65643D005442A7
:101B040031007462310054757262696469747920B9
:101B14004C6F776572204C696D69742056313A2098
:101B240000235442285631293D004F3243414C0092
:101B34006F3263616C004F322063616C6962726161
:101B440074696F6E3A2000234F3220766F6C253D06
:101B540000434F325A00636F327A00434F32207A87
:101B640065726F20766F6C7420280070706D293A4E
:101B7400200023434F3220566F3D00434F324D0027
:101B8400636F326D00434F32204D415820766F6CA5
:101B94007420280023434F3220566D3D0055565A79
:101BA4000075767A00544249007462690054757273
:101BB400626964697479204C6F776572204C696D31
:101BC40069742056696E663A200023544228566987
:101BD4006E66293D0054424C0074626C0054757268
:101BE400626964697479204C6F776572204C696D01
:101BF40069743A200020766F6C746167653D002338
